:100000000C94CB1D0C940B1E0C940B1E0C940B1E0D
:100010000C940B1E0C940B1E0C940B1E0C940B1EBC
:100020000C940B1E0C940B1E0C940B1E0C940B1EAC
:100030000C940B1E0C940B1E0C940B1E0C940B1E9C
:100040000C940B1E0C9489930C940B1E0C940B1E99
:100050000C940B1E0C945F860C940B1E0C949875DC
:100060000C940B1E0C944B360C9441360C940B1EC6
:100070000C940B1E0C940B1E0C940B1E0C940B1E5C
:100080000C940B1E0C940B1E0C940B1E0C940B1E4C
:100090000C940B1E0C940B1E0C940B1E0C940B1E3C
:1000A0000C940B1E0C940B1E0C940B1E0C940B1E2C
:1000B0000C940B1E0C940B1E0C940B1E0C940B1E1C
:1000C0000C940B1E0C940B1E0C940B1E0C94CE283F
:1000D0000C9498280C940B1E0C940B1E0C940B1E65
:1000E0000C940B1E084AD73B3BCE016E84BCBFFD6F
:1000F000C12F3D6C74319ABD56833DDA3D00C77FF8
:1001000011BED9E4BB4C3E916BAAAABE0000008090
:100110003F05A84CCDB2D44EB93836A9020C50B91F
:10012000918688083CA6AAAA2ABE000000803F004B
:100130000C9445730C94A4690C940DC80C94D46A67
:100140000D94CA1B0C9418EC0D948A180C9488DD3D
:100150000C949C4D0C940F370C94D36A0D94AE18EC
:100160000C947F290C94AA740C940C290C948F4D38
:100170000C948E730C946E4C0C94F7DC0C94C46944
:100180000C94C9690D94A5180C94ED730C94E53684
:100190000C9464290C941BEC0D9412170C9448DDFC
:1001A0000C94DD360C94E9360C9407EC0C9479C76A
:1001B0000C940CEC0C94ED270C946CDF0C94C92778
:1001C0000C945D4C0C9457DF0C943FDD0C946B74D5
:1001D0000C946A4C0C94D2730C94E8C70C9470295C
:1001E0000D9493180C947B4C0C9412EC0D94EC270A
:1001F0000C94C7360D943C170C94E4C60C9433DD74
:100200000C94BC690C94CE690C940FEC0C942EC722
:100210000C94A5270D94DD150D94091C0C94A727AB
:100220000C94674C0C9421EC0C9493690C94684DDD
:100230000C94EF270C94B8360C94164D0C9430DDCA
:100240000C94EB270D94D2180C9415EC0C94C72742
:100250000C94A3270D943D180C94594C0C949B6955
:100260000C9424EC0C94224D0C942ADD0C94E04C5C
:100270000C94A8690C94FC360C944A290C949EDFCB
:100280000C94D6360D94151C0C94ED360C94D64C6B
:100290000C9436DD0C94AE690C9483270C94CD74C9
:1002A0000C9442DD0C94784C0C94B6690C94AF4CD1
:1002B0000C94214C0C94C0690C94E6720C943CDDB7
:1002C0000D94FA1B0C94FC4C0C943B290C945A4D45
:1002D0000D94C5180C941C4C0C9492290D941E1866
:1002E0000D940A180C94C9720C94B2690C942DDD0B
:1002F0000C94824D0C94F1360C94D2DD0C943E4D4E
:100300000C9459290C941EEC0D949E150C949EC7C8
:100310000C9463270D94D3170D94C7180C94893649
:100320000C94516A0C94304D0D94AA170C94976953
:100330000C94714C0C9468290C942DDF0D94E717E4
:100340000C947D740D948E160C94D6DD0C944F4C49
:100350000C94CB270C94644C0D94301C0C944C4D95
:100360000C949E690C946C290D947F180C94CA69A6
:100370000C94564C0C9407370C9445DD0D94D61B09
:100380000C9481270C94A2C60C94EE4C0C94782902
:100390000C9409C70C9427EC0C94754D0C9432C83E
:1003A0000C94534C0C940A4D0C948F690D94211CA1
:1003B0000C948A290C94604C0C94744C0C944C4C06
:1003C0000C94E1360C9460290D94CE270C94F536EC
:1003D0000C942AEC0C9489690C94C3C70C9474296E
:1003E0000C9439DD0D94C1180D94B7180D949C1818
:1003F0000C9457274E414E494E495459494E46CDCB
:10040000CCCC3D0AD7233C17B7D13877CC2B3295CB
:1004100095E6241FB14F0A000020410000C84200A9
:10042000401C4620BCBE4CCA1B0E5AAEC59D740073
:10043000407A10F35A00A0724E18090010A5D4E8B3
:100440000000E87648170000E40B54020000CA9A46
:100450003B000000E1F50500008096980000004098
:10046000420F000000A086010000001027000000DD
:1004700000E803000000006400000000000A000023
:100480000000000100000000002C76D888DC674FD7
:100490000823DFC1DFAE59E1B1B796E5E3E453C607
:1004A0003AE651997696E8E6C28426EB898C9B62FF
:1004B000ED407C6FFCEFBC9C9F40F2BAA56FA5F4A9
:1004C00090055A2AF75C936B6CF9676DC11BFCE0D1
:1004D000E40D47FEF520E6B500D0ED902E03009424
:1004E0003577050080841E080000204E0A000000B9
:1004F000C80C333333330F986E12831141EF8D21C3
:1005000014893BE65516CFFEE6DB18D1844B381B29
:10051000F77C1D901DA4BBE424203284725E2281EE
:1005200000C9F124ECA1E53D275A5F53544F505FB9
:1005300050494E005A5F535445505F50494E005A3F
:100540005F4D494E5F50494E005A5F454E41424C07
:10055000455F50494E005A5F4449525F50494E0032
:10056000595F53544F505F50494E00595F535445A3
:10057000505F50494E00595F4D494E5F50494E0003
:10058000595F454E41424C455F50494E00595F44CA
:1005900049525F50494E00585F53544F505F504985
:1005A0004E00585F535445505F50494E00585F4DC0
:1005B000494E5F50494E00585F454E41424C455FA1
:1005C00050494E00585F4449525F50494E005355C0
:1005D00049434944455F50494E00534552564F33B5
:1005E0005F50494E00534552564F325F50494E00BE
:1005F000534552564F315F50494E00534552564F66
:10060000305F50494E00534453530053445F4445B8
:10061000544543545F50494E004D4F534645545F37
:10062000435F50494E004D4F534645545F425F5023
:10063000494E004D4F534645545F415F50494E006F
:1006400054454D505F305F43535F50494E004C4519
:10065000445F50494E004845415445525F4245442D
:100660005F50494E004845415445525F305F504904
:100670004E0046494C5F52554E4F55545F50494EBF
:100680000046414E5F50494E0045315F535445503E
:100690005F50494E0045315F454E41424C455F50E9
:1006A000494E0045315F4449525F50494E00453143
:1006B0005F43535F50494E0045305F535445505F90
:1006C00050494E0045305F454E41424C455F5049D0
:1006D0004E0045305F4449525F50494E0042454507
:1006E0005045525F50494E004156525F53535F5040
:1006F000494E004156525F53434B5F50494E0041B3
:1007000056525F4D4F53495F50494E004156525F1C
:100710004D49534F5F50494E0054454D505F42453F
:10072000445F50494E0054454D505F315F50494E33
:100730000054454D505F305F50494E0046494C577C
:10074000494454485F50494E00545844320052586E
:1007500044320054584430005258443000434F4D06
:100760004D554E49434154494F4E004452595255FC
:100770004E004552524F525300494E464F0045439A
:10078000484F004572726F722077726974696E67A4
:1007900020746F20454550524F4D210A00363726B0
:1007A000033C3D380E2E303E121A1C180A4309082D
:1007B00044000153544F505045442E20005072695C
:1007C0006E7465722073746F7070656420647565F3
:1007D00020746F206572726F72732E2046697820C4
:1007E000746865206572726F7220616E6420757323
:1007F00065204D39393920746F20726573746172C8
:10080000742E202854656D70657261747572652050
:1008100069732072657365742E2053657420697442
:100820002061667465722072657374617274696E9A
:1008300067290A004E6F20436865636B73756D20EE
:1008400077697468206C696E65206E756D6265727B
:100850002C204C617374204C696E653A20004E6FF9
:1008600020436865636B73756D2077697468206CCD
:10087000696E65206E756D6265722C204C617374B3
:10088000204C696E653A2000636865636B73756D13
:10089000206D69736D617463682C204C61737420E2
:1008A0004C696E653A20004C696E65204E756D622C
:1008B0006572206973206E6F74204C617374204CD4
:1008C000696E65204E756D6265722B312C204C610E
:1008D0007374204C696E653A20004D3131300053FD
:1008E000657269616C20737461747573206D6973CE
:1008F0006D617463680A00776169740A005344206B
:1009000072656164206572726F720A002121204B4A
:10091000494C4C2063617573656420627920746F63
:100920006F206D75636820696E61637469766520F8
:1009300074696D65202D2063757272656E74206315
:100940006F6D6D616E643A2000486F74656E64204F
:1009500049646C652054696D656F757400486F74E7
:10096000656E642049646C652054696D656F7574AB
:100970000A003D3D6F6E46696C616D656E7452751F
:100980006E6F75743D3D007061757365004D363056
:1009900030002066696C616D656E745F72756E6F94
:1009A0007574200066696C616D656E745F72756E3A
:1009B0006F757420540046696C616D656E74527574
:1009C0006E6F75742054004D3130303053006275B5
:1009D00073793A2070617573656420666F7220695F
:1009E0006E7075740A00627573793A207061757360
:1009F000656420666F7220757365720A0062757394
:100A0000793A2070726F63657373696E670A0025A7
:100A1000533A202553002A2A2A6B696C6C2A2A2A09
:100A200000706F7765726F6666004B494C4C4544A9
:100A30002E20005072696E7465722068616C746556
:100A4000642E206B696C6C28292063616C6C656472
:100A5000210A006563686F3A004572726F723A004E
:100A600042696C696E656172204C6576656C696E71
:100A70006720477269643A0A002F2F616374696FB7
:100A80006E3A006E6F74696669636174696F6E2097
:100A90000070726F6D70745F00656E6400486F74F3
:100AA000656E6420746F6F20636F6C640A00536519
:100AB0006E64204D31303820746F20726573756D0F
:100AC000650A00496E736572742066696C616D65B4
:100AD0006E7420616E642073656E64204D31303811
:100AE0000A0052656865617420446F6E6500526546
:100AF00068656174696E672E2E2E005265686561A7
:100B000074004865617465722054696D656F757411
:100B10000053656E64204D31303820746F20686555
:100B20006174206E6F7A7A6C650A004E6F7A7A6C07
:100B300065205061726B6564007061757365640057
:100B40005061757365004F46460A00466164652032
:100B50004865696768742000426564204C65766565
:100B60006C696E6720004661696C656420746F2053
:100B7000656E61626C6520426564204C6576656CCB
:100B8000696E670A00496E76616C6964206D6573F1
:100B9000682E0A0050726F62696E6720506F696E2E
:100BA000740025532025692F2569002E0A002F0087
:100BB00050726F62696E67206D65736820706F692F
:100BC0006E742000202844525952554E2900473255
:100BD00039204175746F20426564204C6576656CE0
:100BE000696E67003F20284C2C522C462C4229204D
:100BF0006F7574206F6620626F756E64732E0A00C5
:100C00003F2856296572626F7365206C6576656C46
:100C100020696D706C61757369626C652028302D78
:100C200034292E0A00426164205A2076616C756571
:100C30000A004E6F2062696C696E6561722067728E
:100C400069640A0020440020204D323030205300D7
:100C5000202844697361626C6564293A0046696CB6
:100C6000616D656E742073657474696E67730020BE
:100C7000204D3230312058004D617820416363654A
:100C80006C65726174696F6E2028756E6974732F5C
:100C90007332290020204D3230332058004D6178C6
:100CA000206665656472617465732028756E697469
:100CB000732F73290020520020204D3230342050F1
:100CC00000416363656C65726174696F6E2028759D
:100CD0006E6974732F7332292028503C7072696ECC
:100CE000742D616363656C3E20523C726574726161
:100CF00063742D616363656C3E20543C747261764D
:100D0000656C2D616363656C3E29005741524E4905
:100D10004E4721204C6F77205A204A65726B206D18
:100D20006179206C65616420746F20756E77616EE7
:100D3000746564207061757365732E0A0020540019
:100D400020530020204D323035204200416476612E
:100D50006E6365642028423C6D696E5F7365676DE4
:100D6000656E745F74696D655F75733E20533C6D8D
:100D7000696E5F66656564726174653E20543C6DA2
:100D8000696E5F74726176656C5F666565647261D9
:100D900074653E20583C6D61785F6A65726B3E20D9
:100DA000593C6D61785F6A65726B3E205A3C6D619B
:100DB000785F6A65726B3E20453C6D61785F6A655D
:100DC000726B3E290020440020490020204D333022
:100DD00031205000486F74656E64205049440020F3
:100DE000440020490020204D33303420500042651B
:100DF00064205049440050574D3A20202534640067
:100E000050574D3A20202534640050574D3A202049
:100E10002534640050574D3A202025346400505743
:100E20004D3A20202534640050574D3A2020253477
:100E3000640050574D3A20202534640050574D3AF5
:100E400020202534640050574D3A2020253464007A
:100E500050574D3A20202534640050574D3A2020F9
:100E60002534640050574D3A2020253464005057F3
:100E70004D3A20202534640050574D3A2020253427
:100E8000640050574D3A20202534640050574D3AA5
:100E90002020253464003A200020202020434F4D9C
:100EA000002020206E6F6E2D7374616E6461726419
:100EB0002050574D206D6F646500202020636F6DBA
:100EC0007061726520696E746572727570742065E8
:100ED0006E61626C6564002020206F766572666CBE
:100EE0006F7720696E7465727275707420656E61BB
:100EF000626C6564003A20002020202054494D5344
:100F00004B00423A2000202020205443435200410D
:100F10003A2000202020205443435200202020204B
:100F200043533A20002020202057474D3A200050BC
:100F3000574D3A20202534640050574D3A20202543
:100F400034640047004800000088008A008C00B329
:100F500000B400000098009A009C00A800AA00AC11
:100F60000028012A012C012020202054494D4552FF
:100F700000440045006E00800081006F00B000B1A9
:100F8000007000900091007100A000A1007200208C
:100F9000012101730020697320616C736F207469F3
:100FA000656420746F20746869732070696E0054E2
:100FB000494D45523143000A202E002020002020B8
:100FC000506F72743A200020202000202020416EB3
:100FD000616C6F6720696E203D2025356C64003C94
:100FE000756E757365642F756E6B6E6F776E3E00F0
:100FF0002028412532642920200025336420005018
:10100000494E3A20004F7574707574203D20004998
:101010006E70757420203D2000416E616C6F6720FA
:10102000696E203D2025356C640070726F746563B5
:101030007465642000202841253264292020002581
:101040003364200050494E3A2000580700015307EE
:1010500001014E071101490710013C073B00310710
:10106000430026074500190744000C073201FF061C
:101070003301F3063401E8063501DD062501D20609
:101080001C01C4061801B8061A01AE062C01A306FD
:10109000220195061E0189062401810609017206B6
:1010A000020165060A01560608014E060D014006BA
:1010B000420133060A0126060701190608010B063C
:1010C000310106063501FB050B01F0050601E505BA
:1010D0000501DA050401CE050C01C4053701B70589
:1010E0002601AD050301A2053601970503018D0513
:1010F0003D018005380176050E016B053C01600558
:101100000E015605300149053E013F051201340527
:101110002E0129051201446F6E652E0A0050756C70
:1011200073696E6720202000556E746F7563686563
:10113000642000534552564F206E6F7420736574BF
:101140002075702E0A004D34332057616974204396
:10115000616C6C6564004D343320576169742043C1
:10116000616C6C6564005761746368696E672070B8
:10117000696E730A0064697300656E0061626C6574
:10118000640A00656E6473746F70206D6F6E6974AD
:101190006F72200020580020204D61783A200020F6
:1011A0000020204D696E3A2000203B200020204D79
:1011B0003231312053003F43616E6E6F742077727D
:1011C00069746520746F20494E5055540A00496E69
:1011D00076616C69642050696E204D6F64650A0009
:1011E000203B0020550020204D363033204C004657
:1011F000696C616D656E74206C6F61642F756E6CC7
:101200006F6164004D323453256C6454256C640066
:101210004739322E3945257300473146256400474A
:10122000315A2573463630300047315825735925D9
:10123000734633303030004D3130365025695325F8
:1012400069004D313039532569004D323030442525
:1012500073004739322E395A2573004D34323053DA
:1012600025635A25730047323852305859004731A8
:101270005A257346363030004739322E395A257395
:10128000004739322E394530004D31303953256908
:10129000004D313930532569004D34323020533000
:1012A000205A30003D3D4F6E506F7765724C6F7322
:1012B00073526573756D653D3D00203B2000202015
:1012C0004D343133205300506F7765722D6C6F733E
:1012D00073207265636F76657279004F4646004FE2
:1012E0004E00203B20486F73742068616E646C6907
:1012F0006E672000203B204D6F646520006D6D00FF
:10130000203B2044697374616E6365200046696CFC
:10131000616D656E742072756E6F757420003B2070
:101320000020496E76616C6964206578747275641A
:101330006572200047322F4733206261642070615C
:1013400072616D65746572730A00536C6565702E09
:101350002E2E005A2050726F6265205061737420E7
:101360004265640A005A2050726F626520506173B2
:101370007420426564004732384C3000205A3A20CD
:101380000020593A200042656420583A20004D65FB
:10139000736820706F696E74206F7574206F66209B
:1013A00072616E67650A004D302053746F70004D96
:1013B000312053746F7000436C69636B20746F202D
:1013C000526573756D652E2E2E004E6F204D6F7613
:1013D000652E00456E642066696C65206C697374C7
:1013E0000A00426567696E2066696C65206C6973E6
:1013F000740A004E6F206D656469610A005265735E
:10140000756D696E6720534400286E6F2066696CA5
:1014100065290043757272656E742066696C653A61
:1014200020005072696E742074696D653A20000A5C
:1014300053746174733A2046696C616D656E7420F3
:10144000757365643A20002C204C6F6E6765737469
:10145000206A6F623A2000546F74616C2074696D69
:10146000653A200053746174733A20002C20466161
:10147000696C65643A20002C2046696E6973686562
:10148000643A20005072696E74733A20005374619C
:1014900074733A20006F6B006F6666007E077907F1
:1014A00072076B075D0744454255473A004D31319D
:1014B00033205300544D3344203130532050726F49
:1014C000204F46462E002F2F0046523A0020466CF1
:1014D0006F773A200050726F7465637465642050B2
:1014E000696E0A0064697300656E0043290A006131
:1014F000626C656420286D696E2074656D702000D3
:10150000436F6C64206578747275646573206172D2
:10151000652000504944204175746F74756E6500F4
:10152000504944204175746F74756E652066616919
:101530006C65642120426164206865617465722075
:1015400069640A004D34323120696E636F727265CE
:10155000637420706172616D65746572207573616A
:1015600067650A004D65736820706F696E74206F3F
:101570007574206F662072616E67650A004F66663B
:1015800073657473204170706C6965640045727294
:101590003A20546F6F206661722100546F6F20668D
:1015A00061722066726F6D207265666572656E632A
:1015B0006520706F696E740A00454550524F4D208A
:1015C0004F4B0A00496E76616C69642065787472CD
:1015D000756465720A000A20696E6974207A7072F7
:1015E0006F62655F7A6F6666736574203D20003DAB
:1015F0003D6F6E436F6E66696775726174696F6E79
:1016000053746F7265526561643D3D0045455052AB
:101610004F4D20496E697469616C697A65640A008E
:1016200048617264636F6465642044656661756CCB
:10163000742053657474696E6773204C6F616465C0
:10164000640020286D6D2900203B204C6576656C78
:10165000696E67200020204D3432302053004175E0
:10166000746F20426564204C6576656C696E670016
:1016700046696C616D656E742072756E6F7574204D
:1016800073656E736F7200204A0020204732392044
:101690005720490020204D3134392043203B20552C
:1016A0006E69747320696E2043656C736975730A83
:1016B0000054656D706572617475726520556E6950
:1016C0007473002020473231203B004C696E656105
:1016D0007220556E69747300454550524F4D206419
:1016E00061746173697A65206572726F722E0A0087
:1016F00053657474696E6720566F6C756D65204F05
:101700006E203A200053657474696E6720537461CB
:101710006E646279204F6E203A20005365747469BC
:101720006E6720566F6C756D65203A2000536574A6
:1017300074696E6720526F746174696F6E203A200D
:101740000053657474696E67205374616E646279C6
:101750002054696D65203A200053657474696E6782
:10176000205374616E646279203A2000536574746A
:10177000696E67204272696768746E657373203A98
:1017800020004C6F6164696E67204457494E204CBD
:1017900043442073657474696E672066726F6D20B0
:1017A000454550524F4D0A00446973636172646944
:1017B0006E67204457494E204C434420736574742F
:1017C000696E672066726F6D20454550524F4D20FF
:1017D0002D2073657474696E677320766572736902
:1017E0006F6E20696E636F72726563740A0044697C
:1017F0007363617264696E67204457494E204C439D
:10180000442073657474696E672066726F6D20453D
:101810004550524F4D202D2073697A6520696E63C3
:101820006F72726563740A0053746F72656420731B
:10183000657474696E677320726574726965766524
:101840006400290A002062797465733B2063726327
:1018500020002073746F7265642073657474696E00
:101860006773207265747269657665642028004527
:101870004550524F4D20435243204572726F7200C3
:10188000202863616C63756C6174656429210A00AA
:1018900020213D2000454550524F4D2043524320CA
:1018A0006D69736D61746368202D202873746F7285
:1018B00065642920002053697A653A2000496E64E6
:1018C00065783A20000000FA430000FA4300002047
:1018D0004100008C420000A0420000A0420000C86D
:1018E000430080CF43EE020000EE020000640000DF
:1018F000003C000000454550524F4D205665727324
:10190000696F6E204572726F7200204D61726C6952
:101910006E3D563837290A00454550524F4D2076C6
:10192000657273696F6E206D69736D617463682091
:1019300028454550524F4D3D0024F4D43050C38EBD
:1019400020C2A24017828B7011127A910D816CD93E
:101950000AA861E108C7586607615143061E4B5D3E
:1019600005C145A7041A411104093D980371393195
:10197000034036DB0265339102D4305402802E1DC1
:1019800002632CEE01752AC501B028A00110278141
:10199000018F2564012B244B01E0223401AC211F6F
:1019A000018D200D01801FFC00841EED00971DDFBE
:1019B00000B81CD200E61BC600201BBC00641AB293
:1019C00000B219A8000A19A0006A189900D117914D
:1019D0000040178B00B516840031167E00B31579D0
:1019E000003A157300C7146F0058146A00EE1366AE
:1019F000008813630025135E00C7125B006C12574A
:101A00000015125400C111510070114F0021114BEB
:101A100000D61049008D10470046104400021042C5
:101A200000C00F4000800F3E00420F3C00060F3BFD
:101A300000CB0E3800930E37005C0E3500270E34B5
:101A400000F30D3200C10D3100900D3000600D2EFD
:101A500000320D2D00050D2C00D90C2B00AE0C29E9
:101A600000850C29005C0C2700350C27000E0C2685
:101A700000E80B2400C40B2400A00B23007D0B23E3
:101A8000005A0B2100390B2100180B2000F80A1F07
:101A900000D90A1E00BB0A1E009D0A1D00800A1DF7
:101AA00000630A1C00470A1B002C0A1B00110A1ABB
:101AB00000F7091A00DD091900C4091900AB09195A
:101AC00000920917007B091800630917004C0916DA
:101AD0000036091600200916000A091500F5081538
:101AE00000E0081400CC081400B8081400A408147E
:101AF00000900813007D0812006B081300580812AC
:101B000000460812003408110023081100120811C1
:101B10000001081100F0071000E0071000D00710C6
:101B200000C0071000B0070F00A107100091070EBA
:101B30000083070F0074070F0065070E0057070E9C
:101B40000049070E003B070D002E070E0020070D71
:101B50000013070D0006070D00F9060C00ED060D39
:101B600000E0060C00D4060C00C8060C00BC060CF5
:101B700000B0060C00A4060B0099060C008D060BA5
:101B80000082060B0077060B006C060B0061060A4C
:101B90000057060B004C060A0042060A0038060AE7
:101BA000002E060A0024060A001A060A001006097A
:101BB0000007060A00FD050900F4050900EB050908
:101BC00000E2050900D9050900D0050900C705098B
:101BD00000BE050900B5050800AD050800A505090A
:101BE000009C050800940508008C05080084050881
:101BF000007C050800740508006C050700650508F1
:101C0000005D050700560508004E0507004705075B
:101C1000004005080038050700310507002A0507C0
:101C200000230507001C050600160507000F050721
:101C3000000805060002050700FB040600F504077E
:101C400000EE040600E8040600E2040700DB0406D8
:101C500000D5040600CF040600C9040600C304062C
:101C600000BD040600B7040600B1040500AC04067C
:101C700000A6040600A00405009B040600950405C8
:101C800000900406008A040500850405008004060F
:101C9000007A04050075040500700405006B040556
:101CA0000066040500610405005C04050057040596
:101CB00000520405004D04050048040500430405D6
:101CC000003E0404003A0405003504050030040415
:101CD000002C04050027040400230405001E04044E
:101CE000001A04040016040500110404000D040485
:101CF00000090405000404040000040400FC0304BB
:101D000000F8030400F4030400F0030400EC0304EF
:101D100000E8030400E4030400E0030400DC03041F
:101D200000D8030400D4030400D0030400CC03044F
:101D300000C8030300C503030024F404D9201BC416
:101D40000C5C0E9804C4095F0265077101F405F983
:101D500000FB04B30048048700C103690058035521
:101D60000003034500BE023A008402310053022AF8
:101D7000002902250004022000E4011C00C801190A
:101D800000AF0117009801140084011300710110C5
:101D9000006101100051010E0043010D0036010BDE
:101DA000002B010B0020010B00150109000C01099B
:101DB0000003010800FB000800F3000800EB000727
:101DC00000E4000600DE000600D8000600D200068F
:101DD00000CC000500C7000500C2000500BD0004DE
:101DE00000B9000400B5000400B1000400AD000417
:101DF00000A9000400A5000300A20003009F000446
:101E0000009B00030098000300950002009300036C
:101E100000900003008D0002008B00030088000288
:101E2000008600020084000300810002007F00029F
:101E3000007D0002007B00020079000200770001B3
:101E400000760002007400020072000100710002BE
:101E5000006F0002006D0001006C0002006A0001CA
:101E600000690002006700010066000100650001D2
:101E700000640002006200010061000100600001D6
:101E8000005F0002005D0001005C0001005B0001DA
:101E9000005A0001005900010058000100570001DC
:101EA00000560001005500010054000100530000DD
:101EB00000530001005200010051000100500001D8
:101EC000004F0001004E0000004E0001004D0001D7
:101ED000004C0001004B0000004B0001004A0001D3
:101EE00000490001004800000048000100470001CF
:101EF00000460000004600010045000000450001CA
:101F000000440001004300000043000100420000C3
:101F100000420001004100000041000100400001BA
:101F2000003F0000003F0001003E0000003E0001B5
:101F3000003D0000003D0001003C0000003C0000AE
:101F4000003C0001003B0000003B0001003A0000A3
:101F5000003A00010039000000390001003800009B
:101F60000038000000380001003700000037000191
:101F70000036000000360000003600010035000089
:101F8000003500000035000100340000003400007E
:101F90000034000100330000003300000033000172
:101FA0000032000000320000003200010031000069
:101FB000003100000031000100300000003000005E
:101FC00000300001002F0000002F0000002F000053
:101FD000002F0001002E0000002E0000002E000146
:101FE000002D0000002D0000002D0000002D00013C
:101FF000002C0000002C0000002C0000002C000130
:10200000002B0000002B0000002B0000002B000123
:10201000002A0000002A0000002A0000002A000117
:10202000002900000029000000290000002900000C
:1020300000290001002800000028000000280000FE
:1020400000280000002800010027000000270000F1
:1020500000270000002700000027000100260000E4
:1020600000260000002600000026000000260001D7
:1020700000250000002500000025000000250000CC
:1020800000250000002500010024000000240000BD
:1020900000240000002400000024000100230000B0
:1020A00000230000002300000023000000230000A4
:1020B0000023000000230001002200000022000095
:1020C0000022000000220000002200000022000187
:1020D000002100000021000000210000002100007C
:1020E000002100000021000000210001002000006C
:1020F0000020000000200000002000000020000060
:10210000002000000020000000200001001F00004F
:10211000001F0000001F0000001F0000001F000043
:10212000001F0000001F0001001E0000001E000034
:10213000001E0000001E00000039300000332500A2
:102140000087190000B00F0000DB080000BD04008C
:1021500000740200003F01000020436F756E742080
:10216000583A0023646566696E65204445464155CA
:102170004C545F0000626564004B6420004B692092
:10218000004B7020005049442074756E696E6720C2
:10219000646F6E6500504944204175746F74756EAC
:1021A000652066696E6973686564212050757420C6
:1021B000746865206C617374204B702C204B69200F
:1021C000616E64204B6420636F6E7374616E747310
:1021D0002066726F6D2062656C6F7720696E746F18
:1021E00020436F6E66696775726174696F6E2E68E1
:1021F0000A00504944204175746F74756E652066FD
:1022000061696C6564212074696D656F75740A007D
:102210004175746F74756E65206661696C656421C3
:102220002054696D656F75742E00504944204175C6
:10223000746F74756E65206661696C6564212054E5
:10224000656D706572617475726520746F6F20685A
:102250006967680A00504944204379636C657300DC
:1022600025532025692F256900204B643A20002042
:102270004B693A2000204B703A200020436C617378
:1022800073696320504944200A00204E6F206F7606
:10229000657273686F6F740A002054753A200020CD
:1022A0004B753A2000206D61783A2000206D696EF0
:1022B0003A200020643A200020626961733A2000CD
:1022C00048656174696E672E2E2E00504944204186
:1022D00075746F74756E652073746172740A004151
:1022E00075746F74756E65206661696C65642E2007
:1022F00054656D706572617475726520746F6F20BE
:10230000686967682E00504944204175746F747580
:102310006E65206661696C6564212054656D706529
:1023200072617475726520746F6F20686967680ADE
:1023300000426564004531004500626564002C2060
:1023400073797374656D2073746F70706564212088
:102350004865617465725F49443A2000486561745C
:10236000696E67204661696C6564004865617469DF
:102370006E67206661696C6564004D3131322053AF
:10238000687574646F776E001000C90210012C012B
:102390004001220170011801B0010E01F001040199
:1023A0005002FA00B002F0003003E600D003DC0077
:1023B0009004D2007005C800A006BE000008B4005A
:1023C000B009AA00D00BA000600E960060118C002E
:1023D0000015820020197800C01D6E00A022640044
:1023E000B0275A00902C500000314600E0343C00E9
:1023F00010383200903A2800603C1E00A03D1400C6
:10240000803E0A00203F00004572723A204D41583C
:1024100054454D50004D415854454D5020747269FB
:10242000676765726564004572723A204D494E5483
:10243000454D50004D494E54454D502074726967CA
:10244000676572656400544845524D414C205255B1
:102450004E4157415900546865726D616C20527548
:102460006E61776179000A0A0020205A5F4D494E5B
:102470003A002020595F4D494E3A002020585F4DC8
:10248000494E3A00202F002042403A0020403A00B6
:1024900020573A007C3C3E5E2B3D3F2F5B5D3B2C42
:1024A0002A225C0043616E6E6F74206F70656E202F
:1024B00073756264697220004D6564696120496EBC
:1024C0006974204661696C00534420636172642022
:1024D0006F6B0A006F70656E526F6F742066616972
:1024E0006C65640A00766F6C756D652E696E697433
:1024F000206661696C65640A004E6F205344206356
:102500006172640A000A4D3234004D323320257363
:10251000002E0A006F70656E206661696C65642C20
:102520002046696C653A200046696C652073656CCD
:1025300065637465640A002053697A653A20004631
:10254000696C65206F70656E65643A2000454E4485
:1025500020535542524F5554494E450A002220708F
:102560006F73002220706172656E743A22005355B9
:1025700042524F5554494E452043414C4C207461C2
:10258000726765743A220053756263616C6C204F08
:10259000766572666C6F770045786365656465641F
:1025A000206D617820535542524F5554494E452075
:1025B00064657074683A002E0A0044656C6574693D
:1025C0006F6E206661696C65642C2046696C653AA3
:1025D000200046696C652064656C657465643A002A
:1025E0005344207072696E74696E672062797465F5
:1025F00020004E6F74205344207072696E74696EAF
:10260000670A002F6175746F25632E670057726922
:1026100074696E6720746F2066696C653A20006685
:102620007265736800646F696E67002066696C6527
:102630003A20004E6F7720002020506C616E6E654E
:102640007242756666657242797465733A2000203D
:1026500046726565204D656D6F72793A20002043A2
:102660006F6D70696C65643A204D6179202031206E
:10267000323032320A00204C61737420557064612C
:102680007465643A20323032322D30342D303320AC
:102690007C20417574686F723A20426F6E64746575
:1026A0006368202F20496E73616E69747941757477
:1026B0006F6D6174696F6E0A004D61726C696E2096
:1026C0004457372E342E360A0020536F66747761D4
:1026D00072652052657365740A00205761746368DF
:1026E000646F672052657365740A002042726F77C9
:1026F0006E206F75742052657365740A00204578EA
:102700007465726E616C2052657365740A00506F57
:1027100077657255700A0073746172740A004739E4
:10272000310A47315A350A4739300A4D38340A4D93
:1027300031303453300A4D3134305330004D313064
:102740003031006572726F722077726974696E67DA
:1027500020746F2066696C650A00446F6E65207393
:102760006176696E672066696C652E0A004D3239A4
:1027700000456E6473746F707300255320256320C9
:10278000256320256320256300205A3A0020593A0A
:102790000020583A00656E6473746F707320686926
:1027A000743A200000002100240027002A002D0098
:1027B0003000330001010000040107010A0100009C
:1027C0002200250028002B002E00310034000201D9
:1027D0000000050108010B01000020002300260075
:1027E00029002C002F003200000100000301060127
:1027F0000901050505050705080808080202020287
:102800000A0A08080404040401010101010101018C
:102810000303030303030303040707070C0C0C0C57
:102820000C0C0C0C02020202060606060606060640
:102830000B0B0B0B0B0B0B0B0102102020080810CD
:102840002040102040800201020108040201010220
:1028500004081020408080402010080402018004F9
:102860000201804020100804020108040201010254
:10287000040810204080010204081020408000005D
:102880000A0B02090C0D0E080703040100000000EA
:102890000000000000000000000000000000000038
:1028A00000000000000000000000121110000000F5
:1028B0000000000000000000000000000000000018
:1028C00000000000FFFFFF50726F62696E672046D4
:1028D00061696C65640A0050726F62696E672046B8
:1028E00061696C656400205A3A200020593A200042
:1028F00042656420583A2000726573756D65640006
:102900004469736D69737300526573756D696E67A1
:102910000073686F7700627574746F6E006265672C
:10292000696E0044697361626C6552756E6F75748F
:102930000050757267654D6F726500506175736503
:102940006400436F6E74696E7565004C6F6164203E
:1029500046696C616D656E742054004C6F61642033
:1029600046696C616D656E7400496E7365727420A2
:1029700066696C616D656E7420616E642073656E4E
:1029800064204D3130380A0020204D323036205836
:1029900000486F6D65206F666673657400436170F3
:1029A0003A00434F4E4649475F4558504F525400F6
:1029B0004D4541545041434B00434F4F4C45525FAE
:1029C00054454D5045524154555245004348414DA0
:1029D0004245525F54454D50455241545552450071
:1029E000424142595354455050494E470041524389
:1029F00053004D4F54494F4E5F4D4F444553005483
:102A00004845524D414C5F50524F54454354494FF5
:102A10004E00455854454E4445445F4D32300043C6
:102A20005553544F4D5F4649524D574152455F559E
:102A3000504C4F4144004C464E5F5752495445005C
:102A40004C4F4E475F46494C454E414D4500415520
:102A5000544F5245504F52545F53445F5354415466
:102A600055530053445F5752495445005245504511
:102A70004154004D554C54495F564F4C554D4500FF
:102A80005344434152440050524F4D50545F5355AC
:102A900050504F525400484F53545F414354494F94
:102AA0004E5F434F4D4D414E445300454D455247B7
:102AB000454E43595F50415253455200434153459F
:102AC0005F4C494748545F4252494748544E45532A
:102AD0005300544F47474C455F4C494748545300B7
:102AE000534F4654574152455F504F57455200424D
:102AF00055494C445F50455243454E54004C455651
:102B0000454C494E475F44415441005A5F50524F33
:102B100042450052554E4F5554004155544F4C4577
:102B200056454C005052494E545F4A4F4200505255
:102B30004F4752455353004155544F5245504F5201
:102B4000545F54454D50004155544F5245504F52DB
:102B5000545F504F5300564F4C554D4554524943C6
:102B600000454550524F4D0042494E4152595F4633
:102B7000494C455F5452414E5346455200534552CD
:102B800049414C5F584F4E5F584F464600464952A8
:102B90004D574152455F4E414D453A4D61726C690A
:102BA0006E204457372E342E3620544D3344205354
:102BB000534D444E4220284D61792020312032303F
:102BC00032322031343A35393A30302920534F559A
:102BD0005243455F434F44455F55524C3A687474C5
:102BE00070733A2F2F6769746875622E636F6D2F4B
:102BF000496E73616E6974794175746F6D61746942
:102C00006F6E2F4D61726C696E2F747265652F4304
:102C10007265616C6974794477696E5F322E302019
:102C200050524F544F434F4C5F56455253494F4EAD
:102C30003A312E30204D414348494E455F5459505A
:102C4000453A544D3344203130532050726F204563
:102C5000585452554445525F434F554E543A3120D3
:102C6000555549443A63656465326132662D3431A5
:102C700061322D343734382D396231322D63353598
:102C80006336326633363766660A0050726F6265A5
:102C9000204F6666736574205A0050726F6265201B
:102CA0004F6666736574205A00290A0020746F20ED
:102CB000003F5A206F7574206F662072616E6765E1
:102CC000202800290A0020746F20003F59206F75CA
:102CD00074206F662072616E676520282D00290AB6
:102CE0000020746F20003F58206F7574206F66209D
:102CF00072616E676520282D00203B0020204D3832
:102D000035312058005A2D50726F6265204F66662B
:102D1000736574004D383400446F6E6520707269BD
:102D20006E74696E672066696C650A004D373700FE
:102D30004D33310043616E6E6F74206F70656E208D
:102D400073756264697220002569730025696D20BE
:102D5000256973002569682025696D202569730040
:102D6000256964202569682025696D20256973001F
:102D700025697920256964202569682025696D20E9
:102D800025697300436F6F6C696E672E2E2E0045A8
:102D9000312025530020573A0042656420436F6F6D
:102DA0006C696E672E2E2E00426564204865617442
:102DB000696E672E2E2E003D3D4477696E20496E68
:102DC000697420436F6D706C6574653D3D00202D06
:102DD000206434200064333A2000202D2064322007
:102DE0000064313A2000202D206C656E2000565082
:102DF0002072656365697665643A2000776169745D
:102E0000776179203D3D0020202A2A2A2A2A2A2A71
:102E10005254535F48616E646C65446174612A2A40
:102E20002A2A2A2A2A2A20002A2A2A4E6F7A7A6CEB
:102E30006554656D705374617475735B325D203DCC
:102E4000003D3D48656174696E6720446F6E652082
:102E50004368616E67652046696C616D656E743D9F
:102E60003D002020737461727470726F67726573B5
:102E70007320004D32320A4D3231003D3D77616999
:102E80007477617920353D3D003D3D776169747708
:102E9000617920343D3D003D3D776169747761790A
:102EA00020333D3D003D3D77616974776179203184
:102EB0003D3D00436F6E6669726D20436F6E7469AD
:102EC0006E75650050617573655374617475730038
:102ED000524553554D45204F5054494F4E533A009B
:102EE00048656174696E672E2E2E000000436C6980
:102EF000636B20746F206865617400000052657315
:102F0000756D696E672E2E2E000000507572676910
:102F10006E672E2E2E000000496E7365727420615C
:102F20006E6420436C69636B000000436C69636BE3
:102F300020746F20636F6E74696E756500000045C4
:102F40006A656374696E672E2E2E000000506C65F2
:102F500061736520776169742E2E2E000000506128
:102F6000726B696E672E2E2E0000002A2A2A496E87
:102F70006974696E672063617264206973204F4BC6
:102F80002A2A2A003D3D6F6E5072696E7454696D35
:102F9000657253746F707065643D3D003D3D6F6EAA
:102FA00055736572436F6E6669726D5265717569AE
:102FB0007265643D3D005061757365204D6F6465B9
:102FC00020537461747573004C6F6164696E672E71
:102FD0002E2E0000003D3D6F6E466163746F727966
:102FE00052657365743D3D00270A0A0000272027BB
:102FF000002027002D0063616E63656C00507269CC
:103000006E742041626F727465640055492041629C
:103010006F7274656400726573756D65004D32344E
:10302000002A2A2A43506C617920546F6E652A2A3F
:103030002A003D3D6F6E5072696E7454696D657201
:103040005061757365643D3D00486F6D696E672022
:103050004661696C65640050524553454E54004FBB
:103060005554006F70656E005452494747455245AC
:1030700044003A20004D4F54494F4E203A20004F13
:1030800046460A003A200066696C616D656E740000
:103090007A5F6D696E00795F6D696E00785F6D694A
:1030A0006E005265706F7274696E6720656E64732E
:1030B000746F70207374617475730A0020746F6F7D
:1030C000206C6F6E6720657874727573696F6E20FF
:1030D00070726576656E7465640A0020636F6C6457
:1030E00020657874727573696F6E2070726576658D
:1030F0006E7465640A00486F6D652025732573251D
:1031000073204669727374005761726E696E673A14
:1031100020486F6D696E672042756D702044697636
:1031200069736F72203C20310A0002020400000023
:1031300000000000000000000000809D4300009B94
:10314000430000C8430000004100000041000000AF
:1031500040000000010000000100008000555555AE
:10316000000000400033333300AAAA2A0049922409
:103170000000002000C7711C0099991900D1451763
:1031800000555515003BB1130024491200111111CF
:1031900000000010000F0F0F00E3380E0043790D00
:1031A00000CCCC0C00C3300C00E8A20B0064210B57
:1031B00000AAAA0A00703D0A009DD80900427B09B6
:1031C0000092240900DCD308008888080010420817
:1031D0000000000800F0C10700878707007550074E
:1031E00000711C07003EEB0600A1BC0600699006BA
:1031F0000066660600703E06006118060017F405BA
:103200000074D105005BB00500B290050062720544
:10321000005555050078390500B81E05000505055F
:10322000004EEC040087D40400A1BD040090A70464
:103230000049920400C17D0400EE690400C75604F1
:1032400000444404005C32040008210400411004DE
:1032500000000004003FF00300F8E0030026D20362
:1032600000C3C30300CCB503003AA803000A9B03C4
:1032700000388E0300C08103009F750300D06903EE
:1032800000505E03001D53030034480300913D03CA
:10329000003333030016290300381F03009715037A
:1032A00000300C0300030303000BFA020049F10293
:1032B00000BAE802005CE002002DD802002DD00226
:1032C0000059C80200B0C0020031B90200DAB102F0
:1032D00000AAAA0200A0A30200BC9C0200FA950268
:1032E000005C8F0200DF88020082820200457C02BF
:1032F000002776020027700200436A02007C640205
:1033000000D05E02003F590200C8530200FFFDFCDE
:10331000FAF8F6F4F2F0EEECEAE9E7E5E3E1E0DEF4
:10332000DCDAD9D7D5D4D2D0CFCDCBCAC8C7C5C3A4
:10333000C2C0BFBDBCBAB9B7B6B4B3B2B0AFADAC22
:10334000AAA9A8A6A5A4A2A1A09E9D9C9A99989777
:1033500095949392908F8E8D8B8A898887868483AB
:103360008281807F7E7D7B7A7978777675747372BF
:1033700071706F6E6D6C6B6A6968676665646362B5
:1033800061605F5E5D5C5B5A59585857565554539F
:10339000525150504F4E4D4C4B4A4A494847464671
:1033A000454443424241403F3E3E3D3C3B3B3A392F
:1033B000383837363535343332323130302F2E2EDF
:1033C0002D2C2B2B2A292928272726252524232382
:1033D00022212120201F1E1E1D1C1C1B1B1A191917
:1033E0001818171616151514131312121111100FA1
:1033F0000F0E0E0D0D0C0C0B0A0A09090808070721
:10340000060605050404030302020100003D3D6FAA
:103410006E5072696E7454696D6572537461727422
:1034200065643D3D0000809D4300009B430000C853
:10343000430000000000000000000000005361761F
:10344000696E67204457494E204C4344207365748D
:1034500074696E672066726F6D20454550524F4DFE
:103460000A003D3D6F6E53657474696E67735374E3
:103470006F7265643D3D0053657474696E677320B7
:1034800053746F72656400290A0020627974657351
:103490003B20637263200053657474696E67732008
:1034A00053746F7265642028006001F4017001EAB2
:1034B000019001E001B001D601D001CC010002C2AF
:1034C000013002B8016002AE019002A401D0029A5C
:1034D000012003900170038601C0037C0130047257
:1034E00001A004680120055E01B005540160064A90
:1034F0000120074001F0073601F0082C01100A22D4
:1035000001500B1801C00C0E01500E04013010FACE
:10351000002012F0005014E600C016DC007019D232
:1035200000501CC800501FBE007022B400B025AA75
:1035300000F028A000202C9600302F8C0010328242
:1035400000A0347800F0366E00E0386400803A5A0B
:1035500000403B5500E03B5000F03C4600C03D3C85
:1035600000603E3200E03E2800303F1E00503F1910
:1035700000703F1400A03F0A00C03F0000D03FF69B
:10358000FFE03FECFF220A00556E6B6E6F776E20F6
:10359000636F6D6D616E643A2022002042002050FE
:1035A000006F6B00204500205A0020590020204D5C
:1035B000393220580053746570732070657220751D
:1035C0006E69740020746F6F206C6F6E6720657871
:1035D00074727573696F6E2070726576656E74654E
:1035E000640A0020636F6C64206578747275736977
:1035F0006F6E2070726576656E7465640A004D3278
:103600003520500A4D323400526573756D65005592
:10361000492050617573650043616E6E6F7420655B
:103620006E746572207375626469723A20004E6F21
:10363000204D61746368203A00436F6E7374726149
:10364000696E206D65736856616C20006D657368E6
:1036500056616C200079506E74200078506E742092
:10366000006D657368506F696E74200044697370F3
:103670006C61794272696768746E65737320536513
:10368000743A2000446973706C61794272696768AA
:10369000746E657373204C43443A20004D32320AF5
:1036A0004D3231005265667265736800506755701F
:1036B000005067446F776E0049732046696C65203F
:1036C000004973204469722000476F557044697245
:1036D00000486173204D656469610046696C656EE0
:1036E000616D652053656C6563746564004D3130B0
:1036F000303043004D31303030002046696C616D10
:10370000656E7420526573706F6E7365204E6F0026
:10371000526573756D652059657320647572696EA5
:1037200067207072696E74000A204E6F2046696CC3
:10373000616D656E7400496E76616C6964204F70CE
:1037400074696F6E004D3530300053746F726520B0
:1037500053657474696E6773004D3939390A4D3297
:10376000383050305331363000424C546F756368F6
:10377000205265736574004D3530320A4D35303056
:1037800000496E697420454550524F4D004D35300B
:10379000300053746F72652053657474696E67737B
:1037A00000496E4C616E6743686F696365000A206B
:1037B0002A2A2A7265636461742E646174615B30C5
:1037C0005D203D004732380A4731204631303030E5
:1037D000205A313000556E737570706F7274656465
:1037E000204F7074696F6E2053656C6563746564F7
:1037F000004D32313153300A4739310A47315A309E
:103800002E3032350A4739300A4D323131533100CA
:103810004D32313153300A4739310A47315A2D3050
:103820002E3032350A4739300A4D323131533100AA
:10383000473239533200473239533100473236521A
:10384000323535004D3139305335350A4732380A73
:103850004732390A4D3430300A4D31303453323129
:10386000350A4732380A4D313039533231350A4D35
:1038700034323053310A47315831303059313030D9
:1038800046353030300A47315A300A4D3530300A2B
:103890004D37370A4D31313720536574205A204F48
:1038A0006666736574004731204631303030205AE7
:1038B000302E30004732380A473120463130303020
:1038C000205A302E30005A204F6666736574203AB5
:1038D000202573005A204F6666736574203A2025B0
:1038E00073004732385A0A473146313530305A3042
:1038F0002E30004732380A473146313530305A30A1
:103900002E3000426564204C6576656C204F7074E3
:10391000696F6E200052657475726E203A20004DFA
:10392000383400473146313030305A302E3000477D
:1039300032380A473146313030305A302E30004D5F
:10394000616E75616C53657454656D70005A204FDB
:103950006666736574203A20257300526F756E6435
:10396000696E6720746F207374657000526571759D
:103970006573746564204F666673657420005374C4
:103980006F70205472696767657265640053746F65
:1039900070204E6F0053746F705072696E740048DF
:1039A000616E646C6520446174612041646A757362
:1039B0007420322053657474696E67205363726596
:1039C000656E200048616E646C65204461746120FE
:1039D0005072696E7446696C652033205365747447
:1039E000696E672053637265656E200048616E647E
:1039F0006C652044617461205072696E7446696C14
:103A00006520322053657474696E67205363726554
:103A1000656E20004D38340048616E646C6520444A
:103A2000617461205072696E7446696C6520506FD4
:103A300073740048616E646C652044617461205049
:103A400072696E7446696C652050726500426567E4
:103A5000696E537769746368003D3D204368656310
:103A60006B6B65793D3D007265636461742E6164C2
:103A70006472203D3D007265636461742E646174FC
:103A8000615B305D203D3D0020453A00205A3A0000
:103A900020593A00583A006F6B0A00526573656E00
:103AA000643A20006E6F74696669636174696F6E51
:103AB0002000544D3344203130532050726F205237
:103AC000656164792E005072696E74696E672E2E7E
:103AD0002E005072696E74205061757365640052D7
:103AE0004553554D45204F5054494F4E533A004889
:103AF000656174696E672E2E2E000000436C696349
:103B00006B20746F206865617400000052657375E6
:103B10006D696E672E2E2E00000050757267696EFB
:103B2000672E2E2E0000004C6F6164696E672E2E8A
:103B30002E000000496E7365727420616E6420432C
:103B40006C69636B000000436C69636B20746F20C9
:103B5000636F6E74696E7565000000456A65637415
:103B6000696E672E2E2E000000506C656173652013
:103B7000776169742E2E2E0000005061726B696EA1
:103B8000672E2E2E00000050617573654D73673DE2
:103B90000000F600E40111241FBECFEFD1E2DEBF2A
:103BA000CDBF00E00CBF84B78093131914BE0FB6CD
:103BB000F894A895809160008861809360001092CD
:103BC00060000FBE16E0A0E0B2E0EEE6F0E702E033
:103BD0000BBF02C007900D92A832B107D9F729E1B7
:103BE000A8E2B6E001C01D92A331B207E1F71DE1E2
:103BF000CAECDDE100E006C021970109802FFE013B
:103C00000F946434C93CD10780E00807A9F70F94EA
:103C1000B5200D9425380C94000020912F07833097
:103C200021F425FD0CC024FD0CC030E0A90102C028
:103C3000559547958A95E2F7CA018170089581E00C
:103C4000089580E008958091E60984FD0BC080917D
:103C5000E80987FD07C09091E909937081E019F4A4
:103C600080E0089581E00895082E000C990BFC0176
:103C7000EE50F84DE491EE2391F0F0E0EE0FFF1FCF
:103C8000E852F84DA591B4912C91885C974DFC01B8
:103C90008491282381E090E021F480E0089580E081
:103CA00090E00895082E000C990BFC01EE50F84DA1
:103CB000E491F0E0EE0FFF1FEC55F84DA591B491A3
:103CC0002C91885C974DFC018491822391E009F44A
:103CD00090E0892F0895EDE9F7E09491981739F075
:103CE000319697E0E33BF907C1F780E0089581E062
:103CF0000895269A2E9A08950F931F93CF93DF93DA
:103D000000D01F92CDB7DEB79C0104E119E090E12D
:103D1000E0E4FFE0D80101900D929A95E1F7F901F6
:103D20002081318142815381F801608571858285CE
:103D300093850F946D34F80160877187828793872C
:103D400080E090E0A0EAB0E489839A83AB83BC83EF
:103D5000CE0101960E94B0B70F900F900F900F9078
:103D6000DF91CF911F910F910895CF93DF9300D0F2
:103D70001F92CDB7DEB780E090E0A0EAB0E489837F
:103D80009A83AB83BC8361E0CE0101960E941BB98C
:103D90000F900F900F900F90DF91CF910895BC017D
:103DA000990F880B990B0C945AEA80911F079091F8
:103DB0002007009731F04AE050E070E060E00D9499
:103DC000C02B60E070E0CB01089580911F079091B7
:103DD0002007009731F04AE050E070E060E00D9479
:103DE000922A60E070E0CB0108950E94E51E97FDE5
:103DF0000CC00E94E51E6F3F71058105910509F019
:103E000034F40E94E51E862F089580E008958FEF18
:103E1000089580911F0790912007892B41F00E94FF
:103E2000F51E91E0811101C090E0892F089591E085
:103E3000FCCFFC01659175918591949108958091D5
:103E40005F08882319F080E00E94F3BB80E00895AA
:103E50008F929F92AF92BF92CF92DF92EF92FF929A
:103E6000CF93DF93EC0180909C0A90909D0AA090E4
:103E70009E0AB0909F0A20E030E0A901C501B4017C
:103E80000F94A52D882309F454C0C880D980EA80F6
:103E9000FB80A7019601C501B4010F94A52D18164A
:103EA0000CF04CC02091940A3091950A4091960AEA
:103EB0005091970AC701B6010F94A52D882331F1BF
:103EC000C092940AD092950AE092960AF092970ACC
:103ED0002091980A3091990A40919A0A50919B0A30
:103EE000688179818A819B810F940B2E9B01AC01A3
:103EF00060E070E080E89FE30F946C34609302020E
:103F00007093030280930402909305026091020271
:103F1000709103028091040290910502DF91CF918C
:103F2000FF90EF90DF90CF90BF90AF909F908F90D9
:103F3000089560E070E080E89FE3F0CF60E070E01B
:103F4000CB01ECCF682F70E090E080E00C945AEA4F
:103F50000E94E51ECB0108950F931F93CF9380918C
:103F60001F07909120070097E9F0FC018F01C19194
:103F70002C2F2F7D81F0C53411F0C536B9F7F8012B
:103F8000108270E060E00F943429F801C083CF9173
:103F90001F910F91089570E060E0CF911F910F91F4
:103FA0000D94342960E070E0CB01F1CF2FEB280FA6
:103FB0002A3108F047C0E22FF0E08091E6099091A5
:103FC000E709A091E809B091E90904C0B695A79561
:103FD000979587952A95D2F780FD02C08170089544
:103FE000E853F64FE081EE2341F180918E0A9091E3
:103FF0008F0AE80FF92FF11D808190ED980F9A300C
:1040000030F08E3251F4818180538A3098F4F093ED
:104010002007E0931F0781E008958D3211F08B3265
:1040200049F4818190ED980F9A3088F38E3211F423
:104030008281EACFF0E0E0E0EACF10922007109210
:104040001F07E9CF80E008950E94D61F882341F022
:1040500081E020911F0730912007232B09F480E095
:104060000895CF92DF92EF92FF926A017B010E9446
:104070002420882331F0FF90EF90DF90CF900C94B4
:10408000AC1FC701B601FF90EF90DF90CF9008956D
:10409000CF93DF93EB010E942420882321F0DF914E
:1040A000CF910C94A81FCE01DF91CF910895CF93AB
:1040B000DF93EB010E942420882319F00E94E51E63
:1040C000EB01CE01DF91CF910895CF93C62F0E94CF
:1040D0002420882319F0CF910C94F51E8C2FCF91BA
:1040E0000895CF93DF93C82FD62F0E9424208823D2
:1040F00021F0DF91CF910C94091F8C2F0E94D61FC5
:10410000811101C08D2FDF91CF910895CF92DF9261
:10411000EF92FF92CF936B017C01C42F80916008D6
:104120008F5F09F4B5C08093600880916008809328
:104130000F0920E030E040E752E460912F027091D7
:10414000300280913102909132020F940B2E0F9425
:10415000E0357093720860937108C0927308D09232
:104160007408E0927508F092760880910E09C0FB01
:1041700080F980930E098CE0E1E1F8E0A7E7B8E070
:1041800001900D928A95E1F78CE0E4E3FAE0A3E870
:10419000B8E001900D928A95E1F780913E079091E9
:1041A0000E0980FB94F990930E09882381F0809189
:1041B0003A0790913B07A0913C07B0913D0780934F
:1041C0008F0890939008A0939108B09392088091E3
:1041D0003D1490913E14909394088093930880919D
:1041E00026149091271490939608809395088091B7
:1041F000B50A8093970880910E0990916F0E90FBFD
:1042000083F980930E0980919C0A90919D0AA09158
:104210009E0AB0919F0A8093980890939908A09362
:104220009A08B0939B080E940ABE60930909709394
:104230000A0980930B0990930C0980912F078093B2
:104240000D099091100E80910E0993FB81F99091C8
:10425000410A90FB82F980930E0980E00E94ACA293
:1042600040E050E0BA018AE197E10E947B7A40EB9E
:1042700050E060E678E08AE197E10E940F7B8AE1F6
:1042800097E1CF91FF90EF90DF90CF900C943C7E20
:1042900081E049CF4F925F926F927F928F929F926F
:1042A000AF92BF92CF92DF92EF92FF921F93CF9384
:1042B000DF9300D01F92CDB7DEB719821A821B821E
:1042C0001C82CE0101964C0184E1C82E89E0D82ED3
:1042D00090E4E92E9FE0F92E20E5A22E2FE0B22EE9
:1042E00010E088E5810F0E942420F40181934F01A2
:1042F000882309F4E7C00E94AC1F2B013C01812FE9
:104300000E940D1E882309F4D3C0F701208131815A
:1043100042815381C301B2010F946D34F601608371
:104320007183828393831F5FF4E0CF0ED11C84E0FE
:10433000E80EF11C94E0A90EB11C133091F685E44F
:104340000E9424208C83882309F4C7C00E94AC1FDC
:104350006B017C0183E00E940D1E882371F0209187
:104360004C0F30914D0F40914E0F50914F0FC701A0
:10437000B6010F946D346B017C01C0922009D0927C
:104380002109E0922209F09223098091250E8823C9
:1043900091F18091151782FF2EC087FD2CC08C8172
:1043A000882349F18981811103C08A81882319F109
:1043B0002DEC3CEC4CE45DE36091690870916A0877
:1043C00080916B0890916C080F946D349B01AC0147
:1043D0006091480F7091490F80914A0F90914B0F57
:1043E0000F94CD3618163CF440E060E070E080E0B9
:1043F00090E40E94862040E050E0BA0186E40E94EA
:10440000312020E030E0A9010F94CD36181684F455
:104410000E94AC1F20E030E040E752E40F94673583
:1044200060932F0270933002809331029093320296
:104430008091100E83FD28C08091FD07882321F113
:1044400020914C0F30914D0F40914E0F50914F0FD6
:10445000609120097091210980912209909123098E
:104460000F946C3420910A0830910B0840910C088D
:1044700050910D080F946D3460930A0870930B08E7
:1044800080930C0890930D080F900F900F900F9051
:10449000DF91CF911F91FF90EF90DF90CF90BF9071
:1044A000AF909F908F907F906F905F904F90089506
:1044B000F5012081318142815381C301B2010F9402
:1044C0006C342CCFF70180819181A281B381F601F8
:1044D00080839183A283B38326CF80914C0F9091E8
:1044E0004D0FA0914E0FB0914F0F809320099093E4
:1044F0002109A0932209B093230947CFE0E6F8E011
:1045000080EBDF011D928A95E9F708958091250ED1
:10451000811104C00E947E220C9438A3809115174B
:1045200082FF09C087FD07C040E060E070E080E0E6
:1045300090E40C948620089580916008882361F0AF
:1045400090910F09891308C08091151784FF04C04A
:104550008CE998E00C94EC8180E00895FC012381C3
:1045600021110C943C7E0895CF93DF93C0913D14AC
:10457000D0913E14209729F16091391470913A142A
:1045800080913B1490913C140F94D9356E5F7F4F0E
:1045900024976C177D07ACF47093800760937F07B6
:1045A0000E949B72605A75418F4F9F4F60938107A5
:1045B000709382078093830790938407DF91CF9154
:1045C000089510928107109282071092830710922B
:1045D0008407F4CFCF92DF92EF92FF921F93CF9395
:1045E000DF93182F662351F010921D0710921907C0
:1045F00010921A0710921B0710921C070E949B72C0
:104600006B017C018091190790911A07A0911B07FB
:10461000B0911C07A7019601281B390B4A0B5B0BB5
:10462000DA01C901B7FD3DC020911D0717FD13C078
:10463000412F012E000C550B4C5F5F4F822F022E35
:10464000000C990B4817590764F184EF91E0A0E042
:10465000B0E0211724F488EE93E0A0E0B0E08C0DE8
:104660009D1DAE1DBF1D8093190790931A07A0933F
:104670001B07B0931C072170C22F30E0D32F84E2B8
:104680008C9FB0018D9F700D7C1B112460597C4F55
:1046900082E390E00E942DC280911D078F5F80937E
:1046A0001D07DF91CF911F91FF90EF90DF90CF908A
:1046B0000895CF93DF93C0912614D09127142097AB
:1046C00029F1609122147091231480912414909107
:1046D00025140F94D9356E5F7F4F24976C177D0793
:1046E000ACF470937807609377070E949B72605ECA
:1046F00070448D4F9F4F6093790770937A07809332
:104700007B0790937C07DF91CF91089510927907F2
:1047100010927A0710927B0710927C07F4CFCF9308
:10472000C1E020E030E0A9016091520A7091530A83
:104730008091540A9091550A0F94A52D811101C0C2
:10474000C0E08C2FCF910895CF93C82F882321F0FC
:104750000E948F238823D9F080916F0E8C17B9F0B7
:104760000E94F3AE80916F0E882349F080E49FE0B1
:104770000E9416AF10926F0ECF910C9427BA81E071
:1047800080936F0E80E49FE00E941FAEF5CFCF9123
:1047900008954F925F926F927F928F929F92AF9205
:1047A000BF92CF92DF92EF92FF920F931F93CF931E
:1047B000DF93EC0120914A0A30914B0A40914C0A58
:1047C00050914D0A688179818A819B810F946C3464
:1047D0006B017C0120914E0A30914F0A4091500AA2
:1047E0005091510A6C817D818E819F810F946C3430
:1047F0004B015C01A70196016091110770911207AE
:1048000080911307909114070F94A52D882309F424
:1048100050C0C0921107D0921207E0921307F09295
:1048200014072091090730910A0740910B07509116
:104830000C07C701B6010F940B2E2B013C010F94FE
:104840000F366B017C0120E030E0A9010F94A52D0B
:1048500087FD70C020E030E040E450E4C701B601BD
:104860000F94CD3618162CF4C12CD12CC0E4EC2EAC
:10487000FE2CA7019601C301B2010F946C34609322
:104880000107709302078093030790930407C70101
:10489000B6010F94D9356093FF06062E000C770BF6
:1048A0006F5F7F4F6430710514F064E070E06093D7
:1048B000FD06D091FB061091FF06A50194016091C1
:1048C00015077091160780911707909118070F949C
:1048D000A52D811133C0D11381C02091E306309101
:1048E000E4064091E5065091E6066091010770915B
:1048F000020780910307909104070F940B2E2091DB
:10490000E7063091E8064091E9065091EA060F94D7
:104910006D34DF91CF911F910F91FF90EF90DF9059
:10492000CF90BF90AF909F908F907F906F905F904F
:104930004F900895C12CD12C76019BCF8092150702
:1049400090921607A0921707B092180720910D07B2
:1049500030910E0740910F0750911007C501B40127
:104960000F940B2E4B015C010F940F366B017C01F1
:1049700020E030E0A9010F94A52D87FDF3C020E0D1
:1049800030E040E450E4C701B6010F94CD3618166C
:104990002CF4C12CD12CB0E4EB2EFE2CA7019601F7
:1049A000C501B4010F946C3460930507709306073A
:1049B0008093070790930807C701B6010F94D93574
:1049C00060930007062E000C770B6F5F7F4F6430FB
:1049D000710514F064E070E06093FE06C09100077A
:1049E000D11305C08091FC068C1709F470C080912A
:1049F000FF06909100079093FC068093FB060C2E17
:104A0000000CDD0B25E01203C0011124FC01EC0FAA
:104A1000FD1FEE0FFF1FEE0FFF1FEA54F14F208125
:104A20003181428153812093F7063093F8064093F9
:104A3000F9065093FA060091FE06002E000C110BA9
:104A4000FC01E00FF11FEE0FFF1FEE0FFF1FEA54F6
:104A5000F14F60817181828193810F946C346093F6
:104A6000F3067093F4068093F5069093F606209172
:104A7000FD0635E02303F0011124CE0FDF1FCC0F1C
:104A8000DD1FCC0FDD1FCA54D14F288139814A81E7
:104A90005B812093EF063093F0064093F10650932C
:104AA000F206E00FF11FEE0FFF1FEE0FFF1FEA549B
:104AB000F14F60817181828193810F946C34609396
:104AC000EB067093EC068093ED069093EE068090D3
:104AD000050790900607A0900707B090080720915F
:104AE000F3063091F4064091F5065091F606C501A3
:104AF000B4010F940B2E2091F7063091F8064091E7
:104B0000F9065091FA060F946D346B017C01C09246
:104B1000E706D092E806E092E906F092EA062091D4
:104B2000EB063091EC064091ED065091EE06C50182
:104B3000B4010F940B2E2091EF063091F0064091B6
:104B4000F1065091F2060F946D34A70196010F946F
:104B50006C346093E3067093E4068093E5069093CB
:104B6000E606BBCEC12CD12C760118CFE1E1F7E0EF
:104B700080EF9FEFA9E7B4EC84839583A683B78386
:104B800080839183A283B383EBEFF6E08DE9818389
:104B9000808308958F929F92AF92BF92CF92DF92BF
:104BA000EF92FF92FC0198E0A2E5BAE001900D922D
:104BB0009A95E1F788E0FB01AAE4BAE001900D9232
:104BC0008A95E1F7C090520AD090530AE090540AB7
:104BD000F090550A20E030E0A901C701B6010F941A
:104BE000A52D8823E1F1A701960160E070E080E83F
:104BF0009FE30F9467356B017C018090560A90907B
:104C0000570AA090580AB090590A20E030E0A90154
:104C1000C501B4010F94A52D882329F1A5019401A4
:104C200060E070E080E89FE30F946735C092090769
:104C3000D0920A07E0920B07F0920C0760930D07E1
:104C400070930E0780930F0790931007FF90EF90DB
:104C5000DF90CF90BF90AF909F908F900895C12C20
:104C6000D12C7601CACF60E070E0CB01DFCF8F920C
:104C70009F92AF92BF92EF92FF920F931F93CF93A9
:104C8000DF9310924E0A10924F0A1092500A10921F
:104C9000510A10924A0A10924B0A10924C0A109232
:104CA0004D0A1092560A1092570A1092580A109202
:104CB000590A1092520A1092530A1092540A1092F2
:104CC000550A06EB1EE0C0E0812C912C80ECA82E4A
:104CD0008FE7B82E7801D0E0F70181929192A192EE
:104CE000B1927F016D2F8C2F0F94DB02DF5FD530E7
:104CF00099F7CF5F0C5E1F4FC53061F7DF91CF9101
:104D00001F910F91FF90EF90BF90AF909F908F9069
:104D10000895EFE6F0E080818260808308958091BD
:104D2000601490916114892B79F4809160149091B2
:104D30006114892B49F4209160143091611481E051
:104D4000232B19F480E0089581E00895CF92DF923B
:104D5000EF92FF926B017C0183E3C816D104E1045A
:104D6000F10470F082E3C81AD108E108F10862E3A7
:104D700070E080E090E00E9468720E945489ECCF5D
:104D8000C701B6010E946872FF90EF90DF90CF904C
:104D90000C9454891092700E80914F079091500797
:104DA000A0915107B091520780934B0790934C0705
:104DB000A0934D07B0934E070895909163141092FD
:104DC00063149230B9F09430C1F09130E1F488234B
:104DD00019F0813021F008959093720E089582E0C9
:104DE0008093720E8091700E882369F01092710E7C
:104DF0000C94CA261092730E08958DE190E390935F
:104E0000B50E8093B40E08956C98749A0C94CA26CB
:104E10009091151794FB882780F994FF06C081E0D4
:104E200090917C18911101C080E008950E9408279C
:104E3000882339F08091151782FB882780F991E04B
:104E40008927089580911309811106C08091621409
:104E5000823011F00C94162781E008950C9404C15F
:104E600081E00895CF93DF93EC01E62F660FFF0BEF
:104E7000E258F74DE491E250E13108F0B0C0F0E0C3
:104E80008827EA5BF84D8F4F0D9464345727EF273E
:104E9000EF27EF27EF2781276327A527A32783275E
:104EA000C927C727A727EF27ED27EB27CB2782E1C5
:104EB000E1E6F2E0DE0101900D928A95E1F7CE0184
:104EC000DF91CF91089581E020EB30E03983288392
:104ED00021EB30E03B832A831D821C8223EB30E0F0
:104EE0003F832E8324EB30E0398728871B861A8680
:104EF0001D861C8692E09E878F8781E0888B198AA9
:104F0000DECF80E0E1CF81E08F5F20E930E03983C0
:104F1000288321E930E03B832A8322E930E03D8386
:104F20002C8328E930E03F832E832AE930E039875B
:104F300028872CE930E03B872A8726E930E03D8747
:104F40002C8793E0D8CF80E0DFCF80E0DECF81E018
:104F50008F5F20EA30E03983288321EA30E03B8309
:104F60002A8322EA30E03D832C8328EA30E03F8325
:104F70002E832AEA30E0398728872CEA30E03B8705
:104F80002A8726EA30E03D872C8794E0B4CF80E082
:104F9000DFCF80E0DECF81E08F5F20E231E0398338
:104FA000288321E231E03B832A8322E231E03D8302
:104FB0002C8328E231E03F832E832AE231E03987D7
:104FC00028872CE231E03B872A8726E231E03D87C3
:104FD0002C8795E090CF80E0DFCF80E0DECF82E1CC
:104FE000FE0111928A95E9F76ACF8F929F92AF9254
:104FF000BF92CF92DF92EF92FF920F93CF93DF9306
:105000001F92CDB7DEB75C017B0149016B01C40E75
:10501000D51EF501808191810F94C33389830023CC
:1050200011F0F7018083BE016F5F7F4FC4010E94C2
:105030007CE9F50180819181019691838083FFEF66
:10504000EF1AFF0AEC14FD0421F780E00F90DF91C6
:10505000CF910F91FF90EF90DF90CF90BF90AF90E6
:105060009F908F9008959091D10095FD0CC09091E4
:10507000D00095FF08C08093D6008091D000806456
:105080008093D000089520913E062F5F2F770FB6B2
:1050900007FC27C090913F06921328C09091D00042
:1050A00095FF1EC090913F0640913E06941306C0A6
:1050B0009091D1009F7D9093D10012C0E92FF0E034
:1050C000E25CF94F32819F5F9F773093D6009093D7
:1050D0003F063091D00030643093D000491741F33F
:1050E000D9CF90913F06921301C0FBCFE0913E06CD
:1050F000F0E0E25CF94F828320933E068091D1007C
:1051000080628093D10008958091ED099091EE091D
:105110002FEF3FEF981751F0E92FF0E0E351F64FF2
:10512000228130E09F5F9F739093EE09C90108953B
:105130001F920F920FB60F9211240BB60F922F935E
:105140008F939F93EF93FF9380913F0620913E06AC
:10515000821306C08091D1008F7D8093D10012C050
:10516000E82FF0E0E25CF94F92818F5F8F779093A8
:10517000D60080933F069091D00090649093D00029
:10518000281741F3FF91EF919F918F912F910F90ED
:105190000BBE0F900FBE0F901F9018951F920F928D
:1051A0000FB60F9211240BB60F920F931F932F93EC
:1051B0003F934F935F936F937F938F939F93AF939F
:1051C000BF93CF93DF93EF93FF93C091D6000091ED
:1051D000EE09D091ED0911E01D0F1F7390913D066E
:1051E000913108F09FC0E92FF0E08827E550F74D96
:1051F0008F4F0D9464340C293B294A295929602981
:1052000092296429922968296C2992297029742984
:1052100078297F2992298A29C03229F028F5CA30B5
:1052200011F0CD3031F5011731F0ED2FF0E0E35101
:10523000F64FC283D12FD093ED09FF91EF91DF910B
:10524000CF91BF91AF919F918F917F916F915F911E
:105250004F913F912F911F910F910F900BBE0F9087
:105260000FBE0F901F901895CD3481F081E0CE34A1
:1052700071F080E10CC0CA3338F4C033A0F6C032FC
:1052800091F2CD32B1F7CFCFCD3499F782E0809350
:105290003D06C9CFC13359F018F4C03221F2E9CF2D
:1052A00088E0C433A1F38BE0C83389F3E2CF83E015
:1052B000EECF84E0C03359F386E0C13341F3D9CF58
:1052C00085E0C833B1F6E3CF87E0C23391F6DFCF94
:1052D00089E0C13371F6DBCF8AE0C03351F6D7CF16
:1052E0008CE0C73331F6D3CF8DE0C63311F6CFCF84
:1052F000C03209F498CF8EE0C33549F2BACF80EDC1
:105300008C0F8A3008F08FCF9FE090933D068093FA
:105310003C0689CFCA3019F0CD3009F084CF109205
:105320003D0681CFCA3019F0CD3009F07CCF809195
:1053300009178823A1F3973089F038F4953079F76D
:10534000109222021092730EEACF9A3059F09F30D9
:1053500031F780913C060E94DD26E1CF81E0809309
:105360007E07DDCF81E080937D07D9CF9091C0008B
:1053700095FFFCCF8093C6000895CF93C82FC150EE
:1053800020F080E20E94B629FACFCF910895CF9302
:10539000DF93EC01FE0184912196882319F00E948D
:1053A000B629F8CFDF91CF910895CF93DF93C82F1F
:1053B0008EEB9FE00E94C7290C2E000CDD0BFE0136
:1053C000EE50F84D8491805C0E94B629FE01E85CA5
:1053D000F74DE49180E3E13021F0E6958F5F89336A
:1053E000D1F7DF91CF910C94B629CF92DF92EF9253
:1053F000FF926A017B010E94C72942E0C701B60102
:10540000FF90EF90DF90CF900C9496820E94F52948
:105410008AE00C94B629CF93DF936EEE7DE00F9473
:10542000A503CEE1D4E14B855C856D857E8585EE57
:105430009DE00E94F5292CEA35EC47E25EE36F859A
:10544000788989899A890F946735AB01BC0182EE0E
:105450009DE00E94F5292CEA35EC47E25EE36B897A
:105460007C898D899E890F940B2EAB01BC018FED39
:105470009DE0DF91CF910C94062ACF93DF936CE4EB
:105480007DE00F94A5036091370E7091380E8091E6
:10549000390E90913A0E0F94AA2DAB01BC0183E412
:1054A0009DE00E94F5294091670E5091680E609131
:1054B000690E70916A0E80E49DE00E94F52940918A
:1054C0006B0E50916C0E60916D0E70916E0E8DE3AF
:1054D0009DE00E94F529C5E1DEE0488159816A819D
:1054E0007B8184E991E10E94F5294C815D816E8187
:1054F0007F818AEA95E30E94F529488559856A8566
:105500007B8587EA95E30E94F5294C855D856E854C
:105510007F8584EA95E3DF91CF910C94062ACF939F
:10552000DF9361EC7CE00F94A503C7E2DEE04CA9B9
:105530005DA96EA97FA988EB9CE00E94F52948AD82
:1055400059AD6AAD7BAD85EB9CE00E94F5294CAD71
:105550005DAD6EAD7FAD8DE39DE0DF91CF910C949D
:10556000062ACF93DF936DE97CE00F94A503C7E291
:10557000DEE04CA15DA16EA17FA184E99CE00E94C8
:10558000F52948A559A56AA57BA58AEA95E30E9455
:10559000F5294CA55DA56EA57FA587EA95E30E9438
:1055A000F52948A959A96AA97BA984EA95E3DF915D
:1055B000CF910C94062ACF93DF9368E77CE00F9499
:1055C000A503C7E2DEE0688179818A819B810F941F
:1055D000AA2DAB01BC018FE69CE00E94F5296C81ED
:1055E0007D818E819F810F94AA2DAB01BC018AEA37
:1055F00095E30E94F529688579858A859B850F94B6
:10560000AA2DAB01BC0187EA95E30E94F5296C85C0
:105610007D858E859F850F94AA2DAB01BC0184EA00
:1056200095E3DF91CF910C94062ACF938091E60900
:10563000827161F48091E8098C7841F48091E909E4
:10564000837021F481E0CF910C943D2A82E40E9482
:105650002420882351F00E94D51E6093370E70934A
:10566000380E8093390E90933A0E83E50E942420E1
:10567000882351F00E94AC1F6093670E7093680EF0
:105680008093690E90936A0E84E50E9424208823FB
:1056900051F00E94AC1F60936B0E70936C0E809360
:1056A0006D0E90936E0E88E50E942420882351F0A1
:1056B0000E94AC1F6093150E7093160E8093170E08
:1056C0009093180E89E50E942420882351F00E94AF
:1056D000AC1F6093190E70931A0E80931B0E90935B
:1056E0001C0E8AE50E942420C82F882351F00E94B6
:1056F000AC1F60931D0E70931E0E80931F0E90932F
:10570000200E85E40E942420882351F00E94AC1FC3
:105710006093210E7093220E8093230E9093240E9B
:10572000CC23A9F02DEC3CEC4CEC5DE360911D0E1C
:1057300070911E0E80911F0E9091200E0F94A52D3A
:1057400018162CF08BE09DE0CF910C94C729CF91D7
:105750000895CF93C62F0E94C7298C2FCF910C9408
:1057600090820F931F93CF938C01C62F89E79AE005
:105770000E94C729C8010E94C729CC2331F08AE0C2
:10578000CF911F910F910C94B629CF911F910F913A
:1057900008950F931F93CF938C01C62F60E081E98A
:1057A0009AE00E94B12BC8010E94C729CC2331F096
:1057B0008AE0CF911F910F910C94B629CF911F9140
:1057C0000F91089561E089E99AE00C94C92BEF925A
:1057D000FF920F931F93CF937C018B01C42F60E046
:1057E00081E99AE00E94B12BC7010E94C72980E29B
:1057F0000E94B629C8010E94C729CC2319F08C2F1A
:105800000E94B6298AE0CF911F910F91FF90EF90EF
:105810000C94B629DF92EF92FF920F931F93CF93D0
:10582000DF93D82E7B018A01E9010E94E22BD092FE
:10583000631440E0B7018DE199E20E94E72B011566
:10584000110531F040E0B80186E199E20E94E72BB2
:10585000209731F040E0BE0186E199E20E94E72BFB
:1058600061E081E199E2DF91CF911F910F91FF906B
:10587000EF90DF900C94C92BAF92BF92CF92DF9242
:10588000EF92FF920F931F93CF93DF93EC0180E68B
:105890009AE00E94C729209711F4C6EBDEE010E0E1
:1058A00086E00E94BD29812F0E9490821F5F1530E3
:1058B000B9F78AE00E94B62910E080E20E94B6297A
:1058C000812F0E9490825E0105E080E20E94B6294D
:1058D000F501C080D180E280F380A7019601C70165
:1058E000B6010F945F37882361F180E20E94B629E8
:1058F0008DE30E94B6298DE30E94B6298DE30E94B4
:10590000B6298DE30E94B6298DE30E94B629015085
:10591000F4E1AF0EB11C0111D8CF8AE00E94B62984
:105920001F5F2496153049F68AE0DF91CF911F91D1
:105930000F91FF90EF90DF90CF90BF90AF900C94BD
:10594000B62920E030E0A901C701B6010F94CD3699
:1059500087FD03C08BE20E94B62943E0C701B60170
:105960000E949682D4CF811107C08BED92E10E94F4
:10597000C7298AE00C94B6298FED92E1F8CFCF9336
:1059800067EC72E10F94A503C091250EC05D8EEB0C
:1059900092E10E94C7298C2F0E94B6298AEB92E1DE
:1059A0000E94C7298091250ECF910C94B32C4F9261
:1059B0005F926F927F928F929F92AF92BF92CF929F
:1059C000DF92EF92FF92CF93DF93CDB7DEB72C97A4
:1059D0000FB6F894DEBF0FBECDBF83E50E94D61F81
:1059E0008823C9F00E94091F809335022C960FB6B8
:1059F000F894DEBF0FBECDBFDF91CF91FF90EF9047
:105A0000DF90CF90BF90AF909F908F907F906F90DE
:105A10005F904F90089580913502805D89838DEA73
:105A200091E10E94C72989810E94B62989EA91E102
:105A30000E94C729809135020E94B32C4090500FDC
:105A40005090510F6090520F7090530F2091370279
:105A5000309138024091390250913A02C301B201AB
:105A60000F946D3469837A838B839C838090540F69
:105A70009090550FA090560FB090570F20913B0279
:105A800030913C0240913D0250913E02C501B4016B
:105A90000F946D346D837E838F839887C090580FE9
:105AA000D090590FE0905A0FF0905B0F20913F0279
:105AB000309140024091410250914202C701B6012B
:105AC0000F946D3469877A878B879C872091430276
:105AD000309144024091450250914602C301B20107
:105AE0000F946D342B013C01209147023091480204
:105AF0004091490250914A02C501B4010F946D349E
:105B00004B015C0120914B0230914C0240914D02BF
:105B100050914E02C701B6010F946D346B017C01A8
:105B200081EA91E10E94C72949815A816B817C8178
:105B300084E991E10E94F5294D815E816F8178852C
:105B40008AEA95E30E94F52949855A856B857C850B
:105B500087EA95E30E94F5298FE991E10E94C72920
:105B600087E991E10E94C729B301A20184E991E18B
:105B70000E94F529B501A4018AEA95E30E94F5295E
:105B8000B701A60187EA95E30E94F5298AE02C96E1
:105B90000FB6F894DEBF0FBECDBFDF91CF91FF905F
:105BA000EF90DF90CF90BF90AF909F908F907F90BD
:105BB0006F905F904F900C94B62989E59AE00C9411
:105BC000C729FF920F931F93CF93DF936DE070E08F
:105BD00080E50E944820EC0197FD3EC0F82E60E071
:105BE00089E40E947120811110C08C2F0E946B1ECD
:105BF000882359F00E94DD2D85ED94E1DF91CF914E
:105C00001F910F91FF900C94C72984E50E942420D6
:105C1000082F8823A1F00E94F51E813059F028F04A
:105C2000823001F18EEC91E1E9CF60E08C2F0E948F
:105C30000F7205C061E08C2F0E940F7200E083E5B7
:105C40000E942420882341F00E94F51E182F89E02D
:105C5000F8120AC01093B50ADF91CF911F910F91EE
:105C6000FF90089562E0E2CF86EB91E10111C6CF8B
:105C700061E08C2F0E940F72612F8C2F0E949E7109
:105C8000612F70E08C2FDF91CF911F910F91FF90CA
:105C90000C9430F183E59AE00C94C729CF9384E506
:105CA0000E942420C0E0882309F10E94F51EC82F1D
:105CB0001816E4F40E944A2E8DE40E94B6296091E1
:105CC000E3097091E40990E080E00E94F0E981E24C
:105CD00093E10E94C7296C2FCC0F770B880B990B8F
:105CE0000E945AEA8AE00E94B629CFEF8C2FCF910A
:105CF00008950F931F93CF93811116C0C42F8B016A
:105D00000E944A2E8EE193E10E94C729C8010E9499
:105D1000C729CC2349F08AE30E94B6298AE0CF91B3
:105D20001F910F910C94B629CF911F910F91089557
:105D3000CF92DF92EF92FF92CF938091E60988781D
:105D400009F04DC08091E70987FD49C08091E809BD
:105D5000867009F044C00E944A2E8DE093E10E94B3
:105D6000C7298091710E811134C08BED92E10E94A0
:105D7000C72940914F07509150076091510770918A
:105D8000520780E093E10E94F5298DEF92E10E9495
:105D9000C729F090540784EF92E10E94C7296F2D24
:105DA00070E090E080E00E945AEA82EE92E10E9468
:105DB000C72980911E0781110FC08BED92E10E94CF
:105DC000C7298AE0CF91FF90EF90DF90CF900C949D
:105DD000B6298FED92E1CBCF8FED92E1F0CF88E441
:105DE0000E94D61F882321F00E94091F80931E075E
:105DF000C090E609D090E709E090E809F090E90941
:105E000081E1F694E794D794C7948A95D1F781E01D
:105E1000C822DD24EE24FF2483E50E94D61FC82F6C
:105E2000CD28CE28CF2811F4882341F00E94CA261D
:105E3000CC2321F00E94091F8093710E84E40E94FC
:105E4000D61F882311F10E94AC1F60934F077093F7
:105E50005007809351079093520780E50E94D61F08
:105E60008823C9F00E94A81F9C01332723303105E5
:105E70001CF02730310579F480935407CF91FF90BF
:105E8000EF90DF90CF900C9404278CE40E94D61FF3
:105E90008111D9CFE2CFCF91FF90EF90DF90CF90DB
:105EA0000895CF93C82F41E064ED7DE00E94792EE4
:105EB000C11102C00E944A2E4091401450914114D9
:105EC00060914214709143148BEC9DE00E94F5297F
:105ED0002CEA35EC47E25EE360914414709145147E
:105EE00080914614909147140F946735AB01BC0123
:105EF00088EC9DE00E94F5292CEA35EC47E25EE350
:105F0000609148147091491480914A1490914B14F7
:105F10000F940B2EAB01BC0185EC9DE00E94F5298E
:105F20008AE0CF910C94B629CF93811112C040E042
:105F30006DE57CE00E94792E80913E07811104C0BE
:105F400080E59CE00E94C7298AE00E94B6290E9451
:105F50004A2EC0913E0787E49CE00E94C7298C2FFF
:105F60000E94A21F40913A0750913B0760913C0765
:105F700070913D0784E49CE0CF910C94062A2F9207
:105F80003F924F925F926F927F928F929F92AF92C9
:105F9000BF92CF92DF92EF92FF920F931F93CF9316
:105FA000DF93CDB7DEB76D970FB6F894DEBF0FBEA7
:105FB000CDBF83E50E94D61F182F30906F0E882327
:105FC00019F00E94091F382E8091400F9091410FC7
:105FD000A091420FB091430F8A8F9B8FAC8FBD8FE2
:105FE0008091440F9091450FA091460FB091470FBB
:105FF0008E8B9F8BA88FB98F8091480F9091490FFE
:10600000A0914A0FB0914B0F8A8B9B8BAC8BBD8BB1
:10601000112329F0311003C080E00E94A423809155
:10602000E6099091E709A091E809B091E90925E115
:10603000B695A795979587952A95D1F74C015D015F
:10604000E1E08E229924AA24BB240E948F23882376
:1060500009F4C5C083E40E94D61F882309F4A0C0B8
:106060000E94AC1F2B013C0186EB9EE09F838E8338
:1060700099878887B5E0BD8300E0212CE8ECEE87A6
:10608000F2ECFF871A861B8628EC2C8782E48D872A
:10609000A885B985B98BA88B15E0E889F989C190E5
:1060A000D190E190F190F98BE88B2A853B854C8566
:1060B0005D85C701B6010F94A52D87FF04C0CA8670
:1060C000DB86EC86FD86202F322D4E855F85C7014D
:1060D000B6010F94CD36181624F40C2D2D2CEE8617
:1060E000FF861150D1F6FD81F150FD838885998599
:1060F000449699878887F111CBCF202F322D4E857A
:106100005F856A857B858C859D850F946D3420E045
:1061100030E040E05FE30F940B2EA30192010F9457
:106120006D342B013C012DEB37E346E855EB0F9422
:10613000CD3687FD0AC02DEB37E346E855E3C301B2
:10614000B2010F94A52D18165CF580E00E94A423DF
:1061500010E0EE80FF8000E0D7016D917D918D9180
:106160009D917D016D01B4E0CB1AD108A30192018C
:106170000F946C34F6016083718382839383602F64
:10618000812F0F94DB020F5F053031F71F5F8E8187
:106190009F8144969F838E831530D9F60E94B62541
:1061A00089288A288B2841F00E948F23882321F098
:1061B00090E080E00E943C2C8AE50E94D61F882354
:1061C00051F00E94AC1F69837A838B839C83CE013C
:1061D00001960F945D02832D0E94A4230CC0311000
:1061E00004C089288A288B2839F30E944A2E85E822
:1061F0009BE00E94C729332051F080916F0E8111DE
:1062000006C00E94DD2D86E69BE00E94C7290E9401
:106210004A2E88E59BE00E94C72980916F0E0E945C
:10622000B32C0E944A2E8BE49BE00E94C729C090A9
:106230009C0AD0909D0AE0909E0AF0909F0A20E070
:1062400030E0A901C701B6010F94CD3618160CF045
:1062500051C042E0C701B6010E9496820E94E275D9
:106260002A8D3B8D4C8D5D8D6091400F7091410F5B
:106270008091420F9091430F0F94A52D81111FC063
:106280002E893F89488D598D6091440F7091450F3B
:106290008091460F9091470F0F94A52D81110FC04B
:1062A0002091480F3091490F40914A0F50914B0F68
:1062B0006A897B898C899D890F94A52D81110E9403
:1062C00029BA6D960FB6F894DEBF0FBECDBFDF9131
:1062D000CF911F910F91FF90EF90DF90CF90BF90E3
:1062E000AF909F908F907F906F905F904F903F9076
:1062F0002F90089586E49BE00E94C729B1CFCF93E9
:10630000C82F82E0C11184E060E00E94DCEB0E94B3
:106310004A2E8EEA9AE0CC2311F083EC9AE0CF91DA
:106320000C94C729CF93DF93EB010E94C729CE01BC
:10633000DF91CF910C94CF1E5F926F927F928F92DC
:106340009F92AF92BF92CF92DF92EF92FF920F9304
:106350001F93CF93DF931F92CDB7DEB77C01390136
:106360008B015B01A40EB51ED12CC12CA016B10669
:1063700009F450C0F70180809180F80151908F019D
:106380005982C4010F94C3335816B9F1652DC40165
:106390000F94CB33FFEFCF1ADF0AC6018F7799270F
:1063A000892B21F162E070E080E090E00E94687249
:1063B000C4010F94C33399818917F9F00E944A2EC2
:1063C00083E897E00E94C72981E00F90DF91CF9189
:1063D0001F910F91FF90EF90DF90CF90BF90AF9003
:1063E0009F908F907F906F905F90089562E070E033
:1063F00080E090E00E94A626DBCFBE016F5F7F4F5A
:10640000C3010E947CE9F70180819181019691830B
:106410008083ACCF80E0D9CF0E94C7298AE00C945A
:10642000B6292F923F924F925F926F927F928F92F6
:106430009F92AF92BF92CF92DF92EF92FF920F9313
:106440001F93CF93DF93CDB7DEB7C659D1090FB6EF
:10645000F894DEBF0FBECDBF0E949C228823F1F1CD
:106460008091E6099091E709A091E809B091E909C6
:10647000AC01BD0132E176956795579547953A9500
:10648000D1F740FF45C084EA92E10E940C328EEFC2
:106490008093300A10922F0A81E09AE59093981623
:1064A000809397168CE490E090939A1680939916B7
:1064B00087E080938B1682E880938E1684E890E0C4
:1064C000A0E0B0E080938F1690939016A093911661
:1064D000B09392168BE396E10E943AC0CA56DF4F02
:1064E0000FB6F894DEBF0FBECDBFDF91CF911F91E5
:1064F0000F91FF90EF90DF90CF90BF90AF909F9063
:106500008F907F906F905F904F903F902F90089565
:1065100022E0B695A795979587952A95D1F780FFA4
:106520000CC00E947E220E9438A381E080930B174A
:106530000E9423820E946EC8D1CF409005095090DE
:106540000609609007097090080980910E0981FF83
:1065500005C09091100E98609093100E82FB8827D2
:1065600080F98093410A89E992E10E9461D7809184
:106570009508909196089E012F5F3F4F79010097F3
:1065800099F09F938F9381E992E19F938F933F932B
:106590002F930F943C2DC7010E9433D70F900F907B
:1065A0000F900F900F900F90809193089091940806
:1065B000843B910514F484EB90E09F938F9389E8DA
:1065C00092E19F938F93FF92EF920F943C2DC7011E
:1065D0000E9433D790916908CF56DF4F9883C159F5
:1065E000D04020916A08CE56DF4F2883C259D04050
:1065F00030916B08CD56DF4F3883C359D04080911E
:106600006C08CC56DF4F8883C459D0402091730862
:10661000309174084091750850917608692FCE56D4
:10662000DF4F7881C259D040CD56DF4F8881C359A2
:10663000D040CC56DF4F9881C459D0400F946D3470
:10664000962E872E382E292E81E892E10E9461D75E
:1066500080910E090F900F900F900F900F900F9058
:1066600080FDD8C1CF56DF4FA880C159D040CE564B
:10667000DF4FB880C259D040CD56DF4FC880C359D4
:10668000D040CC56DF4FD880C459D0408E010F5730
:106690001F4F23E041E0B501C6010F9416299F93D7
:1066A0008F9388E792E19F938F93FF92EF920F94DD
:1066B0003C2DC7010E9433D70F900F900F900F9081
:1066C0000F900F909501A601692D782D832D922DA5
:1066D0000F94CD361816FCF423E041E0692D782D97
:1066E000832D922D0F9416299F938F938EE692E11E
:1066F0009F938F93FF92EF920F943C2DC7010E94BE
:1067000033D70F900F900F900F900F900F90A92CF0
:10671000B82CC32CD22C86E692E10E9461D787E088
:106720008093260E8093400A609198087091990892
:1067300080919A0890919B088E010F571F4F21E07E
:1067400041E00F9416299F938F9380910E0983FB4C
:10675000882780F9CB56DF4F8883C559D040CA5669
:10676000DF4F1882C659D040CB56DF4F88819981C0
:10677000C559D040C0969F938F938BE592E19F932C
:106780008F93FF92EF920F943C2DC7010E9433D755
:1067900021E041E0B501C6010F9416299F938F9324
:1067A00082E592E19F938F93FF92EF920F943C2D9D
:1067B000C7010E9433D780910E090FB6F894DEBF4F
:1067C0000FBECDBF84FF1FC060918F0870919008ED
:1067D000809191089091920823E041E00F9416294E
:1067E0009F938F938AE492E19F938F93FF92EF920E
:1067F0000F943C2DC7010E9433D70F900F900F903C
:106800000F900F900F9080919308909194080097AB
:1068100099F09F938F9382E492E19F938F93FF92DD
:10682000EF920F943C2DC7010E9433D70F900F9029
:106830000F900F900F900F90809197088823A1F0F0
:106840001F928F931F921F9287E392E19F938F93E2
:10685000FF92EF920F943C2DC7010E9433D70FB6E1
:10686000F894DEBF0FBECDBF6091650870916608D9
:1068700080916708909168088E010F581F4F23E0A0
:1068800041E00F941629D82EC92E609161087091AD
:1068900062088091630890916408005F1F4F23E0B5
:1068A00041E00F941629CF92DF929F938F9389E254
:1068B00092E19F938F93FF92EF920F943C2DC7012B
:1068C0000E9433D723E041E0CF56DF4F6881C159A2
:1068D000D040CE56DF4F7881C259D040CD56DF4FE1
:1068E0008881C359D040CC56DF4F9881C459D040DD
:1068F0000F9416299F938F938FE192E19F938F932B
:10690000FF92EF920F943C2DC7010E9433D78091E4
:1069100072088F93809171088F9389E192E19F9320
:106920008F93FF92EF920F943C2DC7010E9433D7B3
:1069300060916D0870916E0880916F089091700859
:1069400023E041E00F9416299F938F9380E192E119
:106950009F938F93FF92EF920F943C2DC7010E945B
:1069600033D78CE0E7E7F8E0A1E1B8E001900D92C1
:106970008A95E1F78CE0E3E8F8E0A4E3BAE001905F
:106980000D928A95E1F780E00E9407B481E00E94B1
:1069900007B482E00E9407B480910D0980932F070D
:1069A00081E08093250E0E9486228CE998E09F93D7
:1069B0008F938AE095E29F938F93FF92EF920F94CB
:1069C0003C2D0FB6F894DEBF0FBECDBFC7010E94AD
:1069D00033D780910C098F9380910B098F9380910D
:1069E0000A098F93809109098F937F926F925F922A
:1069F0004F9284E092E19F938F93FF92EF920F94D6
:106A00003C2DC7010E9433D70FB6F894DEBF0FBEEE
:106A1000CDBF64CDA92CB82CC32CD22C37CECF93AC
:106A2000C82F41E06FEE71E10E94792EC11102C0C2
:106A30000E944A2E409136075091370760913807DF
:106A40007091390786EE91E10E94F5294091320755
:106A500050913307609134077091350783EE91E1CF
:106A60000E94F52980EE91E10E94C72982E496E117
:106A7000CF910C940C32CF93DF93EC0160E083E86C
:106A80009AE00E94B12BCE01DF91CF910C940C3291
:106A9000CF93DF93CDB7DEB7A8970FB6F894DEBFDC
:106AA0000FBECDBF8C017B01942E0E94B1860115D3
:106AB000110509F4C8C00E944A2EC8010E940C3278
:106AC000E114F10421F494E7E92E91E2F92E80918A
:106AD000310A80FD89C081608093310ACDB6DEB66F
:106AE00086E19AE00E940C3281E09AE59093981634
:106AF0008093971688E590E090939A168093991664
:106B000087E080938B1682E880938E1684E890E06D
:106B1000A0E0B0E080938F1690939016A09391160A
:106B2000B09392168BE396E10E943AC0C8010F948D
:106B3000F22C5C01C7010F94F22C8A0D9B1D039669
:106B40002DB73EB7281B390B0FB6F8943EBF0FBECA
:106B50002DBF8DB79EB701965C01FF92EF921F93F8
:106B60000F938FE09AE09F938F93BF92AF920F9411
:106B70003C2D8AE289838A838B838C83D501CE0165
:106B80000596EDB7FEB738960FB6F894FEBF0FBE68
:106B9000EDBFBE016F5F7F4FFC01E61BF70B2D9130
:106BA00021110BC0E60FF71F8AE29F01261B370B4E
:106BB0002832310534F48193F8CFFC012193CF01C1
:106BC000EBCF20E630E140E050E08BE396E10E941D
:106BD00099E96AE070E080E090E00E94D2BF0FB6D1
:106BE000F894DEBE0FBECDBE0E94DD2D83E39AE099
:106BF0000E94C72961E081E29AE00E94B12B89EEF0
:106C000093E0019739F000C00000EEE5F9E031971C
:106C1000F0F7F7CFF89489EE93E0019739F000C0D0
:106C20000000E6EEF3E03197F0F7F7CF0E94B1866F
:106C3000992031F00E9402940E94791EA895FECFFF
:106C40000E94C993F9CFE114F10421F484E7E82EFE
:106C500081E2F82E0AE21AE03ACF80915C0F90911F
:106C60005D0F2FEF3FEF981751F0E92FF0E0E45A56
:106C7000F04F228130E09F5F9F7790935D0FC901B5
:106C800008951F920F920FB60F9211240F900FBE0E
:106C90000F901F9018951F920F920FB60F9211240C
:106CA0000BB60F920F931F932F933F934F935F93C6
:106CB0006F937F938F939F93AF93BF93CF93DF9304
:106CC000EF93FF93C091C60000915D0FD0915C0FD0
:106CD00011E01D0F1F7790913B06913108F09FC086
:106CE000E92FF0E08827E858F94C8F4F0D94643471
:106CF0008936B836C736D636DD360F37E1360F3728
:106D0000E536E9360F37ED36F136F536FC360F3716
:106D10000737C03229F028F5CA3011F0CD3031F5EF
:106D2000011731F0ED2FF0E0E45AF04FC283D12F7C
:106D3000D0935C0FFF91EF91DF91CF91BF91AF9115
:106D40009F918F917F916F915F914F913F912F9183
:106D50001F910F910F900BBE0F900FBE0F901F90C1
:106D60001895CD3481F081E0CE3471F080E10CC013
:106D7000CA3338F4C033A0F6C03291F2CD32B1F745
:106D8000CFCFCD3499F782E080933B06C9CFC13392
:106D900059F018F4C03221F2E9CF88E0C433A1F3EE
:106DA0008BE0C83389F3E2CF83E0EECF84E0C033D9
:106DB00059F386E0C13341F3D9CF85E0C833B1F64A
:106DC000E3CF87E0C23391F6DFCF89E0C13371F6BC
:106DD000DBCF8AE0C03351F6D7CF8CE0C73331F632
:106DE000D3CF8DE0C63311F6CFCFC03209F498CFA0
:106DF0008EE0C33549F2BACF80ED8C0F8A3008F0AF
:106E00008FCF9FE090933B0680933C0689CFCA309A
:106E100019F0CD3009F084CF10923B0681CFCA30F3
:106E200019F0CD3009F07CCF809109178823A1F3A8
:106E3000973089F038F4953079F710922202109249
:106E4000730EEACF9A3059F09F3031F780913C06AB
:106E50000E94DD26E1CF81E080937E07DDCF81E0D7
:106E600080937D07D9CF8EBD0DB407FEFDCF089569
:106E70008FEF8EBD0DB407FEFDCF8EB508959091B6
:106E800064009B7F90936400982F906A96959CBDB8
:106E900080FD03C091E0863009F490E09DBD089527
:106EA0002F923F924F925F926F927F928F929F921A
:106EB000AF92BF92CF92DF92EF92FF920F931F9308
:106EC000CF93DF9300D000D01F921F92CDB7DEB7D3
:106ED000B82E80914910843008F0D8C10E949B726E
:106EE0006B017C0180914910811108C080915C0F79
:106EF00090915D0F891B8F7709F4D4C681E6A82E87
:106F000013C08A3019F08D3009F0F6C01092441089
:106F10008091E20F9091E30FFC01E252F04F168254
:106F2000892BF1F40E94548980914910843008F033
:106F3000ECC080915C0F90915D0F891B8F7709F4F5
:106F4000E4C00E942D3697FFDCCF0E94DD2D8FED2F
:106F500098E00E94C72980915C0F80935D0FE4CF79
:106F60001092E30F1092E20F04EE1FE0F8018191FE
:106F7000803209F446C08E3409F0A9C06AED78E089
:106F8000C8010F94222D4C01892B41F06EE470E072
:106F9000C80104960F94BB37009709F4C8014AE072
:106FA00050E070E060E001960F94922A2B013C01C2
:106FB0008091DE0F9091DF0FA091E00FB091E10F73
:106FC0000196A11DB11D481659066A067B0629F0D7
:106FD00060E087EA98E0892851F16AE270E0C80130
:106FE0000F94EA379C01009729F1982F901B912C60
:106FF000992349F09150F801E90FF11D80819826FD
:10700000F7CF8F01B3CF4AE050E070E060E0C901F4
:1070100001960F94922A292D30E050E040E062174B
:1070200073078407950751F060E088E898E00E94B4
:1070300022F27ACF60E08EE598E0F9CF4092DE0F41
:107040005092DF0F6092E00F7092E10F80915D0827
:107050008130E1F467E470E0C8010F94BB3700971A
:10706000A9F04AE050E070E060E001960F94922AA7
:10707000643071058105910548F48DEB97E00E941D
:10708000C72960E083EB97E00E94E2C2C092900AB9
:10709000D092910AE092920AF092930A8091E40FC2
:1070A0008B3309F441CF80914910843008F03CCFF4
:1070B00080914B108A9DC001112464EE7FE0845BB7
:1070C0009F4E0F94C63780E00E94DEF12DCF809155
:1070D000151780FFBBCF6DE677E2C8010F94222D14
:1070E000009731F0FC01838180538A3008F0AECFE5
:1070F00060E084E398E09BCF22EE3FE044EE5FE067
:1071000064E470E10E948ED20FCF8091151783FD49
:10711000BDC082FFBBC087FDB9C01A82198251E68B
:10712000F52E64E0E62E79E6D72E80914910843062
:1071300008F0ACC00E94C6D28111A8C041E050E066
:10714000BE016D5F7F4F89E798E10E948F7C0B81C4
:1071500010E0019711F00FEF1FEF809181189091CF
:107160008218A0918318B09184188093111790937E
:107170001217A0931317B09314170E94C6D20F3F93
:10718000100749F4811107C00E94DD2D8DEF98E0B2
:107190000E94C729CACF40914B10242F30E00A30FB
:1071A00061F00D3051F0882309F462C089819A8121
:1071B000009719F001969A8389831092C0068981FD
:1071C0009A81F29EF001F39EF00D1124E75BFF4ED1
:1071D000E80FF91F1382892B59F50E9454890E94E8
:1071E000C6D2882309F4A1CF89E798E10E943C7EAA
:1071F00080910C17882391F1815080930C178D9DFD
:10720000C001112462E08557984F0E949DA4E0912F
:107210000C1724E0E29FF0011124E957F84F608138
:107220007181828193810E9470D20E944D767DCFC0
:107230001A82198281E00E94DEF1809111179091EB
:107240001217A0911317B0911417809345109093C3
:107250004610A0934710B0934810C1CF0E94457EBE
:1072600080911517886080931517E0925D085DCFB7
:107270004F9DA0011124445B5F4E9E012F5F3F4F45
:1072800060EC76E0802F0E948ED24FCF0E949B72DE
:107290006B017C01B11004C080911309882351F067
:1072A000C0925C14D0925D14E0925E14F0925F1470
:1072B000BB24B39480912B0790912C07A0912D07AC
:1072C000B0912E070097A105B105B1F040915C1473
:1072D00050915D1460915E1470915F14840F951F3E
:1072E000A61FB71FA7019601281B390B4A0B5B0B82
:1072F000DA01C901B7FF08C1809107029091080225
:10730000A0910902B0910A02892B8A2B8B2B09F0DC
:107310000CC10E949B724B015C011091730E111104
:1073200008C0909135158091361511E0981301C071
:1073300010E020E030E04AE253E4609139147091AB
:107340003A1480913B1490913C140F94CD3687FDF4
:107350002FC181E0182781E04091C5065091C606F3
:107360006091C7067091C806452B462B472B09F440
:1073700080E0811799F080E090E0DC01112331F08A
:10738000D501C40180569444A24FBF4F8093C506D7
:107390009093C606A093C706B093C80640904C0FC2
:1073A00050904D0F60904E0F70904F0F2091C1067E
:1073B0003091C2064091C3065091C406C301B20188
:1073C0000F94A52D882319F18091C5069091C606CA
:1073D000A091C706B091C8064092C1065092C2065D
:1073E0006092C3067092C406892B8A2B8B2B09F4FA
:1073F00049C0D501C40180569444A24FBF4F809329
:10740000C5069093C606A093C706B093C8068091A0
:10741000C5069091C606A091C706B091C806009710
:10742000A105B10579F1881A990AAA0ABB0AB7FC25
:1074300029C01092C5061092C6061092C706109277
:10744000C8068DE599E00E94C72960E089E499E0CB
:107450000E94E2C280913D1490913E1418161906C4
:1074600024F490E080E00E9451AE80912614909127
:1074700027141816190634F41092271410922614A3
:107480000E9459238091D1069091D206A091D306F3
:10749000B091D40646015701881A990AAA0ABB0A74
:1074A000D501C401B7FDB8C130913515909136159D
:1074B0002091000280911202391709F47BC0E091FB
:1074C00036153BE6E39FF0011124E25FF44F908113
:1074D000899FC0011124880F892F881F990B9195CE
:1074E000281709F493C0809300020E949B72209198
:1074F0000002211162C01092C9061092CA061092B1
:10750000CB061092CC067CC00E94DD2D60918E0AC5
:1075100070918F0A8CE099E00E943FA240E070E0F9
:1075200060E090E080E00E944835909135158091B0
:107530003615981749F0C0925C14D0925D14E09211
:107540005E14F0925F14E5CEBB2019F01092D506C0
:10755000E0CE0E949B7200915C1410915D1420910A
:107560005E1430915F148090070290900802A09002
:107570000902B0900A02080D191D2A1D3B1D601B4F
:10758000710B820B930B97FDE1CF8091D506811192
:10759000C0CE81E08093D50680E00E94D89381E040
:1075A0000E94D89382E00E94D8930E94C993B1CEE2
:1075B00010E0D1CE9091B50A8BCF0091C906109101
:1075C000CA062091CB063091CC0601151105210584
:1075D000310581F46C597F4F8F4F9F4F6093C906DF
:1075E0007093CA068093CB069093CC068FEF80935E
:1075F000000206C0601B710B820B930B97FDF6CF48
:107600006091000270E089E00E9430F1809186076D
:10761000882309F4F4C000912D0210912E02C801B4
:10762000029720913D1430913E14281739070CF42D
:10763000E6C0809036158C821D821E821F821886BD
:10764000809135159C80891509F464C0892D90E0DE
:107650003BE6A32EA89EF001A99EF00D1124E8544C
:10766000F54F458956896789708D452B462B472BE9
:1076700081F4418D528D638D748D452B462B472BA4
:1076800041F4458D568D678D70A1452B462B472BB8
:10769000E1F12BE6B22EB89E9001B99E300D112477
:1076A000A9014854554F1A01FA0161817281838101
:1076B00094810F941B374B015C01F10161A172A110
:1076C00083A194A10F94AA2D2B013C01F10165A186
:1076D00076A187A190A50F94AA2D9B01AC01C301AF
:1076E000B2010F946735A50194010F940B2E4B0145
:1076F0005C012D813E814F8158850F94CD3618163F
:1077000024F48D829E82AF82B8868C818F5F8770D1
:107710008C8396CFB801110F880B990B0F94AC2D69
:107720005B018C01209127023091280240912902AF
:1077300050912A026D817E818F8198850F940B2E46
:107740009501A8010F946D342B013C0180902B0210
:1077500090902C029B01AC01B501C8010F94CD366D
:10776000181694F0B401990C880B990B0F94AC2D5A
:107770005B018C019B01AC01B201C3010F94CD36BA
:10778000181614F0520183014090CD065090CE0699
:107790006090CF067090D0069501A801C301B20198
:1077A0000F94CD361816D4F420E037ED43EA5CE3AD
:1077B000B501C8010F940B2E4B015C0128E431EE9A
:1077C0004AE75FE3C301B2010F940B2E9B01AC01AA
:1077D000C501B4010F946D345B018C01C501D80162
:1077E0008093CD069093CE06A093CF06B093D0069B
:1077F000B501C8010F94D935CB010E9451AEF4E612
:10780000CF0ED11CE11CF11CC092D106D092D20641
:10781000E092D306F092D4060E94548980915D08CC
:10782000882309F4E1C18091710E882309F4A4C072
:1078300080915407882309F49FC08091700E8111B4
:107840009BC08091130981110AC08091621481301C
:1078500031F08091151782FF8FC087FD8DC0F8949D
:1078600080915407873009F0D8C18CB1829581701E
:107870009091D60698278093D60680915307892B3E
:107880008093530760914B0770914C0780914D078F
:1078900090914E07789420E030E0A9010F94A52D37
:1078A00087FF6AC001E00093700E80911309811177
:1078B00061C082E799E00E940C3284E080933A0F25
:1078C00081E09AE590939816809397168EE490E065
:1078D00090939A168093991687E080938B1682E88E
:1078E00080938E1684E890E0A0E0B0E080938F163D
:1078F00090939016A0939116B09392168BE396E115
:107900000E943AC00E94E22B0093631440E366EBAE
:1079100079E08DE199E20E94E72B61E081E199E253
:107920000E94C92B10911E0760E0102789E39BE09D
:1079300069F484EA99E00E94B12B80E30E94B629A1
:107940008AE00E94B62960E087E899E00E94B12BA6
:1079500082E999E00E94C72980E30E94B6298AE063
:107960000E94B629112331F08DE899E09093B50E6D
:107970008093B40E0E94F3AE90910901892F8095F7
:107980008170109101021817C9F020911517206419
:10799000209315178093010290FD61C164EF71E09F
:1079A00080E090E00E94A6260E946D7E80911517CF
:1079B00084FDA0C1111155C10E9429C90E949B726A
:1079C0006B017C01109106021123F1F080913E09B8
:1079D0008823D1F04091D7065091D8066091D906FE
:1079E0007091DA0646015701841A950AA60AB70A69
:1079F000B501A40177FD1AC0833009F44EC10CF023
:107A00003DC181300CF042C1212F30E0A8EEB3E03F
:107A10000F943534C60ED71EE81EF91EC092D70645
:107A2000D092D806E092D906F092DA0680916214DC
:107A3000813009F073C00E949B726B017C018091C0
:107A4000DF069091E006A091E106B091E206A70161
:107A50009601281B390B4A0B5B0BDA01C901B7FDF4
:107A60003AC0D701C601805F984DAF4FBF4F80939A
:107A7000DF069093E006A093E106B093E2068090C3
:107A8000460A9090470AA090480AB090490A0E947E
:107A90000ABEAB01BC014093460A5093470A60936B
:107AA000480A7093490A8091020890910308A091B6
:107AB0000408B091050888199909AA09BB09840F1F
:107AC000951FA61FB71F8093020890930308A093E9
:107AD0000408B09305088091DB069091DC06A09124
:107AE000DD06B091DE0646015701881A990AAA0AF6
:107AF000BB0AD501C401B7FD11C020E8C20E2EEEAD
:107B0000D21E26E3E21EF11CC092DB06D092DC06F8
:107B1000E092DD06F092DE060E94CAAD0E94A7C187
:107B20000E94E6DA80912A07882379F10E949B72ED
:107B30006B017C018091260790912707A09128076F
:107B4000B091290746015701881A990AAA0ABB0A67
:107B5000D501C401B7FD19C020912A0730E0A8EE75
:107B6000B3E00F943534C60ED71EE81EF91EC0923E
:107B70002607D0922707E0922807F092290780E095
:107B80000E9438838AE00E94B629809125078823C5
:107B900059F10E949B726B017C01809121079091A9
:107BA0002207A0912307B0912407A7019601281B63
:107BB000390B4A0B5B0BDA01C901B7FD15C02091E7
:107BC000250730E0A8EEB3E00F943534C60ED71E7B
:107BD000E81EF91EC0922107D0922207E0922307E7
:107BE000F09224070E941A7628960FB6F894DEBF0A
:107BF0000FBECDBFDF91CF911F910F91FF90EF90FE
:107C0000DF90CF90BF90AF909F908F907F906F90BC
:107C10005F904F903F902F900895882309F432CEC3
:107C2000649B63C091E0823009F090E081E09111A3
:107C300014C091E0891326CE80914F079091500790
:107C4000A0915107B091520780934B0790934C0736
:107C5000A0934D07B0934E0715CE90E0EBCF0E9456
:107C6000557E123008F0AACE0E9429C9A7CE87EC13
:107C700099E09093B50E8093B40EA0CE843009F0B5
:107C8000C3CE0E944A2E8EEC99E004C00E944A2E78
:107C90008DEF99E00E94C729B7CE0E944A2E86EE4A
:107CA00099E0F8CF8091900A9091910AA091920A60
:107CB000B091930AA7019601281B390B4A0B5B0B65
:107CC000DA01C901885E9340A109B109B7FD16C95F
:107CD00087EF98E00E94C729C092900AD092910A3B
:107CE000E092920AF092930A09C9823009F4A4CF73
:107CF00080E09FCF123018F40E94D5DA5FCE1230A8
:107D000009F05CCE0E947C82882379F081E00E9499
:107D1000ACA240EB50E060E678E08AE197E10E9497
:107D20008F7C8AE197E10E943C7E0E949C22811117
:107D30009ECF0E947E220E9438A381E080930B1781
:107D40000E9423823BCE2F923F924F925F926F927E
:107D50007F928F929F92AF92BF92CF92DF92EF92DB
:107D6000FF920F931F93CF93DF93CDB7DEB7CA591E
:107D7000D1090FB6F894DEBF0FBECDBF80916F0E54
:107D8000888B8091E6099091E709A091E809B0916C
:107D9000E909AC01BD01E6E17695679557954795F0
:107DA000EA95D1F740FF00C10E948F23811107C0DF
:107DB0000E94DD2D82E39CE00E94C7290FC18AE565
:107DC0000E942420882339F10E94AC1F2091580F73
:107DD0003091590F40915A0F50915B0F0F946C34B2
:107DE0006B017C0120E030E040E251ECC701B601BC
:107DF0000F94CD3687FD0AC020E030E040E251E428
:107E0000C701B6010F94A52D181674F40E94DD2D3C
:107E100085E29CE0D1CFC090480FD090490FE09010
:107E20004A0FF0904B0FDECF40E050E060EC7FE770
:107E300088E50E9431202091500F3091510F4091E0
:107E4000520F5091530F0F946C342B013C0140E0C2
:107E500050E060EC7FE789E50E9431202091540FCB
:107E60003091550F4091560F5091570F0F946C342D
:107E70004B015C016FEF89E40E946520182F6FEFC2
:107E80008AE40E946520082FA3019201C301B20178
:107E90000F945F37811156C0A5019401C501B4014B
:107EA0000F945F3781114EC020914A0A30914B0ADE
:107EB00040914C0A50914D0AC301B2010F946C34A9
:107EC0002091520A3091530A4091540A5091550A18
:107ED0000F94673520E030E040E05FE30F946D34AD
:107EE0000F94D935162F20914E0A30914F0A4091A8
:107EF000500A5091510AC501B4010F946C3420917D
:107F0000560A3091570A4091580A5091590A0F94D5
:107F1000673520E030E040E05FE30F946D340F946C
:107F2000D935062F812F012E000C990B97FD34C0F7
:107F30000597A4F5802F002E000C990B97FD30C0FB
:107F4000059784F5153008F049C0053008F046C0A3
:107F500080E00E94A42325E01202F0011124E00F2A
:107F6000F11D07FDFA95EE0FFF1FEE0FFF1FEA54FC
:107F7000F14FC082D182E282F3820E94B625602F47
:107F8000812F0F94DB0288890E94A423888988238B
:107F900029F10E9429BA22C010E0CCCF14E0CACF48
:107FA00000E0D0CF04E0CECF69E0B695A7959795D5
:107FB00087956A95D1F780FD0CC070E060E086E59A
:107FC0000E9448209A838983059710F180E09CE005
:107FD000F3CE80E00E94A4230E943726C656DF4FCE
:107FE0000FB6F894DEBF0FBECDBFDF91CF911F91CA
:107FF0000F91FF90EF90DF90CF90BF90AF909F9048
:108000008F907F906F905F904F903F902F9008954A
:1080100060E084E40E9471208F8740E050E0BA0164
:108020008AE50E9431206BA77CA78DA79EA740E020
:1080300050E86BE376E483E50E94312020E030E0F5
:1080400040E752E40F946735609323027093240253
:1080500080932502909326020091301510913115DE
:10806000F801C080D180E280F38020E030E0A901F7
:10807000C701B6010F946D34C956DF4F6883C759E5
:10808000D040C856DF4F7883C859D040C756DF4F1D
:108090008883C959D040C656DF4F9883CA59D0400B
:1080A00020E030E040E251E40F94A52D87FF16C098
:1080B000C956DF4F1882C759D040C856DF4F1882C3
:1080C000C859D040F0E2C756DF4FF883C959D040B5
:1080D00021E4C656DF4F2883CA59D04020E030E85B
:1080E0004DE953E4C701B6010F946D34CD56DF4F0F
:1080F0006883C359D040672ECC56DF4F8883C4595C
:10810000D040CB56DF4F9883C559D04020E030E0B7
:1081100041E953E40F94CD36181694F4CD56DF4F51
:108120001882C359D040612C31E9CC56DF4F3883D7
:10813000C459D04083E4CB56DF4F8883C559D04023
:10814000F80184809580A680B78020E030E0A90106
:10815000C501B4010F946D347B018C0120E030E047
:1081600040EA51E40F94A52D87FF04C0E12CF12CC7
:1081700000EA11E420E030E04BE953E4C501B4012A
:108180000F946D34B62EC72ED82ECA56DF4F988363
:10819000C659D04020E030E04CE853E40F94CD368F
:1081A000181654F4B12CC12C5CE8D52EF3E4CA5651
:1081B000DF4FF883C659D04088E40E94D61F882339
:1081C00009F45FC20E94AC1F0F94D9351B0177FFE1
:1081D00002C06F5F7F4F75956795719561957109C5
:1081E0006A567F4F072E000C880B990B0F94AC2D0D
:1081F000762E872E982EA92E9701A8010F94CD36A2
:10820000181624F4E72CF82C092D1A2DC956DF4F27
:108210002881C759D040C856DF4F3881C859D0404F
:10822000C756DF4F4881C959D040C656DF4F5881E5
:10823000CA59D040672D782D892D9A2D0F94CD36AF
:108240001816A4F0C956DF4F7880C759D040C856D9
:10825000DF4F8880C859D040C756DF4F9880C95932
:10826000D040C656DF4FA880CA59D040872D982DE0
:10827000A92DBA2D8B8B9C8BAD8BBE8BC701D801E2
:108280008F8B988FA98FBA8FB101330C880B990B04
:108290000F94AC2D1B012C01AC019B01B701C8014F
:1082A0000F946D347B018C012B2D3C2D4D2DCA5626
:1082B000DF4F5881C659D0400F94A52D87FF08C0C5
:1082C000BE2CCF2CD02ECA56DF4F1883C659D040B3
:1082D000A2019101672D782D892D9A2D0F946D346F
:1082E0007B018C01CD56DF4F2881C359D040362DFC
:1082F000CC56DF4F4881C459D040CB56DF4F588110
:10830000C559D0400F94A52D87FF10C0CD56DF4F23
:10831000E882C359D0406F2CCC56DF4F0883C45934
:10832000D040CB56DF4F1883C559D040CD56DF4FD4
:108330008881C359D040962DCC56DF4FA881C459AF
:10834000D040CB56DF4FB881C559D0408B8F9C8F22
:10835000AD8FBE8F8B2D9C2DAD2DCA56DF4FB881B2
:10836000C659D0408F8F98A3A9A3BAA3BE01695E56
:108370007F4FCE0143960E94926D882309F4D0C1AD
:10838000BE01615E7F4FCE014B960E94926D082F19
:10839000882309F4C5C12F89388D498D5A8D6F8D79
:1083A00078A189A19AA10F946C3420E030E040E8D4
:1083B0005EE30F940B2E6B017C012B893C894D8968
:1083C0005E896B8D7C8D8D8D9E8D0F946C3420E03D
:1083D00030E040E85EE30F940B2E6BA37CA38DA3EB
:1083E0009EA3CFA2D8A6E9A6FAA689819A811816DB
:1083F000190674F48EEC9BE00E94C7298F858823B0
:1084000021F084EC9BE00E94C7298AE00E94B629F3
:108410000E94F3AE0E9491B780E00E94A423809155
:108420005F08811103C081E00E94F3BB8F85811139
:1084300046C02091520A3091530A4091540A5091FB
:10844000550A6BA17CA18DA19EA10F94A52D811130
:1084500030C02091560A3091570A4091580A5091E5
:10846000590A6FA178A589A59AA50F94A52D811108
:1084700020C020914A0A30914B0A40914C0A5091F9
:108480004D0A6B897C898D899E890F94A52D811158
:1084900010C020914E0A30914F0A4091500A5091DD
:1084A000510A6F89788D898D9A8D0F94A52D882317
:1084B00031F080E00E94A4230E943726188A60E0F1
:1084C00085E40E947120882309F42DC121E0CD5656
:1084D000DF4F2883C359D0401B861C861D861E860D
:1084E0001A8A902E24E9C22E2BE0D22E32EAA32E35
:1084F0003BE0B32EFA8884E08F150CF42CC16B8519
:108500007C858D859E859B01AC010F945F37811121
:1085100022C1992009F40EC191E0CC56DF4F988317
:10852000C459D04095E0292E91E099261F2D110FB6
:10853000110F1F0D1F5F898BF9886A89F21409F4E6
:1085400006C1062E000C770B880B990B0F94AC2DEF
:108550002FA138A549A55AA50F940B2E2F89388D28
:10856000498D5A8D0F946D342B013C016F2DFF0CFA
:10857000770B880B990B0F94AC2D2BA13CA14DA12F
:108580005EA10F940B2E2B893C894D895E890F9437
:108590006D346B837C838D839E834F82588669867E
:1085A0007A8689819A81892B79F0612F80EB9BE013
:1085B0000E94A92B69E170E08EEA9BE00E94923153
:1085C0008BEA9BE00E94C7291F92F9E1FF931F925B
:1085D0001F93DF92CF92BF92AF921F920E94BEEF85
:1085E0002981CD56DF4F4881C359D040BE01695F14
:1085F0007F4FCE0103960E94C46E2B013C014B8637
:108600005C866D867E860FB6F894DEBF0FBECDBF4A
:10861000AC019B010F945F37811196C089883A881D
:1086200035E0282D230370011124E30CF11C37FCE5
:10863000FA94EE0CFF1CEE0CFF1C81E090E08C0F16
:108640009D1FE80EF91EA30192016BA57CA58DA5C7
:108650009EA50F946D34F70166A777A780AB91AB09
:10866000632D882D0F94DB02188A81E00E94503719
:108670001F5F8989CC56DF4FF881C459D0408F0FD6
:108680005ACFA701B80186E40E9431201B012C01BA
:10869000C956DF4F4881C759D040C856DF4F58816F
:1086A000C859D040C756DF4F6881C959D040C65617
:1086B000DF4F7881CA59D0408CE40E9431206B8B07
:1086C0007C8B8D8B9E8B2F8A388E498E5A8E4B2DAC
:1086D0005C2D6D2DCA56DF4F7881C659D04082E49B
:1086E0000E9431206B017C01CD56DF4F4881C35978
:1086F000D040562DCC56DF4F6881C459D040CB5660
:10870000DF4F7881C559D04082E50E9431206B8FC0
:108710007C8F8D8F9E8FCF8ED8A2E9A2FAA226CE13
:1087200084EE9BE049CB33E0CD56DF4F3883C3590D
:10873000D040D2CEEFEFCC56DF4FE883C459D040C3
:1087400022242A9484E0F0CE88890E94A4238A8976
:108750008F5F8A8BCFCE0E942CEC0E941F1F882334
:1087600059F088890E94A42380E090E0A0ECBFE744
:108770008B879C87AD87BE876B857C858D859E8525
:108780009B01AC010F945F37811133C08F85882323
:10879000D1F1CE018F960E943C2C8F85811124C08F
:1087A00088E49FE00E94281F6B017C0180E49FE029
:1087B0000E94C9239B01AC01C701B6010F940B2E87
:1087C0009B01AC016091480F7091490F80914A0F55
:1087D00090914B0F0F946C346093480F7093490F36
:1087E00080934A0F90934B0F8F85811108890093D6
:1087F0006F0E0E9478B780916F0E81110E9427BA88
:108800000E94B51EC6CBBE016D5E7F4FCE01839622
:108810000E94CA2584E6FE01BF96A6EBBEE0019049
:108820000D928A95E1F70E94B62590E080E0B3CFE3
:10883000CF93DF93C82FD62F8091100E83FD14C0E5
:108840008091410A811110C08091330290913402CD
:108850009C012150310940913D1450913E14421722
:10886000530714F40E9451AE6D2F8BE00E94DCEB95
:10887000CC2331F061E080E0DF91CF910C94A983AB
:108880008091410A91E089278093220280912202FF
:108890008823F1F020E030E040E05FE3609139149C
:1088A00070913A1480913B1490913C140F946D3464
:1088B0000F94D93520913D1430913E14621B730BF7
:1088C00077FF03C07195619571096230710544F4B9
:1088D000109222028091100E83FF06C0C1E01AC0E0
:1088E00080E00E945037D2CFC091410AC11112C01E
:1088F0008091330290913402019720913D14309180
:108900003E142817390754F70E944A2E8DE99AE041
:108910000E94C7298C2FDF91CF910895AF92BF920B
:10892000CF92DF92EF92FF920F931F93CF93DF933B
:10893000CDB7DEB764970FB6F894DEBF0FBECDBFDC
:108940000E944E2E87FDABC08AE50E94242088231A
:1089500009F4B6C040E050E0BA018AE50E94312037
:108960007B018C0163E085E00E94DCEB2091480FE5
:108970003091490F40914A0F50914B0F60E070E0E9
:1089800088EC93E40F946C345B016C019701A801AF
:108990000F94CD36181614F075018601C701D80161
:1089A0008D839E83AF83B88720E030E0A901B701B3
:1089B000C8010F94A52D882321F0CE0105960E94B1
:1089C0007C1E80E090E0A0EAB1E489879A87AB87BB
:1089D000BC871D861E861F86188A8CE40E94D61FBF
:1089E000882309F472C00E94AC1F6B017C0120E057
:1089F00030E0A901C701B6010F94CD3687FF04C04E
:108A0000F7FAF094F7F8F094C98ADA8AEB8AFC8ACC
:108A100000913D1410913E1404301105DCF020E06B
:108A200030E040E05FE36091391470913A14809136
:108A30003B1490913C140F946D340F94D935601B06
:108A4000710B77FF03C071956195710901E0643086
:108A500071050CF400E063E080E00E94184481118D
:108A60003DC063E089E00E94DCEB6D817E818F81F7
:108A700098858B019C01305809831A832B833C8392
:108A800020E030E0A9010F94A52D882321F0CE012C
:108A900001960E947C1E60E089E00E94DCEB6496F7
:108AA0000FB6F894DEBF0FBECDBFDF91CF911F91FF
:108AB0000F91FF90EF90DF90CF90BF90AF9008950F
:108AC000E12CF12C00E211E44DCFC0903607D0909C
:108AD0003707E0903807F090390789CF83E0E82E18
:108AE00022E0AE01475F5F4FBE016F5E7F4FCE0158
:108AF0000D960E94876CB9CF4F925F926F927F92D2
:108B0000AF92BF92CF92DF92EF92FF921F93CF93DB
:108B1000DF9300D000D01F921F92CDB7DEB75C016B
:108B2000E62EF42E642F80E00E941844182F811145
:108B30001BC0EE2021F060E089E00E94DCEB812F79
:108B400028960FB6F894DEBF0FBECDBFDF91CF9150
:108B50001F91FF90EF90DF90CF90BF90AF907F90EC
:108B60006F905F904F900895EE2021F06F2D83E07D
:108B70000E94DCEB80E090E0A0E7B2E48D839E836E
:108B8000AF83B88780E090E0A0E8B0EC89839A8357
:108B9000AB83BC83BE016B5F7F4FCE0101960E9409
:108BA0006BB968E873E180E090E00E94A626C12CD2
:108BB000D12C88ECE82E81E4F82ECD82DE82EF8283
:108BC000F88680E090E0A0E8B0E489839A83AB83E4
:108BD000BC83BE016B5F7F4FCE0101960E946BB9D3
:108BE00040905F0E5090600E6090610E7090620E2B
:108BF000C0925F0ED092600EE092610EF092620E13
:108C000080E090E0A0EAB1E48D839E83AF83B887D3
:108C1000F50180819181A281B38189839A83AB839D
:108C2000BC83BE016B5F7F4FCE0101960E946BB982
:108C300040925F0E5092600E6092610E7092620ED2
:108C40000E94C99364E670E080E090E00E94A6264E
:108C500076CF8F929F92AF92BF92CF92DF92EF9298
:108C6000FF921F93CF93DF9300D000D01F921F92EB
:108C7000CDB7DEB70E944E2E182F87FDACC08AE517
:108C80000E942420812C912C90E2A92E91E4B92EEF
:108C9000882341F040E050E0BA018AE50E9431208B
:108CA0004B015C0164E083E00E94DCEB20E030E0FB
:108CB000A901C501B4010F94CD3618167CF580E0EA
:108CC00090E0A0EAB0E48D839E83AF83B8872091C3
:108CD000480F3091490F40914A0F50914B0FC501F9
:108CE000B4010F946D346B017C0120E030E048EC5E
:108CF00053E40F94A52D87FD06C0C12CD12C88EC20
:108D0000E82E83E4F82EC982DA82EB82FC82BE016F
:108D10006B5F7F4FCE0101960E94FCB885E50E94F3
:108D2000D61F882309F469C00E94AC1F6B017C0127
:108D300020E030E0A901C701B6010F94CD3687FFCE
:108D400004C0F7FAF094F7F8F094F7FAF094F7F813
:108D5000F094C982DA82EB82FC8244E061E0CE01C9
:108D600001960E947C4520E030E0A901C501B401D4
:108D70000F94CD3618165CF580E090E0A0EAB0E4E0
:108D80008D839E83AF83B887A50194016091480FBE
:108D90007091490F80914A0F90914B0F0F946C3452
:108DA0006B017C0120E030E0A9010F94CD3618164C
:108DB0001CF0C12CD12C7601C982DA82EB82FC82B4
:108DC000BE016B5F7F4FCE0101960E94FCB860E050
:108DD00089E00E94DCEB28960FB6F894DEBF0FBE48
:108DE000CDBFDF91CF911F91FF90EF90DF90CF909B
:108DF000BF90AF909F908F90089588E01802F00187
:108E00001124EE5CF84FC080D180E280F38090CFD7
:108E10002F923F924F925F926F927F928F929F928A
:108E2000AF92BF92CF92DF92EF92FF920F931F9378
:108E3000CF93DF9300D000D000D0CDB7DEB74C0188
:108E40008B014987590161E089E39BE00E94B12BC6
:108E500040E059E260E47BE085E00E94D3EB909132
:108E6000130981E0890F809313098091151782FB04
:108E7000222720F9288782FF08C087FDCDC08B7F7D
:108E8000809315179E5F909313090E94A3C280E1FF
:108E9000E0E4FFE0A4E2B9E001900D928A95E1F7E9
:108EA00087E00E9427B4782E60E070E080E090E4D4
:108EB000711040C02090480F3090490F40904A0FE9
:108EC00050904B0F20E030E040E050E4C201B1018F
:108ED0000F946D346B017C0120E030E048EC53E4EA
:108EE0000F94CD36181634F4C12CD12C88ECE82E12
:108EF00093E4F92EF8016084F185FD83F801F28591
:108F0000FE83F801F385FF839601A701662D7D811D
:108F10008E819F2F0F94CD36181624F06C2CDD8295
:108F2000EE82FF82A2019101662D7D818E819F815B
:108F30000F946C342885222349F02091250E22239A
:108F400029F041E0711040E00E9486200E94F3AEBB
:108F500080911109811109C081E0809311098091EC
:108F6000B50A809310091092B50A20E030E0A901FB
:108F7000F40160817181828193810F94A52D8823F2
:108F800091F00E945DAE81110EC080E090E0A0E7FC
:108F9000B2E489839A83AB83BC83BE016F5F7F4F4A
:108FA000C4010E946BB9711004C0B80180E00E9436
:108FB00057BE20E030E0A901F50160817181828116
:108FC00093810F94A52D882329F042E06985C5017E
:108FD0000E947C450E94C99364E670E080E090E0C6
:108FE0000E94A62681E029960FB6F894DEBF0FBE38
:108FF000CDBFDF91CF911F910F91FF90EF90DF9048
:10900000CF90BF90AF909F908F907F906F905F9028
:109010004F903F902F900895188637CFCF92DF92D0
:10902000EF92FF92CF93DF936B017C01D42FC0911D
:109030003E0983E080933E0981E08093730EC11462
:10904000D104E104F10431F00E949B72C60ED71ED8
:10905000E81EF91E8091730E882389F0C114D10493
:10906000E104F10421F48D2F0E945037F3CF0E94C8
:109070009B726C197D098E099F0997FDF4CF1092A0
:10908000730EC0933E09DF91CF91FF90EF90DF9078
:10909000CF900895FF920F931F93CF93DF93CDB797
:1090A000DEB72D970FB6F894DEBF0FBECDBF082FE9
:1090B000162F0E947F3161E0812F0E94EA220E94D8
:1090C0009B72685370458F4F9F4F60933409709324
:1090D0003509809336099093370910923809F0903A
:1090E0003E0983E080933E0930E020E042E459E20B
:1090F0006BE27BE082E00E940A2C8BE29BE00E9404
:109100003CC881E08093730E8091730E882309F42C
:109110006AC060E0812F0E94EA228091380988238A
:1091200009F45DC060E08AE00E94DCEB0E944A2EF8
:1091300081E19BE00E94C72930E020E04BEF5AE03C
:1091400062E07BE082E00E940A2C82E09BE00E94C9
:109150003CC841E060E070E0CB010E940E4830E086
:1091600020E050E040E06EEE7AE085E00E940A2CBC
:109170006EEE7AE0CE0101960F94EB2CCE010196B3
:109180000E945AC20E940CBF60E080E00E94184416
:10919000802F0E947F310E949B72685370458F4FD1
:1091A0009F4F6093340970933509809336099093EB
:1091B00037091092380930E020E042E459E262EECB
:1091C0007AE082E00E940A2C82EE9AE00E943CC87B
:1091D00081E08093730E61E0812F0E94EA2281E09A
:1091E0000E94503791CFF0923E092D960FB6F89419
:1091F000DEBF0FBECDBFDF91CF911F910F91FF90CA
:109200000895BF92CF92DF92EF92FF920F931F9338
:10921000CF93DF93CDB7DEB7A0970FB6F894DEBF3C
:109220000FBECDBF0E944E2E87FDDCC061E081E005
:109230000E94DCEB85E40E942420882309F4E2C02C
:109240000E94AC1F6B017C0120E030E0A9010F946B
:10925000CD3687FF04C0F7FAF094F7F8F094F7FAE8
:10926000F094F7F8F094C98EDA8EEB8EFC8E8CE0D9
:10927000E3E7F2E0DE01119601900D928A95E1F7A5
:1092800088E50E942420882351F040E050E0BA0194
:1092900088E50E94312069837A838B839C8389E5EA
:1092A0000E942420882351F040E050E0BA0189E573
:1092B0000E9431206D837E838F8398878AE50E9488
:1092C0002420882351F040E050E0BA018AE50E9452
:1092D000312069877A878B879C87C0903207D0902E
:1092E0003307E0903407F090350785E50E9424208D
:1092F000882321F00E94AC1F6B017C0120E030E04C
:10930000A901C701B6010F94CD3687FF04C0F7FA53
:10931000F094F7F8F094F7FAF094F7F8F094CD8E13
:10932000DE8EEF8EF8A262E070E082E40E944820B8
:10933000B82E80911309811155C09E01235E3F4FC5
:1093400041E0BE016F5F7F4FCE0149960E94084702
:10935000882309F447C06B2D81E00E944A4870E0E1
:1093600060E082E50E9448208C0180E090E0A0EA65
:10937000B1E48D8B9E8BAF8BB88FC0903607D090A9
:109380003707E0903807F09039078CE40E942420DA
:10939000882321F00E94AC1F6B017C0120E030E0AB
:1093A000A901C701B6010F94CD3687FF04C0F7FAB3
:1093B000F094F7F8F094C98ADA8AEB8AFC8A1D8661
:1093C0001E861F86188A80911309882359F02B2D39
:1093D000AE014B5E5F4FBE016F5E7F4FCE010D96BB
:1093E0000E9449AAA0960FB6F894DEBF0FBECDBF6B
:1093F000DF91CF911F910F91FF90EF90DF90CF9071
:10940000BF900895C12CD12C80E8E82E80E4F82E7E
:1094100026CFCF92DF92EF92FF920F931F93CF93BD
:10942000DF93CDB7DEB76C970FB6F894DEBF0FBEF3
:10943000CDBF8CE40E942420882309F4AFC00E9491
:10944000AC1F6B017C0120E030E0A9010F94CD3608
:1094500087FF04C0F7FAF094F7F8F094F7FAF09465
:10946000F7F8F094C98EDA8EEB8EFC8E8CE0E3E791
:10947000F2E0DE01119601900D928A95E1F788E500
:109480000E9424208823A1F040E050E0BA0188E542
:109490000E9431202091500F3091510F4091520F76
:1094A0005091530F0F946C3469837A838B839C8320
:1094B00089E50E9424208823A1F040E050E0BA0111
:1094C00089E50E9431202091540F3091550F409131
:1094D000560F5091570F0F946C346D837E838F839A
:1094E00098878AE50E942420882351F040E050E0CC
:1094F000BA018AE50E94312069877A878B879C8729
:1095000061E080E00E94DCEB1D861E861F86188AC3
:1095100080911309811133C09E01235F3F4F40E0CA
:10952000BE016F5F7F4FCE0149960E940847882396
:1095300031F160E080E00E944A48898D9A8DAB8DC0
:10954000BC8DB0588D8B9E8BAF8BB88F198A1A8AC1
:109550001B8A1C8A1D861E861F86188A8091130905
:10956000882369F010E000E020E0AE014B5E5F4F21
:10957000BE016F5E7F4FCE010D960E9449AA6C9688
:109580000FB6F894DEBF0FBECDBFDF91CF911F9114
:109590000F91FF90EF90DF90CF900895C12CD12CC8
:1095A00080E8E82E80E4F82E59CF2F923F924F9218
:1095B0005F926F927F928F929F92AF92BF92CF9263
:1095C000DF92EF92FF920F931F93CF93DF93CDB76C
:1095D000DEB764970FB6F894DEBF0FBECDBFD82EAE
:1095E000662E442E26E0829F80011124F801ED585A
:1095F000F04FA590B490C8018F58904F7C01FC01AA
:1096000025903490F501808190E095958795F10142
:1096100020812370382F3470722E732AF4E04F1398
:1096200002C08870782A30E3532E5D0C87E69FE0F5
:109630000E94C729852D0E94B629862D0E94B62931
:1096400083E00E94BD29862C062C000C9908F401A9
:10965000E154F10923E0D29EE00DF11D1124EE0F3B
:10966000FF1FED5BF04FCE0101966C0193E04912B4
:10967000ABC0A591B4918C911F928F9389E39FE029
:109680009F938F93DF92CF920F943C2DC6010E943F
:10969000E8750F900F900F900F900F900F90672D1F
:1096A00085E29FE00E94A92BF701C590D49089E93B
:1096B0009EE00E94C729852D0E94B629862D0E9412
:1096C000B629F601608170E083E090E0881999097D
:1096D000880F991F02C0759567958A95E2F76370A8
:1096E000772786E99EE00E949231F50160816770DC
:1096F00070E08CE19FE00E94923183E19FE00E9444
:10970000C729852D0E94B629F10160818FE09FE075
:109710000E94A92B86E09FE00E94C729852D0E9408
:10972000B629F501608182E09FE00E94A92BF80133
:10973000EB58F04F0591149188EF9EE00E94C729E5
:10974000852D0E94B629F801608185EF9EE00E9478
:10975000A92BF0EC6F0E23E0872D421240C0897FC9
:1097600021F481EA9EE00E94C729F801808190E0FF
:1097700002C0959587956A94E2F780FF04C08AEB52
:109780009EE00E94C729F801808180FF04C087ED18
:109790009EE00E94C72964960FB6F894DEBF0FBE04
:1097A000CDBFDF91CF911F910F91FF90EF90DF9090
:1097B000CF90BF90AF909F908F907F906F905F9071
:1097C0004F903F902F900895A591B49111968C9150
:1097D00011978F938C918F938FE29FE051CF8B7F66
:1097E00009F4BFCF84EF870D823008F0BECFB9CF28
:1097F000CF93DF93C82FD0E0FE01E258F74DE491FC
:10980000E150E231F0F4F0E08827E65FF34B8F4F50
:109810000D9464341C4C4C4C4F4C534C564C214CC6
:10982000594C5D4C604C644C674C6A4C6E4C714CAE
:10983000214C744C784C7B4C43E061E480E00E9406
:10984000D54A8BEB9FE00E94C729FE01EE50F84DF0
:10985000E491E23009F052C0FE01E85CF74DE4917A
:10986000E03809F04BC087EB9FE00E94C72982E1F6
:109870000E94BD298FEA9FE00E94C72985E99FE0E9
:109880000E94C7298EE00E94BD2944E063E481E084
:10989000DF91CF910C94D54A43E062E4CFCF44E00E
:1098A00061E481E0CCCF44E062E4FBCF44E063E4D8
:1098B000F8CF43E061E482E0C2CF43E062E4FBCF53
:1098C00044E061E483E0BBCF44E062E4FBCF44E0EA
:1098D00063E4F8CF44E061E484E0B1CF44E062E4C3
:1098E000FBCF44E063E4F8CF44E061E485E0A7CF38
:1098F00044E062E4FBCF44E063E4F8CFDF91CF9132
:1099000008950F931F93CF93DF93CDB7DEB764977E
:109910000FB6F894DEBF0FBECDBFE82FF0E0E258DF
:10992000F74DE491E150E23108F006C1F0E08827FC
:10993000E356F34B8F4F0D946434AF4CD64CE04C50
:10994000EE4CFC4C9C4D0A4D164D224D304D3E4D7B
:109950004C4D5A4D684D9C4D754D824D8F4D84B583
:10996000807C09F4E9C087B51F928F938CE89EE054
:109970009F938F938E010F5F1F4F1F930F930F9431
:109980003C2DC8010E94E8750F900F900F900F902A
:109990000F900F9081E064960FB6F894DEBF0FBE73
:1099A000CDBFDF91CF911F910F91089584B5807342
:1099B00009F4C2C088B51F928F9382E89EE0D8CF89
:1099C00080918000807C09F4B7C0809188009091DC
:1099D00089009F938F9388E79EE0CACF8091800093
:1099E000807309F4A9C080918A0090918B009F93A5
:1099F0008F938EE69EE0BCCF809180008C7009F43E
:109A00009BC080918C0090918D009F938F9384E6F2
:109A10009EE0AECF8091B000807C09F48DC0809133
:109A2000B3001F928F938AE59EE0A2CF8091B00091
:109A3000807309F481C08091B4001F928F9380E5F8
:109A40009EE096CF80919000807C09F475C0809153
:109A50009800909199009F938F9386E49EE088CF21
:109A600080919000807309F467C080919A00909172
:109A70009B009F938F938CE39EE07ACF8091900020
:109A80008C7009F459C080919C0090919D009F9327
:109A90008F9382E39EE06CCF8091A000807C09F4DC
:109AA0004BC08091A8009091A9009F938F9388E26A
:109AB0009EE05ECF8091A000807309F43DC080914C
:109AC000AA009091AB009F938F938EE19EE050CFC0
:109AD0008091A0008C7081F18091AC009091AD00DC
:109AE0009F938F9384E19EE043CF80912001807CFF
:109AF00019F180912801909129019F938F938AE019
:109B00009EE036CF809120018073B1F080912A01D0
:109B100090912B019F938F9380E09EE029CF8091BD
:109B200020018C7049F080912C0190912D019F9320
:109B30008F9386EF9DE01CCF80E02DCF2F923F9238
:109B40004F925F926F927F928F929F92AF92BF924D
:109B5000CF92DF92EF92FF920F931F93CF93DF93F9
:109B6000CDB7DEB7AB970FB6F894DEBF0FBECDBF53
:109B7000782E6BA7442E7901D12CC12C19A6612C0B
:109B8000082F082E000C110B2AEC280F2AA7CE0153
:109B900001965C01F601E45BFF4E5490852C912CFC
:109BA0008016910609F084C0611057C0E114F104D9
:109BB00019F0C7010E94C72984E490E10E94C729D7
:109BC0001F925F928FE390E19F938F93BF92AF922A
:109BD0000F943C2DC5010E94E875872D0E94D52960
:109BE0000F900F900F900F900F900F908AA587FD08
:109BF00030C096E3891A91089F928F9285E390E195
:109C00009F938F93BF92AF920F943C2DC5010E94FA
:109C1000E8750F900F900F900F900F900F90F60136
:109C2000E65BFF4E25903490912C812CF101E80DDC
:109C3000F91D549051101DC087E290E088199909D0
:109C40004C0158141904FCF480E20E94B629539484
:109C5000F8CF88E00E94BD29E2CF8EE20E94B629AB
:109C60008AE1E114F104B1F3C7010F94F22C865E8E
:109C7000F1CF852D0E94B6299FEF891A990A27E214
:109C80008216910499F6442069F0872D0E946B1E7C
:109C9000882309F493C08BA5811190C08AE290E1DA
:109CA0000E94C7298AE00E94B62969A666246394A7
:109CB00024E0C20ED11C8CECC816D10409F06ACF86
:109CC000611063C0E114F10419F0C7010E94C729B3
:109CD0008FEF9FE00E94C7291F930F938AEF9FE0A9
:109CE0009F938F93CE0101967C019F938F930F9446
:109CF0003C2DC7010E94E875872D0E94D5298AEC6A
:109D0000D82ED70C0F900F900F900F900F900F90B0
:109D1000D7FC93C0065311091F930F9380EF9FE068
:109D20009F938F93FF92EF920F943C2DC7010E9457
:109D3000E8750F900F900F900F900F900F908FED90
:109D40009FE00E94C7294420E9F0872D0E94814CA2
:109D5000811112C0872D0E94521E882309F471C000
:109D600087E10E94BD2985E090E10E94C729872DE7
:109D70000E94341E0E94CF1E87E10E94BD29872DBC
:109D80000E94F84B8AE00E94B629AB960FB6F89471
:109D9000DEBF0FBECDBFDF91CF911F910F91FF901E
:109DA000EF90DF90CF90BF90AF909F908F907F907B
:109DB0006F905F904F903F902F900895F601E35B76
:109DC000FF4EE491E11122C08AA50E944B72092E38
:109DD000000CAA0BBB0BBF93AF939F938F9389E1AA
:109DE00090E19F938F93BF92AF920F943C2DC5014A
:109DF0000E94E8750FB6F894DEBF0FBECDBF99A5DF
:109E0000911150CF872D0E94F84B4CCF872D0E9487
:109E1000521E81110AC08FE090E10E94C729872D50
:109E20000E94341E0E94CF1EEACF872D0E94814CD3
:109E30008111E5CF85E090E1F0CF88E00E94BD2957
:109E40007ECF9FE09D1510F18D2D0E944B72092E43
:109E5000000CAA0BBB0BBF93AF939F938F938BEC1C
:109E60009FE09F938F93FF92EF920F943C2DC70139
:109E70000E94E87587EC9FE00E94C7290FB6F8940E
:109E8000DEBF0FBECDBF8FE090E16FCF87E10E94B4
:109E9000BD29F9CF2F923F924F925F926F927F929E
:109EA0008F929F92AF92BF92CF92DF92EF92FF92EA
:109EB0000F931F93CF93DF93CDB7DEB74DB65EB64A
:109EC00084E50E94D61F882309F493C060E089E4EA
:109ED0000E947120082F61E070E082E50E94482016
:109EE0006C0170E060E083E50E944820182F65E473
:109EF00070E08CE40E9448205C0164EF71E087E52B
:109F00000E9448203C01990F880899081A151B04E3
:109F100011F00CF052C01634A0F4011114C0812FBE
:109F20000E946B1E882379F028E231E141E060E075
:109F3000812F0E949E4D8AE00E94B6298AE00E94ED
:109F4000B6291F5FE3CFA8952DE131E141E0602FF5
:109F5000812F0E949E4D812F0E94521E382E61E05B
:109F6000812F0E940F72F12CE12CEC14FD0404F5FA
:109F7000A89560E0812F0E949E71C401B3010E94E8
:109F8000A626A89561E0812F0E949E71C401B301AD
:109F90000E94A626A89560E0812F0E949E71C401B0
:109FA000B3010E94A626A8952FEFE21AF20ADDCF90
:109FB000632D812F0E940F72C1CF86E191E10E9433
:109FC000C7290FB6F8945EBE0FBE4DBEDF91CF918C
:109FD0001F910F91FF90EF90DF90CF90BF90AF90C7
:109FE0009F908F907F906F905F904F903F902F90B9
:109FF000089585E40E94D61F8823B1F00E94091FAE
:10A000008093850783E891E10E94C72980918507A5
:10A01000811107C085E791E10E94C7298CE791E192
:10A02000CECF89E791E1F8CF83E50E94D61F882340
:10A0300029F00E94DD2D83E391E1C1CF70E060E063
:10A0400080E50E9448208C01F82E80E50E942420A3
:10A05000811149C035E485E4E82E301708F4B1CF0A
:10A0600060E089E40E947120782E60E087E50E941C
:10A070007120882309F491C0ADB6BEB686E691E1A1
:10A080000E94C729480199248E2D90E088199909CA
:10A090000196EDB7FEB7E81BF90B0FB6F894FEBFBB
:10A0A0000FBEEDBF2DB73EB72F5F3F4F6901E016E2
:10A0B00010F10634B0F47720C1F062E0802F0E94E6
:10A0C0000F7261E070E080E090E00E946872802F83
:10A0D0000E947571E02FF0E0E819F909EC0DFD1D03
:10A0E00080830F5FE4CFE02EBBCF802F0E946B1EDA
:10A0F000882319F3F6CF20903E0983E080933E0930
:10A1000081E08093730E30E020E042E459E266E59E
:10A1100071E182E00E940A2C86E491E10E943CC831
:10A120006F2C10E000E0E61418F135E43615E0F08D
:10A130007720A9F0862D0E947571382E4601800E79
:10A14000911EF4018081381679F030E020E040E083
:10A15000672D862D0E949E4DF401308205C0862D0C
:10A160000E946B1E882331F363940F5F1F4FDBCF78
:10A170000E94E6DA8091730E882339F068EC70E073
:10A1800080E090E00E94A626CBCF20923E090FB639
:10A19000F894BEBE0FBEADBE14CFEF1408F411CFBD
:10A1A000F5E4FF1538F030E020E041E0672D8F2D19
:10A1B0000E949E4DF394F1CF2F923F924F925F9267
:10A1C0006F927F928F929F92AF92BF92CF92DF92C7
:10A1D000EF92FF920F931F93CF93DF93CDB7DEB72C
:10A1E000CB56D1090FB6F894DEBF0FBECDBFAC96EB
:10A1F0008FAFAC97C0903E092D96CFAE2D9721E042
:10A2000020933E098091E5098D3409F41AC78435FD
:10A2100011F40C94BE65873409F045C10091E3093F
:10A220001091E4090B31110509F469C308F03EC12E
:10A230000430110508F02FC180915D08023011052E
:10A2400008F4C9C1833008F4CCC1332433940230FC
:10A25000110509F0312C0E944A2182E50E94242038
:10A26000882309F4D5C10E94AC1F6B017C0120E05A
:10A2700030E0A9010F94A52D882309F405C1409071
:10A28000400F5090410F6090420F7090430F20910B
:10A29000440F3091450F4091460F5091470F2CA726
:10A2A0003DA74EA75FA78090140990901509A09034
:10A2B0001609B09017098091180990911909A09179
:10A2C0001A09B0911B0988AB99ABAAABBBABA5012E
:10A2D0009401C301B2010F94A52D81110DC028A9CD
:10A2E00039A94AA95BA96CA57DA58EA59FA50F9448
:10A2F000A52D882309F4C8C0A3019201C501B401AA
:10A300000F946C3420E030E040E05FE30F940B2EBC
:10A3100068A779A78AA79BA72CA53DA54EA55FA5F1
:10A3200068A979A98AA99BA90F946C3420E030E030
:10A3300040E05FE30F940B2E6CA77DA78EA79FA72D
:10A3400020E030E0A901C701B6010F94A52D881FB8
:10A350008827881F381609F452C120E030E040E811
:10A360005FEB28AB39AB4AAB5BAB28A539A54AA557
:10A370005BA5CA01B9010F940B2E4B015C012CA502
:10A380003DA54EA55FA5CA01B9010F940B2E9B01F7
:10A39000AC01C501B4010F946D340F941B374B0110
:10A3A0005C01AC019B01C701B6010F946C342B0119
:10A3B0003C01A5019401C701B6010F946D349B01C6
:10A3C000AC01C301B2010F940B2E6B017C0120E0A4
:10A3D00030E0A9010F94CD36412C512C320187FD7C
:10A3E00006C0C701B6010F941B372B013C016CA5B9
:10A3F0007DA58EA59FA59058A50194010F94673562
:10A4000028A939A94AA95BA90F940B2EA30192018F
:10A410000F940B2E28A539A54AA55BA50F946D3482
:10A420006B017C01A501940168A579A58AA59BA56E
:10A430000F94673528A939A94AA95BA90F940B2E57
:10A44000A30192010F940B2E2CA53DA54EA55FA54F
:10A450000F946D3468A779A78AA79BA720E030E006
:10A46000A901C701B6010F94A52D81110C940066B6
:10A4700020E030E0A90168A579A58AA59BA50F94E5
:10A48000A52D81110C9400660E94DD2D84E393E1DB
:10A490000E94C729A6C00430110509F4F6C1053190
:10A4A000110509F49EC00F944B049BC00A3211059C
:10A4B00009F443C408F080C00D31110509F40BC440
:10A4C00008F436C20E31110571F700913015109164
:10A4D0003115D8012D913D914D915C916091400FC6
:10A4E0007091410F8091420F9091430F0F946D3402
:10A4F000AB01BC0188E50E94312069837A838B839C
:10A500009C83F80124813581468157816091440FF5
:10A510007091450F8091460F9091470F0F946D34C5
:10A52000AB01BC0189E50E9431206D837E838F835E
:10A530009887BE016B5F7F4FCE0101960E94926D9E
:10A54000882309F44EC080E00E94A4230E9491B7A2
:10A5500061E085E40E947120182F21E0482FBE01A0
:10A560006B5F7F4FCE0101960E94C46E6B017C0130
:10A57000AC019B010F945F37811116C049815A814C
:10A580006B817C8186E893E10E94F5294D815E8193
:10A590006F81788581E893E10E94F529B701A601D2
:10A5A0008CE793E10E94062A0E9478B711110E945D
:10A5B000B51E0E9429BA15C00B35110509F498C4BF
:10A5C0000C35110509F498C40A35110509F06BCF53
:10A5D00010922F0706C0833020F00E944A210E946B
:10A5E000E9B4AC96CFACAC97C11002C00F94F8039D
:10A5F0002D96DFAC2D97D0923E090C940D5F80E034
:10A6000090E0A0E8BFE388AB99ABAAABBBABADCE03
:10A6100089E40E942420C12CD12C7601882321F0CA
:10A620000E94AC1F6B017C018AE40E9424208823D5
:10A6300011F40C94F1650E94AC1F0CCF2CA93DA91C
:10A640004EA95FA96CA57DA58EA59FA50F940B2E85
:10A650006B017C0128AD39AD4AAD5BAD68A979A924
:10A660008AA99BA90F940B2E9B01AC01C701B601CF
:10A670000F946D346B017C0128AD39AD4AAD5BADF3
:10A680006CA57DA58EA59FA50F940B2E4B015C019B
:10A690002CA93DA94EA95FA968A979A98AA99BA956
:10A6A0000F940B2E9B01AC01C501B4010F946C34C7
:10A6B000A70196010F94EC346B017C0120E030E09F
:10A6C000A9010F94A52D882309F4D4C020E030E01F
:10A6D000A901C701B6010F94A52D87FF2CC082E008
:10A6E00090E083298130910549F1029791F120E0B2
:10A6F00030E0A901C701B6010F94CD3646015701DC
:10A7000087FF04C0B7FAB094B7F8B0942BED3FE0E0
:10A7100049EC50E4C501B4010F94673520E030E006
:10A7200040E952E40F940B2E0F944B350F94E03513
:10A730008B010C94DD6690E080E0D3CF2BED3FE001
:10A7400049EC50E4C701B6010F946C346B017C01F5
:10A75000CECF2BED3FE049EC50E4C701B6010F949A
:10A760006D34F4CF08E410E07BED872E7FE0972E68
:10A7700079ECA72E70E4B72E750164010C94DD66A8
:10A780005DEC852E5CEC952EA92C5DE3B52E0C942A
:10A790009C67B10190E080E00F94AA2D2CAD3DADF7
:10A7A0004EAD5FAD0F940B2E4B015C010F946235E3
:10A7B0006B017C01C501B4010F940D374B015C01A5
:10A7C000A70196016CA57DA58EA59FA50F940B2EC4
:10A7D0002B013C0128A539A54AA55BA5C501B401FB
:10A7E0000F940B2E9B01AC01C301B2010F946D3489
:10A7F0002B013C01A50194016CA57DA58EA59FA50B
:10A800000F940B2E4B015C0128A539A54AA55BA529
:10A81000C701B6010F940B2E9B01AC01C501B40119
:10A820000F946C3468AB79AB8AAB9BAB49E14CAB12
:10A830000C94176980E1E4E1F9E0DE0111960190E2
:10A840000D928A95E1F7CE0101960E9441B420E075
:10A8500030E0A901BE01645E7F4FCE0101960F94E6
:10A86000820180E1FE013196A0E4BFE001900D92EB
:10A870008A95E1F70E949B7260935C1470935D145B
:10A8800080935E1490935F14ACCE80E50E942420E8
:10A89000C12CD12C7601882321F00E94D51E6B019A
:10A8A0007C0183E50E942420882361F00E94AC1F74
:10A8B00020E030E04AE754E40F940B2E0F94E0358B
:10A8C0006B017C010E94F3AE8091DD13811105C004
:10A8D00060E08AE493E10E94E2C20E949B72C60E8D
:10A8E000D71EE81EF91E0E949B726C197D098E0905
:10A8F0009F0997FF76CE80E00E945037F4CF87E023
:10A900000E945AD881116DCE8CE0EFE7F2E0DE01B3
:10A91000119601900D928A95E1F770E060E080E574
:10A920000E945720BE016F5F7F4F0E9457BE59CED5
:10A9300087E00E9427B4811111C08091E6099091AF
:10A94000E709A091E809B091E9092EE0B695A7952D
:10A95000979587952A95D1F780FD43CE0E94F3AE57
:10A960001092360260916F0E8CE40E947120A82E26
:10A9700080E00E94A4230E949B7260935C147093F9
:10A980005D1480935E1490935F140E9491B781E0F0
:10A9900080930F080E94E4BBC090E609D090E709BD
:10A9A000E090E809F090E90989E1F694E794D794FA
:10A9B000C7948A95D1F7C0FE0DC081E00E9427B4EC
:10A9C000182F82E00E9427B411110C94ED6511E05C
:10A9D000811101C010E08091E6099091E709A091F2
:10A9E000E809B091E90907E1B695A795979587958C
:10A9F0000A95D1F780FF02C00C94DF6511114BC19D
:10AA00008091E9098170B82E811347C18C2D817026
:10AA1000B12E811342C111E0BB24B39401E082E561
:10AA20000E942420F82E60E070E080E890E4F110AD
:10AA30000E94AC1F6CA37DA38EA39FA320E030E0F7
:10AA4000A9010F94A52D882371F0F11007C01111F1
:10AA500005C0B11003C0002309F42DC160E0CE0190
:10AA600084960E941BB9112309F45AC0BB2009F433
:10AA700054C01092400F1092410F1092420F10924A
:10AA8000430F1092440F1092450F1092460F1092F0
:10AA9000470F0E9427BA8EED9BE6ADE8B2E488A38B
:10AAA00099A3AAA3BBA38DE391E30E94191F20E001
:10AAB00030E040EC5FE30F940B2E905869837A836B
:10AAC0008B839C8389E391E30E94191F20E030E08F
:10AAD00040EC5FE30F940B2E90586C8F7D8F8E8F20
:10AAE0009F8FAE01405E5F4FBE016F5F7F4FCE0113
:10AAF0004C960E94DAB80E94FCBD1092400F109252
:10AB0000410F1092420F1092430F1092440F109277
:10AB1000450F1092460F1092470F80E00E9460BCD4
:10AB2000BB2019F081E00E9460BC002309F4C3C07F
:10AB30008091E6099091E709A091E809B091E909AF
:10AB4000F7E0B695A79597958795FA95D1F780FD8B
:10AB50009EC083E00E945AD88111ADC00E9427BADE
:10AB60002091110830911208409113085091140857
:10AB700060E070E086E193E40F946C346B017C013B
:10AB80002091150830911608409117085091180827
:10AB900060E070E086E193E40F946C342B013C019B
:10ABA0008091480F9091490FA0914A0FB0914B0F9F
:10ABB00080931C0990931D09A0931E09B0931F094F
:10ABC0000091301510913115D8012D913D914D9185
:10ABD0005C91C701B6010F946C346B017C01C0928B
:10ABE0001409D0921509E0921609F0921709F8019C
:10ABF0002481358146815781C301B2010F946C34A1
:10AC00002B013C01409218095092190960921A09CF
:10AC100070921B0927E137EB41ED58EB0F94CD36CD
:10AC200087FD3EC023E030E04BE953E4C301B201AD
:10AC30000F94A52D1816A4F127E137EB41ED58EB41
:10AC4000C701B6010F94CD3687FD2AC023E030E856
:10AC50004DE953E4C701B6010F94A52D181604F170
:10AC60001C8E1D8E1E8E1F8E88E0E4E1F9E0DE0151
:10AC7000119601900D928A95E1F7AE01445E5F4F07
:10AC8000BE016B5F7F4FCE0101960E94DAB882E071
:10AC90000E9460BC10C0B12E10E00C2D0170BFCE20
:10ACA00060E085E693E10E94E2C20E944A2E83E5BD
:10ACB00093E10E94C7290E9427BA80910E088093D1
:10ACC0000F08AA2019F081E00E94A4230E9478B7FF
:10ACD0000E9429BA86CC0E949B7260935C14709388
:10ACE0005D1480935E1490935F1480916F0E8111B8
:10ACF0001DC08091E6099091E709A091E809B09103
:10AD0000E909EDE0B695A79597958795EA95D1F76E
:10AD100080FF04C086E793E10E9461D787E00E942C
:10AD20005AD881115ECC0E94A33E5BCC60E08FE4D8
:10AD30000E9471208823E9F254CC80915D08833011
:10AD400008F44FCC89E40E942420E82E00E08823F8
:10AD500019F00E94A81F082F8AE40E942420F82ED0
:10AD600010E0882319F00E94A81F182FEE2011F080
:10AD7000053020F4FF2039F0153028F08EE893E1FB
:10AD80000E94C7292ECC80E1E0E4FFE0A4E1B9E015
:10AD900001900D928A95E1F7EE2019F1602F000FD6
:10ADA000770B880B990B0F94AC2D2091520A3091A0
:10ADB000530A4091540A5091550A0F940B2E20913A
:10ADC0004A0A30914B0A40914C0A50914D0A0F9417
:10ADD0006D3460931409709315098093160990934C
:10ADE0001709FF2019F1612F110F770B880B990BB1
:10ADF0000F94AC2D2091560A3091570A4091580A71
:10AE00005091590A0F940B2E20914E0A30914F0AFF
:10AE10004091500A5091510A0F946D346093180973
:10AE20007093190980931A0990931B0960E080E5DB
:10AE30000E9471208823C1F1EE20D1F0E0913015FD
:10AE4000F091311520813181428153816091140943
:10AE50007091150980911609909117090F946C341F
:10AE6000609314097093150980931609909317093C
:10AE7000FF20D1F0E0913015F0913115248135811A
:10AE800046815781609118097091190980911A09BA
:10AE900090911B090F946C346093180970931909F1
:10AEA00080931A0990931B0940E050E0BA0186E4B0
:10AEB0000E9431206B017C0120E030E0A9010F9459
:10AEC000CD3618168CF420E030E040E752E4C7019C
:10AED000B6010F94673569837A838B839C83CE0197
:10AEE00001960E94B0B77DCB60E070E0CB01F3CF5C
:10AEF0008FE080932F0775CB8091E209882381F141
:10AF0000893009F06ECB6BE8A62E62E0B62E70E4B5
:10AF1000C72E7FE0D72EE12C00E010E0D5018D9107
:10AF20005D010E942420F82E882361F0133011F077
:10AF3000E82EF02E0E94AC1FF6016083718382839D
:10AF400093830F2D1F5FF4E0CF0ED11C143031F727
:10AF5000EE2009F464C00E9427BA0E9429BA41CBAE
:10AF60005BE8C52E52E0D52EF12CE12C00E010E07C
:10AF7000D6018D916D010E942420382E882309F47A
:10AF800047C00E94AC1F4B015C01133059F0F70120
:10AF9000E05BF04F20813181428153810F946C340A
:10AFA0004B015C01F701E05CF04F2081318142816F
:10AFB0005381C501B4010F946C342B013C012DEB7E
:10AFC00037E346E855EB0F94CD3687FD0AC02DEBED
:10AFD00037E346E855E3C301B2010F94A52D1816D7
:10AFE000BCF4133021F1F701EC5CF54F5F01A301D4
:10AFF000920160817181828193810F946D34D501BA
:10B000006D937D938D939C931397812F0E9407B42A
:10B010001F5FB4E0EB0EF11C143009F0A9CF002340
:10B0200009F49BCF8CE49FE00E9488B296CF809277
:10B030004C0F90924D0FA0924E0FB0924F0F032DD8
:10B04000E7CF8091E3099091E4098837910511F4E5
:10B050000C940D6108F0CCC18C34910509F43AC60A
:10B0600008F0EEC08A31910509F44DC508F093C08F
:10B070008431910509F486C408F06EC081319105D0
:10B0800009F425C408F042C0029708F00CCA80E514
:10B090000E942420C12CD12C7601882321F00E940B
:10B0A000D51E6B017C0183E50E942420882361F07A
:10B0B0000E94AC1F20E030E04AE754E40F940B2ECE
:10B0C0000F94E0356B017C010E94F3AE8091EA0998
:10B0D0009091EB09009709F4F5C30E946FC6809127
:10B0E000E3099091E4096FEA73E1892B11F467EAAF
:10B0F00073E130E020E042E459E282E00E940A2C51
:10B1000040E0C701B6010E940E486BCA429709F0A1
:10B11000CAC983E50E942420882309F45AC70E94E3
:10B120009B7260935C1470935D1480935E14909393
:10B130005F140E94AC1F20E030E04AE754E40F9413
:10B140000B2E0F94E03560930702709308028093F2
:10B15000090290930A0245CA8731910509F44FC448
:10B1600080F48531910509F446C4469709F09BC9DE
:10B170008091151782FF02C087FF33CA0E94557E57
:10B1800030CA8831910509F454C4499709F08BC934
:10B190000E94094A26CA8032910509F444C5B0F5D7
:10B1A0008D31910509F428C570F48B31910509F4AE
:10B1B000BDC44C9709F077C98091EA099091EB09D9
:10B1C0000E945FA20ECA8E31910509F41CC54F97EB
:10B1D00009F069C90E940ABE6C8F7D8F8E8F9F8F88
:10B1E000BE016F5F7F4FCE014C960E9491D160E00F
:10B1F000CE0101960E9422D80E944A2EBE016F5FA6
:10B200007F4F82E294E10E943FA2EBC98B3291050D
:10B2100009F438C550F48132910509F42FC58A9795
:10B2200009F041C90E94E12DDCC98934910509F476
:10B230002DC58B34910509F036C90E942E27D1C93E
:10B240008B36910509F403C608F098C08435910542
:10B2500009F45FCF50F58135910509F49AC6B0F431
:10B260008D34910509F43AC58E34910509F01BC956
:10B2700070E060E083E50E9448208E34910509F07B
:10B2800032C50E94F0AD0E942CECABC9823591050D
:10B2900009F497C68335910509F005C980912F07F8
:10B2A0008F7E806280932F079CC98836910509F4B0
:10B2B0009BC5E0F58535910509F4CEC68C35910521
:10B2C00009F0F1C80E944E2E87FD8BC98091E609D6
:10B2D00084FD09C08091E80987FD05C08091E909D6
:10B2E000837009F441C77BE8C72E72E0D72EE7E2EE
:10B2F000EE2EEEE0FE2E10E0D6018D916D010E9443
:10B300002420882351F0133009F4CBC60E94AC1FCF
:10B31000F701648B758B868B978B1F5FF4E0EF0EC4
:10B32000F11C143049F70E94CFAE5BC989369105F4
:10B3300009F45FC58A36910509F0B5C860E080E57B
:10B340000E94652081114DC98091E6096091B50A7E
:10B35000062F80FD02C00FEF10E083E50E9424203D
:10B36000882349F00E94E51E8B016F3F710519F09B
:10B3700010F00FEF10E00093B50A33C98137910543
:10B3800009F4BFC5D0F48E36910509F46BC560F49D
:10B390008C36910509F425C98D36910509F083C8CD
:10B3A00081E00E94F3D01DC98F36910509F46DC567
:10B3B0008037910509F415C976C88537910509F4D8
:10B3C000E0C658F48237910509F4D3C68337910556
:10B3D00009F069C80E944ED604C98637910509F460
:10B3E000E3C68737910509F05EC80E9473BBF9C8B0
:10B3F0008239E1E09E0711F40C940B6408F02FC130
:10B40000833D910511F40C944C6208F058C0883CBF
:10B41000910509F412C7D0F48C38910509F48DC553
:10B4200048F48937910509F400C78D37910509F46F
:10B43000AFCE39C88B39910509F484C58E3B91058F
:10B4400009F031C881E00E9413CFCBC88C3C910534
:10B4500009F48FC7D0F4893C910509F42CC78B3CC3
:10B46000910509F020C88091E60984FD5FC78091AD
:10B47000E809887809F05AC78091E909837009F0D2
:10B4800055C781E00E94B12AACC88D3C910509F4F2
:10B49000C5C78E3C910511F00C9453528091E6097A
:10B4A0009091E709A091E809B091E909892B8A2BCD
:10B4B0008B2B09F0B7C781E00E9411D792C88D325B
:10B4C00021E0920711F40C94026308F06CC0823EF4
:10B4D000910511F40C94AD6208F045C08C3D9105C6
:10B4E00009F4DEC78D3D910511F00C9453520E9472
:10B4F0004E2E082F87FD75C883E50E942420002E5C
:10B50000000C110B7801EE0CFF1C882311F40C9435
:10B5100093620E94A81FF701EB5AFD4F918380832D
:10B52000000F111F000F111FF801EF5AFD4F7F018F
:10B53000BC01990F880B990B0F94AC2D2AE037EDC5
:10B5400043E25CE30F940B2E0F5E114FD8012D9157
:10B550003D914D915C910F940B2EF70160837183A7
:10B56000828393833EC8823241E0940711F40C94A5
:10B57000FE628C32914011F00C94535264E071E001
:10B5800083E50E9457208C0168EE73E080E50E94FD
:10B590005720893823E1920710F088E893E1B80139
:10B5A0000E942DC21EC88033A1E09A0711F40C94AA
:10B5B0004C6310F58E32E1E09E0711F40C94966313
:10B5C0008F32914011F00C94535270E060E085E4AA
:10B5D0000E944820F82E3FEF831711F40C94046466
:10B5E000882311F40C94DC6380E295E10E94C72962
:10B5F0000E9484EE0C94F152803921E0920711F4FC
:10B600000C9407648139914011F00C945352C0900E
:10B61000E609D090E709E090E809F090E90987E0B1
:10B62000F694E794D794C7948A95D1F741E0C42261
:10B63000DD24EE24FF2483E50E94D61FCD28CE28EA
:10B64000CF2811F00C94F15281110C94F152809199
:10B650005F08811182CC81E00E94F3BB7ECC8C30EC
:10B6600042E0940711F40C94ED6408F0D1C08C3AD8
:10B67000A1E09A0711F40C94266408F095C08D3966
:10B68000E1E09E0711F40C94A86578F48A3921E072
:10B69000920711F40C94F1528C39914011F00C94F2
:10B6A00053520E94982E0C94F152843A41E0940730
:10B6B00011F40C941364853A914011F00C94535298
:10B6C0006FEF7FEF89E40E944820082F6FEF7FEF34
:10B6D0008AE40E944820182F8AE50E942420D12C59
:10B6E000811108C081E50E942420D82E882311F4FE
:10B6F0000C94E565C02E81E0800F863010F00C942C
:10B700001E64912E81E0810F863010F00C941E642F
:10B710000E94AC1F2B013C01F02E07FDF12C07FF0E
:10B7200002C004E0C02E812E17FD812C17FF02C03D
:10B7300014E0912EB5E03B2ECF1410F40C941A6453
:10B74000E82C3F9C500111249E1410F40C941764B3
:10B750000E2D10E020E030E0A901DD2069F0F501B8
:10B76000E00FF11FEE0FFF1FEE0FFF1FEA54F14F26
:10B7700020813181428153810A0D1B1D000F111F51
:10B78000000F111F0A54114FC301B2010F946D3401
:10B79000D8016D937D938D939C9313976E2D8F2D70
:10B7A0000F94DB02E394D0CF863FA1E09A0711F417
:10B7B0000C94DF6478F4843FE1E09E0711F40C946C
:10B7C000DB64853F914011F00C9453520E942DA1EF
:10B7D0000C94F152873F21E0920711F40C94E3643A
:10B7E000883F914011F00C94535281E080934307BD
:10B7F0000E94AFAD10924307882311F40C94F152CC
:10B800000E944A2E89EB95E10E94C7290C94F152BF
:10B81000833543E0940711F40C94946520F58B353F
:10B82000A2E09A0711F40C94036570F48F34E2E0FF
:10B830009E0709F436CF8835924011F00C9453528C
:10B840000E9401490C94F1528D3B22E0920711F4C1
:10B850000C9490658E3B924011F00C9453520E94D0
:10B8600029460C94F152873E43E0940711F40C945E
:10B870009865C8F48C36A3E09A0711F40C94F15241
:10B88000803A934011F00C9453522091EA09309180
:10B89000EB0990911517926090931517C9010E94BA
:10B8A0005FA20C94F152883EE3E09E0711F40C94E1
:10B8B000BA65893E934011F00C9453520E94D3D73D
:10B8C0000C94F15287EB93E10E943CC808CC0E9493
:10B8D000231E882309F444C085E40E94D61F8823D0
:10B8E00061F080911F0790912007892B21F00E9421
:10B8F000A81F811102C00E94D1938091E609909106
:10B90000E709A091E809B091E90947E1B695A79543
:10B91000979587954A95D1F780FF03C080E00E94F4
:10B920000D948091E90980FF03C081E00E940D948D
:10B930008091E6099091E709A091E809B091E909A1
:10B9400039E1B695A795979587953A95D1F780FDFA
:10B9500002C00C94F15282E00E940D940C94F152BA
:10B9600060E08AEC93E10E94E2C280E00E940D94C4
:10B9700081E00E940D9482E00E940D940E94D19378
:10B980000C94F1528091151784FF2DC082EE93E143
:10B990000E94C72960E08CE40E947120182F8091DA
:10B9A000151784FF1AC085E397E10E94D77E8BE1CB
:10B9B000E5E3F7E1DE01119601900D928A95E1F73A
:10B9C00030E020E0412F70E060E0CE0101960E945F
:10B9D00043A3CE0101960E94AE2283ED93E10E9423
:10B9E000C7290C94F1520E944A2E83EF93E10E94E2
:10B9F000C7290C94F1520E946D7E0C94F152E09193
:10BA0000EA09F091EB098191882331F08032D9F76E
:10BA1000DF0111971C92F7CF60E08091EA099091C5
:10BA2000EB090E949DA41092330A1092320A0C94E2
:10BA3000F15283E50E942420882321F00E94E51E14
:10BA40000E9470D284E50E9424208823A9F00E94DD
:10BA5000E51E6B017C010E943CBEC092420AD0925E
:10BA6000430AE092440AF092450ACD28CE28CF2816
:10BA700019F081E080936214809113098823F9F012
:10BA800080E090E0A0EAB1E489839A83AB83BC8331
:10BA90001C8E1D8E1E8E1F8E18A219A21AA21BA20A
:10BAA00010E000E020E0AE014F5F5F4FBE01645E3A
:10BAB0007F4FCE0180960E9449AA0C94F1520E94B9
:10BAC0000827882381F00E944D760E942E278CE95A
:10BAD00098E00E94F57D1092451010924610109249
:10BAE00047101092481061E086E190E30E94B12B6C
:10BAF00040E059E26DEF73E185E00E94D3EB0E94D4
:10BB00002CEC0C94F1528091151784FD02C00C941A
:10BB1000F15283E50E942420882311F40C94F15201
:10BB20000E94E51E0E9470D20C94F1528091E609A9
:10BB30009091E709A091E809B091E90922E0B69552
:10BB4000A795979587952A95D1F780FF2CC083E11B
:10BB500094E10E94C72980917C188823F9F0BE01E6
:10BB60006F5F7F4F89E798E10E94887DCE01019643
:10BB70000E94E875CE0101960E941D7F809171148C
:10BB8000882339F080E20E94B62981E794E10E947F
:10BB9000E8758AE00E94B6290C94F15289E094E19C
:10BBA0000E94C729F6CF83E50E942420882301F153
:10BBB0000E94F51E182F8C3308F08CE38093250724
:10BBC0000E949B726B017C01212F30E0A8EEB3E054
:10BBD0000F943534C60ED71EE81EF91EC0922107F9
:10BBE000D0922207E0922307F09224070C94F1529E
:10BBF0000E941A760C94F152809115178E7F8093D3
:10BC000015170C94F1528091151784FD02C00C9405
:10BC1000F1520F94DE038091EA099091EB090E94A2
:10BC2000D3A20C94F1528091151782FF03C087FFB5
:10BC30000E94F3AE8091151784FD02C00C94F1525E
:10BC400060E080E50E947120182F682F8091EA093A
:10BC50009091EB090E949DA483E50E9424208823F3
:10BC600021F00E94E51E0E9470D20E944D761111B3
:10BC70000C94F1520E942E270C94F1520E94B0E8CD
:10BC80000C94F1520E944A4F0C94F15280E50E94AC
:10BC900024208823A1F00E94AC1F20E030E048EC73
:10BCA00052E40F940B2E0F94E035603127E27207B7
:10BCB00010F060E177E27093330A6093320A82E514
:10BCC0000E942420882311F40C94F1520E94D51E66
:10BCD0000C94F1520E94A3C20C94F15281E00E9494
:10BCE000B2C80C94F1528DE894E10E94C72960918A
:10BCF000FE077091FF0784E894E10E9411C06091F3
:10BD000000087091010887E794E10E9411C06091DA
:10BD1000FE077091FF078091000890910108681B51
:10BD2000790B80916214815021E030E0823010F074
:10BD300030E020E0621B730B8CE694E10E9430C07F
:10BD400084E694E10E94C72980910208909103083B
:10BD5000A0910408B09105088C8F9D8FAE8FBF8F86
:10BD6000BE016F5F7F4FCE014C960E9491D1BE0104
:10BD70006F5F7F4F87E594E10E94AFD880910608FE
:10BD800090910708A0910808B09109088C8F9D8FA9
:10BD9000AE8FBF8FBE016F5F7F4FCE014C960E946A
:10BDA00091D1BE016F5F7F4F87E494E10E94AFD8CD
:10BDB00020E030E04AE754E460910A0870910B08F3
:10BDC00080910C0890910D080F946735AB01BC0170
:10BDD0008FE294E10E94F5298DE60E94B6298AE05F
:10BDE0000E94B6290C94F15280E00E94F3D00C948A
:10BDF000F1520E944E2E182F87FD0AC085E994E16A
:10BE00000E94C729812F0E9438838AE00E94B629A8
:10BE10002D96CFAC2D97C0923E09C559DF4F0FB676
:10BE2000F894DEBF0FBECDBFDF91CF911F910F9170
:10BE3000FF90EF90DF90CF90BF90AF909F908F904A
:10BE40007F906F905F904F903F902F90089560E0AB
:10BE500080E50E94652081110C94F1521092B50A80
:10BE60000C94F1528EE40E942420882311F40C9447
:10BE7000F1520E94E51E6093DE0F7093DF0F8093F6
:10BE8000E00F9093E10F0C94F15283E50E9424207F
:10BE9000882321F00E94F51E8093100E0E944A2EE6
:10BEA00086EA94E10E94C7298091100E882331F11F
:10BEB00010E000E020E08091100E90E0002E02C023
:10BEC000959587950A94E2F780FF12C0FF24F394BA
:10BED000F20E222319F08CE20E94B629F801EE0F2F
:10BEE000FF1FE456FB4E859194910E94C7292F2D88
:10BEF0000F5F1F4F05301105F1F64BCE88E994E135
:10BF00004FCE83E50E942420882369F00E94F51E0D
:10BF10008D3320F4809306020C94F1528CE38093CD
:10BF200006020C94F1520E944A2E609106028DEA9C
:10BF300094E10E940CD70C94F15280E00E9413CF40
:10BF40000C94F15283E50E942420882311F40C9470
:10BF5000F1520E94F51E182F8C3308F08CE3809369
:10BF60002A070E949B726B017C01212F30E0A8EE12
:10BF7000B3E00F943534C60ED71EE81EF91EC092EA
:10BF80002607D0922707E0922807F09229070C9401
:10BF9000F1520E9404AF1092B50A0E94B18681E06E
:10BFA0000E94B2C868EE73E080E090E00E94A6268E
:10BFB00060E084EB94E10E94E2C20E94791E0C943E
:10BFC000F15280912F078F7D806180932F070C9411
:10BFD000F1520E94231E8823D9F10E94F3AE85E41A
:10BFE0000E94D61F81110E94C9938091E609909109
:10BFF000E709A091E809B091E90917E1B695A7957D
:10C00000979587951A95D1F780FF03C080E00E942D
:10C01000D8938091E90980FF03C081E00E94D89302
:10C020008091E6099091E709A091E809B091E909AA
:10C03000F9E1B695A79597958795FA95D1F780FD83
:10C0400002C00C94F15282E00E94D8930C94F152F9
:10C050000E9404AF0C94F15283E50E94D61F8823FE
:10C0600011F40C94F1520E949B7260935C147093D3
:10C070005D1480935E1490935F140E94AC1F20E0C7
:10C0800030E04AE754E40F940B2E0F94E0356093B0
:10C090002B0770932C0780932D0790932E070C94F9
:10C0A000F1520E94AC1F4B015C0120E030E040EAFD
:10C0B00051E40F94A52D87FF4EC0A5019401609116
:10C0C000470E7091480E8091490E90914A0E0F9440
:10C0D00067352B013C01AC019B016091210E7091F1
:10C0E000220E8091230E9091240E0F940B2E6093BC
:10C0F000210E7093220E8093230E9093240EA301A1
:10C1000092016091570E7091580E8091590E909146
:10C110005A0E0F940B2E6093570E7093580E809307
:10C12000590E90935A0E6091AD0A7091AE0A8091AB
:10C13000AF0A9091B00A0F94AA2DA30192010F9417
:10C140000B2E0F94E0356093AD0A7093AE0A809386
:10C15000AF0A9093B00A8092470E9092480EA09238
:10C16000490EB0924A0ED9C881E00F94B1030C94E5
:10C17000F1520E9446F287E495E10E942C930C94C0
:10C18000F1528091EA099091EB09009749F0DC01A6
:10C190002C91222329F061E00E9422D80C94F152C4
:10C1A0000E942CEC0C94F1520091EA091091EB09D9
:10C1B00094E0F12C40E09150F9F0F8018081282FB3
:10C1C0002B7F213499F421812133B1F4813411F191
:10C1D000853409F441E098012E5F3F4F89012F5FBC
:10C1E0003F4FF80180818032C9F3E5CF803521F4DB
:10C1F000818180538A3078F341110E944A2EFF20BA
:10C2000021F086EC94E10E94C729C8010E9401D860
:10C210000C94F152FF24F394DECF20930F08209367
:10C220000E080E94E4BB0C94F15210920F08109279
:10C230000E080E94E4BB0C94F1528091E60983FD44
:10C2400009C08091E8098C7029F481E00E94942F44
:10C250000C94F1520E944E2E182F87FF02C00C94AE
:10C26000F15200913E0784E40E942420F82E882396
:10C27000B1F00E94AC1F4B015C0120E030E0A9014D
:10C280000F94A52D8823A9F024E01202F0011124B7
:10C29000E65CF84F80829182A282B3820F2D602FDC
:10C2A00083E50E94712080933E070E944CAF0C945E
:10C2B000F15280E0F8CF8091E60984FD0DC08091B5
:10C2C000E809887849F48091E909837029F481E0CC
:10C2D0000E94DB2A0C94F1520E944E2E87FF02C06E
:10C2E0000C94F1520BE812E057E2E52E5EE0F52ED9
:10C2F0006FE8C62E62E0D62ED8018D918D010E9486
:10C300002420882359F00E94AC1F0F94E035F701D8
:10C3100060837183828393830E9481AEF4E0EF0E89
:10C32000F11CC016D10641F70C94F1520E944E2E1A
:10C3300087FF02C00C94F1524BE8E42E42E0F42E49
:10C3400010E000E0D7018D917D010E942420882318
:10C3500049F00E94AC1FF801E95DF14F64A375A399
:10C3600086A397A30C5F1F4F0031110559F70C945A
:10C37000F1528091E70987FD09C08091E8098E702C
:10C3800029F481E00E948F2A0C94F15283E50E94E7
:10C390002420882391F00E94AC1F60935B0E709361
:10C3A0005C0E80935D0E90935E0E6093630E7093AF
:10C3B000640E8093650E9093660E80E50E942420A3
:10C3C000882351F00E94AC1F60935B0E70935C0E4B
:10C3D00080935D0E90935E0E82E50E942420882358
:10C3E00051F00E94AC1F60935F0E7093600E8093BB
:10C3F000610E9093620E84E50E942420882311F43C
:10C400000C94F1520E94AC1F6093630E7093640E03
:10C410008093650E9093660E0C94F1520E94152B3A
:10C420000C94F15288E50E94D61F882369F00E947F
:10C43000AC1F6093110870931208809313089093B7
:10C44000140880E00E9407B489E50E94D61F882363
:10C4500069F00E94AC1F60931508709316088093D2
:10C4600017089093180881E00E9407B48AE50E949B
:10C47000D61F882311F40C94AD570E94AC1F609313
:10C48000150870931608809317089093180881E098
:10C490000E9407B40C94AD570E94D72C0C94F15213
:10C4A00082E40E94D61F882341F080914F02909130
:10C4B000500290930C0280930B0282E50E94D61FDB
:10C4C000882341F080910B0290910C0290935002CE
:10C4D00080934F0283E50E942420882331F00E943C
:10C4E000A81F9093500280934F028091E60990918B
:10C4F000E709A091E809B091E909892B8A2B8B2BD8
:10C5000011F00C94F15260914F027091500289EC3D
:10C5100094E10E94923185E20E94B6298AE00E944D
:10C52000B6290C94F1520E944A2E85E40E94B62945
:10C5300080E3800F0E94B629F701EB5AFD4F60811E
:10C5400071818DEC94E10E94923185E20E94B629BE
:10C550008AE00E94B6290C94F15280E50E94D61F11
:10C56000882311F40C94F15270E060E080E50E94A1
:10C570004820F82E6FEF7FEF83E50E9448208C0162
:10C580000196039710F00C94F152F7FE02C00C9440
:10C59000F1528F2D0E946B1E882341F00E94DD2DE9
:10C5A00085ED94E10E94C7290C94F1520E94F3AEEC
:10C5B00060E08F2D0E940F720F3F100789F001304D
:10C5C0001105C9F010E000E08F2D0E9475718017F1
:10C5D000910711F40C94F15280E00E945037F4CF8F
:10C5E0008F2D0E94757131E020E0892B09F030E039
:10C5F000032F122FE9CF01E010E0E6CF0E94BDD556
:10C600000C94F1528091E60983FD09C08091E709FD
:10C61000817829F481E00E94512F0C94F15280E539
:10C620000E942420882351F00E94AC1F6093401484
:10C6300070934114809342149093431489E40E94B0
:10C640002420882381F00E94AC1F2CEA35EC47E2BD
:10C650005EE30F940B2E6093441470934514809303
:10C6600046149093471484E40E942420882311F4F4
:10C670000C94F1520E94AC1F2CEA35EC47E25EE3C9
:10C680000F946735609348147093491480934A144B
:10C6900090934B140C94F1528091E60983FD09C0EC
:10C6A0008091E709817829F481E00E940B2A0C949B
:10C6B000F15280E50E94D61F882351F00E94AC1FE2
:10C6C0006093291470932A1480932B1490932C1444
:10C6D00089E40E94D61F882381F00E94AC1F2CEAB7
:10C6E00035EC47E25EE30F940B2E60932D147093AC
:10C6F0002E1480932F149093301484E40E94D61F3C
:10C70000882311F40C94F1520E94AC1F2CEA35ECF2
:10C7100047E25EE30F9467356093311470933214EF
:10C7200080933314909334140C94F15283E50E9457
:10C73000D61F182F882369F00E94A81F9C01909390
:10C7400034028093330291E0232B09F090E0909320
:10C75000410A80E50E94D61F882361F020913302B0
:10C7600030913402232B11F00E94091F8093410A5B
:10C770000C94F15211110C94F1520E944A2E80E057
:10C7800095E10E94C7298091410A882391F088EEA3
:10C7900094E10E94C72960913302709134028FEEB8
:10C7A00094E10E9492318BEE94E10E94C7290C948F
:10C7B000F15284EE94E1EDCF04EB10E083E40E94AB
:10C7C000242095E0E92E882319F00E94A81FE82E66
:10C7D00083E50E942420882319F00E94A81F8C0161
:10C7E00060E085E50E947120D82E60E083E195E14C
:10C7F0000E94E2C22D2D4E2D6F2DC8010E94D58DB5
:10C800000E942CEC0C94F15206E410E0D7CF0E9469
:10C81000F3AE0C94F1520E941F1F0E94B51E0E949D
:10C8200029BA0C94F1520E94BF2F0C94F152F39448
:10C830000C949C5B0E94B6250C94F1520E94DD2D55
:10C8400084E695E10E94C7290C94F15287E00E948A
:10C850005AD881110C94F1526DE2C62E61E3D62EA6
:10C86000E0E4FFE0F9A7E8A79E012F5F3F4F190121
:10C87000790110E000E0C6010E94191FA8A5B9A522
:10C880008D909D90AD90BD90B9A7A8A7A5019401EA
:10C890000F946C342B013C01F7014082518262827B
:10C8A000738220E030E040EA51EC0F94CD3687FDF2
:10C8B0000AC020E030E040EA51E4C301B2010F9425
:10C8C000A52D181684F4F801EC53F74DE4911E16CB
:10C8D00054F4B7FAB094B7F8B094D7018D929D9202
:10C8E000AD92BC921397F70181909190A190B19075
:10C8F0007F0120E030E040EA51ECC501B4010F9423
:10C90000CD3687FD45C020E030E040EA51E4C50166
:10C91000B4010F94A52D1816DCF10F5F1F4FF4E042
:10C92000CF0ED11C0330110509F0A5CF51E1E52E42
:10C9300058E0F52E10E0F10181919191A191B19112
:10C940001F01F70181939193A193B1937F01812FEF
:10C950000E9407B41F5F133071F70E9429BA60E08C
:10C960008DE795E10E94E2C263E972E084E690E01F
:10C970000E942DC270E060E08AE090E00E942DC22B
:10C980006AEB72E084E690E00E942DC20C94F152B2
:10C990000E94DD2D8BE995E10E94C72961E08DE8B9
:10C9A00095E10E94E2C268E270E080E991E00E94B5
:10C9B0002DC20C94F1520E9424C30C94F1520E9497
:10C9C0009B9F0C94F15261E083E50E94712091E0FD
:10C9D00089270E94EE9E0C94F1521091151712FFB8
:10C9E0000AC017FD08C00E94082780FB17F91093A2
:10C9F00015170C94F15214FD02C00C94F1520F94CF
:10CA0000DE030C94F1528091E70983FD09C0809107
:10CA1000E809887129F481E00E940F350C94F152E5
:10CA20000E944E2E082F87FF02C00C94F15285E51C
:10CA30000E94D61F882359F10E94AC1F4B015C0154
:10CA4000E02E002E000CFF0820E030E0A9010F943A
:10CA5000CD3687FF04C0B7FAB094B7F8B09420E0A1
:10CA600030E84BE354E4C501B4010F94CD3697018F
:10CA700043E0220F331F4A95E1F72E5C384F18161A
:10CA8000D4F1D9018D929D92AD92BC9213978CE412
:10CA90000E94D61F882311F40C94F1520E94AC1FFF
:10CAA0006B017C01002E000C110B20E030E0A9018D
:10CAB0000F94CD3687FF04C0F7FAF094F7F8F0949E
:10CAC00020E030E84BE354E4C701B6010F94CD36C3
:10CAD000980193E0220F331F9A95E1F72E5C384FAF
:10CAE00018169CF0D9011496CD92DD92ED92FC922D
:10CAF00017970C94F15280E090E8ABE3B4E4F901AD
:10CB000080839183A283B383C2CF80E090E8ABE3BC
:10CB1000B4E4F90184839583A683B7830C94F1521E
:10CB20000E948E440C94F1520E9412D30C94F15244
:10CB300083E080935D0810921D1460E083E50E94FD
:10CB4000712081110C94F1520E9407F20C94F15261
:10CB500083E50E94D61F882341F00E94091F80931D
:10CB6000250E0E9486220C94F15281E00E94BF2C77
:10CB70000C94F1520E9411320C94F1521091E3097D
:10CB80000E949B7260935C1470935D1480935E149A
:10CB900090935F14112311F40C94F1520E944A2EC9
:10CBA00084E50E94B629812F0E94908280E20E9433
:10CBB000B62984EC95E10E94C7290C94F152111119
:10CBC0000C94065511E00C9400550E94DD2D84E470
:10CBD00095E10E94C7290C94F152882399F30C9493
:10CBE0000B5520E030E0A901C701B6010F94A52D37
:10CBF000882311F40C94445218A619A61AA61BA651
:10CC0000A701960150582CA73DA74EA75FA788A55E
:10CC100099A5AAA5BBA5B05888AB99ABAAABBBABED
:10CC2000A7019601C701B6010F940B2E4B015C01C1
:10CC300028A539A54AA55BA5CA01B9010F940B2EF9
:10CC40009B01AC01C501B4010F946D340F941B37E7
:10CC500024966CAF7DAF8EAF9FAF24978090400F2E
:10CC60009090410FA090420FB090430FA701960102
:10CC7000C501B4010F946D3461966CAF7DAF8EAF7A
:10CC80009FAF6197C090440FD090450FE090460F42
:10CC9000F090470FCCAEDDAEEEAEFFAE28A539A5C5
:10CCA0004AA55BA5C701B6010F946D3465966CAFBC
:10CCB0007DAF8EAF9FAF65974090140950901509D6
:10CCC000609016097090170961962CAD3DAD4EAD80
:10CCD0005FAD6197C301B2010F946C346CAB7DAB57
:10CCE0008EAB9FABC0901809D0901909E0901A093B
:10CCF000F0901B0965962CAD3DAD4EAD5FAD6597CF
:10CD0000C701B6010F946C3468AF79AF8AAF9BAF9F
:10CD1000A3019201C501B4010F946C344B015C0175
:10CD20002DEB37E346E855EB0F94CD3687FF02C075
:10CD30000C941E532DEB37E346E855E3C501B401CF
:10CD40000F94A52D181614F40C941E53A7019601E8
:10CD50006CAD7DAD8EAD9FAD0F946C346B017C01DD
:10CD60002DEB37E346E855EB0F94CD3687FF02C035
:10CD70000C941E532DEB37E346E855E3C701B6018B
:10CD80000F94A52D181614F40C941E53023011059F
:10CD900011F00C94B25308E410E0EBED8E2EEFE0AE
:10CDA0009E2EE9ECAE2EE0E4BE2EFBEDCF2EFFE092
:10CDB000DF2EF9ECEF2EF0ECFF2E2091480F309192
:10CDC000490F40914A0F50914B0F69962CAF3DAFE0
:10CDD0004EAF5FAF699760911C0970911D098091FA
:10CDE0001E0990911F090F946C3428966CAF7DAF8B
:10CDF0008EAF9FAF289780914C0F90914D0FA091CF
:10CE00004E0FB0914F0F6D968CAF9DAFAEAFBFAFD1
:10CE10006D979C01AD01609120097091210980916D
:10CE20002209909123090F946C342C966CAF7DAF3E
:10CE30008EAF9FAF2C97A501940124966CAD7DAD6C
:10CE40008EAD9FAD24970F940B2E1B012C0127E173
:10CE500037EB41ED58E30F94A52D87FF10C027E174
:10CE600037EB41ED58E328966CAD7DAD8EAD9FADAF
:10CE700028970F94A52D87FF02C00C943A542AE0FE
:10CE800037ED43E25CE360912F02709130028091B4
:10CE90003102909132020F940B2E4B015C01609194
:10CEA0004F0270915002072E000C880B990B0F94C3
:10CEB000AC2D9B01AC01C501B4010F940B2E6C8FFE
:10CEC0007D8F8E8F9F8FC201B1010F940F363B0172
:10CED0004C01B80190E080E00F94AA2D5B018C0119
:10CEE0009B01AC01B301C4010F94CD36181614F4A4
:10CEF000530184019501A801C201B1010F94673566
:10CF00004B015C012DEC3CEC4CEC5DE30F94A52D4A
:10CF100087FF02C00C94C05320E030E040E85FE39C
:10CF2000C501B4010F94CD36181634F4812C912C20
:10CF300060E8A62E6FE3B62EA5019401C201B101EF
:10CF40000F9467350F940F360F94E03524966CAF2D
:10CF50007DAF8EAF9FAF24972296AEADBFAD229727
:10CF60006F96BFAFAEAF6F97BD0190E080E00F94BA
:10CF7000AA2D6CAB7DAB8EAB9FAB9B01AC01C50109
:10CF8000B4010F940B2E68AF79AF8AAF9BAF27E146
:10CF900037EB41ED58E3C201B1010F946C34A39615
:10CFA0006CAF7DAF8EAF9FAFA3979B01AC0168AD17
:10CFB00079AD8AAD9BAD0F94A52D812C912C40E8C5
:10CFC000A42E4FE3B42E87FF0AC0A201910168ADE1
:10CFD00079AD8AAD9BAD0F9467354B015C01A5011E
:10CFE0009401C701B6010F940B2E2CA93DA94EA99F
:10CFF0005FA90F9467356CAF7DAF8EAF9FAF9B017C
:10D00000AC010F940B2E6B017C01AC019B016CAD4C
:10D010007DAD8EAD9FAD0F940B2E20E030E040EC47
:10D0200050E40F9467359B01AC016CAD7DAD8EADC6
:10D030009FAD0F946C34A7966CAF7DAF8EAF9FAF52
:10D04000A79720E030E040E05FE3C701B6010F940E
:10D050000B2E9B01AC0160E070E080E89FE30F9431
:10D060006C34AB966CAF7DAF8EAF9FAFAB97A50125
:10D07000940128966CAD7DAD8EAD9FAD28970F9431
:10D080000B2E2CA93DA94EA95FA90F9467352896B0
:10D090006CAF7DAF8EAF9FAF2897A50194012C9602
:10D0A0006CAD7DAD8EAD9FAD2C970F940B2E2CA942
:10D0B0003DA94EA95FA90F9467352C966CAF7DAF43
:10D0C0008EAF9FAF2C97A3962CAD3DAD4EAD5FAD0F
:10D0D000A39768AD79AD8AAD9BAD0F94A52D87FF61
:10D0E0000AC022962EAD3FAD22972F5F3F4F6F961D
:10D0F0003FAF2EAF6F976996CCACDDACEEACFFAC1A
:10D100006997C986DA86EB86FC866D96CCACDDAC79
:10D11000EEACFFAC6D97CD86DE86EF86F88A0E9476
:10D120009B729B01AC0128533F4F4F4F5F4F28AF7D
:10D1300039AF4AAF5BAF4CA45DA46EA47FA4222498
:10D140002394312C39E13CAB6F96CEACDFAC6F97BA
:10D150002C143D0410F00C941A540E9454890E941F
:10D160009B728B019C01C8ACD9ACEAACFBAC0C192E
:10D170001D092E093F0937FD0DC09B01AC01285345
:10D180003F4F4F4F5F4F28AF39AF4AAF5BAF80E0A3
:10D190000E9450373CA931503CAB332311F40C941E
:10D1A000C9539201A301A7966CAD7DAD8EAD9FAD25
:10D1B000A7970F940B2E6B017C0128A939A94AA9C6
:10D1C0005BA9AB966CAD7DAD8EAD9FADAB970F946B
:10D1D0000B2E9B01AC01C701B6010F946D347B018E
:10D1E0008C019201A301AB966CAD7DAD8EAD9FAD70
:10D1F000AB970F940B2E4B015C0128A939A94AA9C2
:10D200005BA9A7966CAD7DAD8EAD9FADA7970F9432
:10D210000B2E9B01AC01C501B4010F946C342B01A2
:10D220003C01C701D80188AB99ABAAABBBAB92015B
:10D23000A30161966CAD7DAD8EAD9FAD61970F94EE
:10D240006D3469837A838B839C8328A939A94AA981
:10D250005BA965966CAD7DAD8EAD9FAD65970F9466
:10D260006D346D837E838F83988728962CAD3DAD7A
:10D270004EAD5FAD289769857A858B859C850F9427
:10D280006D3469877A878B879C872C962CAD3DAD52
:10D290004EAD5FAD2C976D857E858F8598890F94F7
:10D2A0006D346D877E878F87988BCE0101960E94A3
:10D2B00041B420E030E0A901BE01645E7F4FCE01A1
:10D2C00001960F948201882311F40C941A545FEF95
:10D2D000251A350A39CF8150823108F05AC0E82F1B
:10D2E000F0E08827E958F6498F4F0D946434976928
:10D2F0009B6989698F699369C9699E69A469A869ED
:10D30000AE69B269B669BC69C069C969C469CA69EC
:10D31000CE69809180008F778093800008958091FE
:10D3200080008F7DF9CF80918000877FF5CF84B515
:10D330008F7784BD089584B58F7DFBCF8091B00039
:10D340008F778093B00008958091B0008F7DF9CFE2
:10D35000809190008F778093900008958091900045
:10D360008F7DF9CF80919000877FF5CF8091A000CD
:10D370008F778093A00008958091A0008F7DF9CFD2
:10D380008091A000877FF5CF809120018F778093D7
:10D3900020010895809120018F7DF9CF8091200197
:10D3A000877FF5CF3FB7F8948091C4099091C50964
:10D3B000A091C609B091C70926B5A89B05C02F3F0B
:10D3C00019F00196A11DB11D3FBFBA2FA92F982FAB
:10D3D0008827BC01CD01620F711D811D911D42E0A6
:10D3E000660F771F881F991F4A95D1F708958BE123
:10D3F000E5E3F7E1A0E5B7E101900D928A95E1F749
:10D400008091151780648093151710920A1708955C
:10D41000CF938091D813C1E08823C9F08091D913AC
:10D420009091DA134091D0135091D1136091D2139F
:10D430007091D313DC01ED91FC910288F389E02D0A
:10D4400020ED31E11995C82F811104C0C0E08C2F67
:10D45000CF9108954091D4135091D5136091D61374
:10D460007091D7134115510561057105B9F080918F
:10D47000D9139091DA13DC01ED91FC910288F389C4
:10D48000E02D20ED31E11995882301F31092D4139A
:10D490001092D5131092D6131092D7131092D8135E
:10D4A000D6CF0F931F93CF93DF93CDB7DEB760979F
:10D4B0000FB6F894DEBF0FBECDBF8C01DC01ED913D
:10D4C000FC910280F381E02DBE016F5F7F4F1995C3
:10D4D000882309F464C08981807CC9F56F816370F9
:10D4E00070E0762F6627770F770F8885B4E08B9FE3
:10D4F000C0011124682B792B8985829586958695A4
:10D500008370682B6F5F7F4F90E080E02A852370E7
:10D51000220F3B8537FB332730F9232B3E813F70A9
:10D52000230F3327331F2750310904C0660F771F9D
:10D53000881F991F2A95D2F760960FB6F894DEBF20
:10D540000FBECDBFDF91CF911F910F910895803411
:10D5500019F568856695669570E090E080E0CB01EE
:10D56000772766272A85622B098510E0102F002770
:10D57000012E000C220B330B602B712B822B932B73
:10D580006F5F7F4F8F4F9F4F4AE0660F771F881F57
:10D59000991F4A95D1F7D0CF8BE0F801848360E0E2
:10D5A00070E0CB01C9CF0895FC0182810895CF932B
:10D5B000DF93C0913D14D0913E1481E0CE31D1056E
:10D5C000E4F020E030E040E05FE3609139147091D6
:10D5D0003A1480913B1490913C140F946D340F9445
:10D5E000D9356C1B7D0B77FF03C07195619571096F
:10D5F00081E0633071050CF080E0DF91CF910895F8
:10D600008F929F92AF92BF92CF92DF92EF92FF9252
:10D610000F931F93CF93DF93B0E2A0E06A2F70E0E7
:10D62000AB014B0F511D55954795411119C0EAE8C3
:10D63000F3E265917491072E000C880B990B0F94FF
:10D64000AC2DDF91CF911F910F91FF90EF90DF9064
:10D65000CF90BF90AF909F908F900895B42FE0CF60
:10D66000A41711F0B41303C0E6E0F4E2E2CF9A018C
:10D6700021503109220F331F220F331FF901E857C0
:10D68000FC4DE590F490F901E457FC4DC591D4911F
:10D690008E159F0518F3A42FC817D90708F4BECF1D
:10D6A000F901E657FC4D05911491F901E257FC4D43
:10D6B000C590D4908E199F09BC0190E080E00F9432
:10D6C000AA2D4B015C01B601601B710B072E000CEB
:10D6D000880B990B0F94AC2D9B01AC01C501B401D3
:10D6E0000F940B2E4B015C01CE19DF09BE0190E0B7
:10D6F00080E00F94AA2D9B01AC01C501B4010F94E9
:10D7000067356B017C01B801110F880B990B0F94E1
:10D71000AC2D9B01AC01C701B6010F946D3491CFC4
:10D72000EF92FF920F931F93E0924707F092480702
:10D730000093490710934A07609355077093560763
:10D74000809357079FEFFF27621B730B840B30F406
:10D75000809570956195790B890B99279093340684
:10D76000A6E06A9F00922806512DEE277A9F500D61
:10D77000E11D8A9FE00D50932906E0932A06AFE051
:10D780006A9F00922C06512DEE277A9F500DE11DC5
:10D790008A9FE00D50932D06E0932E06AAE06A9F23
:10D7A00000923006512DEE277A9F500DE11D8A9F81
:10D7B000E00D50933106E09332061F910F91FF90D8
:10D7C000EF90089500008091100880FF23C0899891
:10D7D0008FEF809340098091100881FF1EC08F9ABF
:10D7E0008FEF809341098091100882FF19C08091CA
:10D7F0000B0180958270809309018FEF809342091D
:10D800008091100883FF13C016988FEF809343090F
:10D8100000000895899A81E0DCCF8F9881E0E1CF04
:10D8200080910B0182708093090181E0E7CF169A05
:10D8300081E0ECCF0F930091430721E0022724E41D
:10D8400037E04CE050E0BC0180E397E00E94F52710
:10D850000F9108950F930091430721E0022724E4DC
:10D8600037E041E050E0BC0180E397E00E94F527FB
:10D870000F9108950F930091430721E0022724E4BC
:10D8800037E041E050E0BC0180E397E00E94F527DB
:10D890000F9108950F930091430721E0022724E49C
:10D8A00037E048E050E0BC0180E397E00E94F527B4
:10D8B0000F9108950F930091430721E0022724E47C
:10D8C00037E04CE050E0BC0180E397E00E94F52790
:10D8D0000F9108950F930091430721E0022724E45C
:10D8E00037E044E050E0BC0180E397E00E94F52778
:10D8F0000F9108950F9301E024E437E041E050E0F8
:10D90000BC0180E397E00E94F5270F9108954F92A4
:10D910005F926F927F928F929F92AF92BF92CF92BF
:10D92000DF92EF920F931F93CF93DF9300D01F925C
:10D93000CDB7DEB74C015B016A01122F002309F459
:10D9400040C06E2D84E00E94DCEB0E944A2E89E6E6
:10D9500099E20E94C72961E0812F0E94EA2200918A
:10D960003E0983E080933E0981E08093730E8BE54E
:10D9700099E20E943CC80E94E22B82E080936314EB
:10D9800040E36BE479E28DE199E20E94E72B40E00D
:10D9900062E479E286E199E20E94E72B61E081E1AD
:10D9A00099E20E94C92B8091730E882341F060E0B8
:10D9B000812F0E94EA2281E00E945037F4CF009329
:10D9C0003E096E2D85E00E94DCEB20E030E0A901ED
:10D9D000F40160817181828193810F94A52D882348
:10D9E00071F080E090E0A0ECB0E489839A83AB838F
:10D9F000BC83BE016F5F7F4FC4010E946BB920E002
:10DA000030E0A901F50160817181828193810F94D9
:10DA1000A52D882351F140905F0E5090600E6090CC
:10DA2000610E7090620E80E090E0A0E7B1E4809318
:10DA30005F0E9093600EA093610EB093620E80E033
:10DA400090E0A0EAB1E489839A83AB83BC83BE01F2
:10DA50006F5F7F4FC5010E946BB940925F0E50927D
:10DA6000600E6092610E7092620E812C912C80E4A7
:10DA7000A82EBA2C03E020E030E0A901F601608175
:10DA80007181828193810F94CD36181674F460E011
:10DA900086E00E94DCEB89829A82AB82BC82BE0166
:10DAA0006F5F7F4FC6010E946BB98091700E22E4B8
:10DAB00039E2882311F023E239E241E359E26BE3D2
:10DAC00079E281E00E940A2C10913E0900933E0900
:10DAD0001092730E60E087E00E94DCEB8091720E82
:10DAE000811104C081E00E945037F8CF10933E09A5
:10DAF000813009F4C0CF0E94E22B81E00F900F909B
:10DB00000F900F90DF91CF911F910F91EF90DF90C9
:10DB1000CF90BF90AF909F908F907F906F905F90CD
:10DB20004F9008954F925F926F927F928F929F9243
:10DB3000AF92BF92CF92DF92EF92FF92CF93DF939B
:10DB400000D000D01F921F92CDB7DEB75C01DB0181
:10DB5000CD90DD90ED90FC90E0913015F091311575
:10DB6000FE83ED8384819581A681B78189839A8321
:10DB7000AB83BC839C01AD01C701B6010F946C342B
:10DB80002B013C01F50180809180A280B380AD81A2
:10DB9000BE818D919D910D90BC91A02D8D839E8312
:10DBA000AF83B88727E137EB41ED58EBC301B201F2
:10DBB0000F94CD3687FDD1C023E030E04BE953E42C
:10DBC000C301B2010F94A52D18160CF4C6C02D8107
:10DBD0003E814F815885C501B4010F946C342B01EF
:10DBE0003C0127E137EB41ED58EB0F94CD3687FD33
:10DBF000B4C023E030E84DE953E4C301B2010F940F
:10DC0000A52D18160CF4A9C020E030E0A9016D8103
:10DC10007E818F8198850F946D342B013C0120E02B
:10DC200030E040E251E40F94A52D87FF06C0412C5F
:10DC3000512C30E2632E31E4732E27E137EB41EDB6
:10DC400058E3C301B2010F946C349B01AC01C501D0
:10DC5000B4010F94CD3687FD80C020E030E84DE957
:10DC600053E46D817E818F8198850F946D342B01F3
:10DC70003C0120E030E041E953E40F94CD36181622
:10DC800034F4412C512C21E9622E23E4722E27E139
:10DC900037EB41ED58E3C301B2010F946D349B01A2
:10DCA000AC01C501B4010F94A52D18160CF455C094
:10DCB00020E030E0A90169817A818B819C810F94F9
:10DCC0006D344B015C0120E030E040EA51E40F94F8
:10DCD000A52D87FF06C0812C912C90EAA92E91E4F6
:10DCE000B92E27E137EB41ED58E3C501B4010F949C
:10DCF0006C349B01AC01C701B6010F94CD3687FD92
:10DD00002CC020E030E04BE953E469817A818B81BB
:10DD10009C810F946D344B015C0120E030E04CE8B5
:10DD200053E40F94CD36181634F4812C912C8CE8E2
:10DD3000A82E83E4B82E27E137EB41ED58E3C50167
:10DD4000B4010F946D349B01AC01B1E0B983C701FC
:10DD5000B6010F94A52D18160CF419828981289606
:10DD60000FB6F894DEBF0FBECDBFDF91CF91FF900D
:10DD7000EF90DF90CF90BF90AF909F908F907F906B
:10DD80006F905F904F9008952F923F924F925F92C5
:10DD90006F927F928F929F92AF92BF92CF92DF92BB
:10DDA000EF92FF920F931F93CF93DF93CDB7DEB720
:10DDB0006C970FB6F894DEBF0FBECDBF1C017B8FF2
:10DDC0006A8F498F2C8FFC01408051806280738064
:10DDD00049825A826B827C82FB01C080D180E280C2
:10DDE000F380CD82DE82EF82F8868090480F90909B
:10DDF000490FA0904A0FB0904B0F89869A86AB8648
:10DE0000BC86BE016B5F7F4FCE0101960E94926D72
:10DE1000882309F444C10091301510913115F8019F
:10DE20002081318142815381C301B2010F946C344E
:10DE30002B013C0149825A826B827C82F801248149
:10DE4000358146815781C701B6010F946C349B011F
:10DE5000AC012D833E834F8358878091230290919C
:10DE60002402A0912502B09126028D879E87AF875C
:10DE7000B88BCE010D966C0185017401C301B2010E
:10DE80000E941FB880915F08811103C081E00E9449
:10DE9000F3BB8091260E82FFE8C020912C153091B3
:10DEA0002D1540912E1550912F1560E070E080EAFD
:10DEB00090EC0F946C346D8B7E8B8F8B988F80E001
:10DEC00090E0A0E4B1E4898B9A8BAB8BBC8BBE0154
:10DED0006F5E7F4FCE0145960E94FCB810915E08A0
:10DEE00010925E0882E00E949BB90E9427BAC090FF
:10DEF000480FD090490FE0904A0FF0904B0F2091BF
:10DF00002C1530912D1540912E1550912F1560E054
:10DF100070E080EA90E40F946C349B01AC01C7017F
:10DF2000B6010F94CD3618160CF0C0C060E070E05A
:10DF300080EC9FE720912C1530912D1540912E15E6
:10DF400050912F150F946D346B017C01AC019B0136
:10DF50000F945F37811161C0898D8350823008F042
:10DF600089C06091480F7091490F80914A0F90913C
:10DF70004B0FE98D20E030E040EA50E4E43021F43A
:10DF800020E030E048EC51E40F946D346D8B7E8BD3
:10DF90008F8B988F63EC72E0CE0145960E94FCB89F
:10DFA000FC8DF33008F446C02091500F3091510F92
:10DFB0004091520F5091530FF10160817181828124
:10DFC00093810F946D34AB01BC0180EF98E20E9405
:10DFD000F5292091540F3091550F4091560F5091D3
:10DFE000570FEA8DFB8D60817181828193810F943F
:10DFF0006D34AB01BC018BEE98E20E94F529B701AC
:10E00000A60186EE98E20E94062AA7019601C701A2
:10E01000B6010F945F37882369F00E941F1F60E0EC
:10E0200087ED98E20E94E2C20E94DD2D87EC98E223
:10E030000E94C729C701B6016C960FB6F894DEBFDF
:10E040000FBECDBFDF91CF911F910F91FF90EF9049
:10E05000DF90CF90BF90AF909F908F907F906F9008
:10E060005F904F903F902F90089560E070E080E2C5
:10E0700091EC21CF898D8150823008F091CF0E94A0
:10E080001F1F882309F48CCFFC8DC12CD12C80EC70
:10E09000E82E8FE7F82EF33008F4BFCF85CFC12CE0
:10E0A000D12C90ECE92E9FE7F92EC4CF12FF3ECF82
:10E0B00020E030E040EA50E4C701B6010F946D342F
:10E0C0006D877E878F87988B63EC72E0CE010D960B
:10E0D0000E94FCB880E090E0A0ECB0E48D879E87C1
:10E0E000AF87B88BBE01635F7F4FCE0145960E941C
:10E0F000FCB810915E0810925E0882E00E949BB905
:10E100000E9427BA4090480F5090490F60904A0FE4
:10E1100070904B0F20912C1530912D1540912E159C
:10E1200050912F1560E070E080EA90E40F946C3419
:10E130009B01AC01C301B2010F94CD3618160CF44B
:10E14000F5CE12FFF3CE20E030E040E450E4C3010E
:10E15000B2010F940B2E2B013C01A7019601C701C0
:10E16000B6010F946D349B01AC01C301B2010F9451
:10E170006D342DEC3CEC4CE45EE30F940B2EDACEC8
:10E180004F925F926F927F928F929F92AF92BF92C7
:10E19000FF920F931F93CF93DF93CDB7DEB76897AE
:10E1A0000FB6F894DEBF0FBECDBFF82E4A015B015B
:10E1B0002801390120E030E0A901C301B8010F9422
:10E1C000A52D811111C0FF2019F081E0F81288C03F
:10E1D00060E070E88BE395E420E030E040E752E453
:10E1E0000F9467352B013C014D8A5E8A6F8A788EC9
:10E1F0000F2D10E0F801EC53F74DE4917724739460
:10E200001E160CF4712CFF24F39420E030E0A901D9
:10E21000C501B4010F94CD3618160CF0F12C80E036
:10E220000E9499B369837A838B839C8381E00E94E7
:10E2300099B36D837E838F83988782E00E9499B320
:10E2400069877A878B879C8783E00E9499B36D8763
:10E250007E878F87988B000F111F000F111FE1E041
:10E26000F0E0EC0FFD1F0E0F1F1FF801108211824E
:10E2700012821382CE0101960E94DCB2F8018082E4
:10E280009182A282B382198A1A8A1B8A1C8A80917F
:10E29000B60A9091B70A892B51F4AE014F5E5F4FD9
:10E2A000BE016B5E7F4FCE0101960E945FF30E941C
:10E2B000F3AE7F100E94FCBD68960FB6F894DEBFE7
:10E2C0000FBECDBFDF91CF911F910F91FF90BF90F7
:10E2D000AF909F908F907F906F905F904F90089538
:10E2E00060E070E086E194E477CFCF93DF93282F4E
:10E2F00030E0F901E258F74D8491F901E85CF74DFF
:10E30000D491F901EE50F84DC491CC23A1F08111C4
:10E310000E946B69EC2FF0E0EE0FFF1FE852F84D02
:10E32000A591B491EC91ED2381E090E009F480E0B7
:10E33000DF91CF91089580E090E0FACF1F93CF93C3
:10E34000DF93282F30E0F901E258F74D8491F9016D
:10E35000E85CF74DD491F901EE50F84DC491CC230F
:10E36000A9F0162F81110E946B69EC2FF0E0EE0FDF
:10E37000FF1FE254F84DA591B4918FB7F894EC913A
:10E38000111108C0D095DE23DC938FBFDF91CF91B0
:10E390001F910895DE2BF8CFCF93DF93EC018D8191
:10E3A0000E943F3760E08B81DF91CF910C949E718A
:10E3B00061E0FC0183810E949E718FEF0C943337E2
:10E3C000CF93DF93EC016EBDFA01CA019E5F0DB4DD
:10E3D00007FEFDCF20812EBD0DB407FEFDCF2181AC
:10E3E0002EBD3296E817F90791F70DB407FEFDCF61
:10E3F0008FEF0E9433378FEF0E9433370E943837F8
:10E400008E838F71853049F083E18C83CE010E9429
:10E41000D87180E0DF91CF91089581E0FBCFCF9359
:10E42000DF9390E0FC01E85CF74D24918E50984D0D
:10E43000FC0184918823C9F090E0880F991FFC01AA
:10E44000EC55F84DA591B491FC01E254F84DC591FD
:10E45000D49161110DC09FB7F8948C9120958223BF
:10E460008C938881282328839FBFDF91CF910895C3
:10E47000623051F49FB7F8943C91822F80958323AA
:10E480008C93E8812E2BEFCF8FB7F894EC912E2B45
:10E490002C938FBFEACF863308F0865320917B0000
:10E4A000982F9870277F922B90937B0087708064C1
:10E4B00080937C0080917A00806480937A008091C0
:10E4C0007A0086FDFCCF80917800909179000895C4
:10E4D0008F929F92AF92BF92CF92DF92EF92FF9274
:10E4E0006B017C010E94D2694B015C01C114D10413
:10E4F000E104F104B9F00E94D269681979098A0926
:10E500009B09683E73408105910580F321E0C21AA2
:10E51000D108E108F10888EE880E83E0981EA11C5E
:10E52000B11CE4CFFF90EF90DF90CF90BF90AF9001
:10E530009F908F9008952FB7F8946091C0097091C3
:10E54000C1098091C2099091C3092FBF0895CF924C
:10E55000DF92EF92FF920E949B726B017C0128E593
:10E56000C20E22E0D21EE11CF11C0E9438378F3F00
:10E5700071F00E949B726C197D098E099F0997FDAD
:10E58000F4CF80E0FF90EF90DF90CF90089581E08E
:10E59000F9CF0F931F93CF938C010E94CC710E94EF
:10E5A000A772C82F882371F08DEF0E9433370E9425
:10E5B000A772C82FC8010E94D8718C2FCF911F91CC
:10E5C0000F91089582E1F8018483F4CF0F931F9394
:10E5D000CF93DF93EC018B010E94CC710E94A77254
:10E5E00081110CC085E18C8310E0CE010E94D871AE
:10E5F000812FDF91CF911F910F910895A8016CEFAA
:10E60000CE010E94E071182F882361F3EECFDF92D4
:10E61000EF92FF920F931F93CF93DF938C01C62F3E
:10E62000D22FF32EE42ED52E0E94CC710E94A77219
:10E630008C2F80640E9433378D2D0E9433378E2DAE
:10E640000E9433378F2D0E9433378D2F0E9433372E
:10E6500087E8C11101C085E90E943337CC3011F43D
:10E660000E943837C0E00E943837F801868387FF60
:10E6700004C0CF3F11F0CF5FF6CFDF91CF911F9154
:10E680000F91FF90EF90DF9008958F929F92AF923D
:10E69000BF92CF92DF92EF92FF920F931F93CF938F
:10E6A000DF93EC016A017B01590120E030E0A90110
:10E6B00067E30E940773A501980167E1CE010E94FC
:10E6C0000773811127C08F81833039F089E0CC0C2A
:10E6D000DD1CEE1CFF1C8A95D1F7A701960169E1AC
:10E6E000CE010E94077311E0882319F010E087E043
:10E6F0008C83CE010E94D871812FDF91CF911F9121
:10E700000F91FF90EF90DF90CF90BF90AF909F90D0
:10E710008F90089589E08C8310E0EBCF0F931F93C7
:10E72000CF93DF93EC0189018F81833039F089E049
:10E73000440F551F661F771F8A95D1F79A01AB01C9
:10E7400068E1CE010E94077381112AC0A8016EEF13
:10E75000CE010E94E071182F8823B1F00E94A772A9
:10E76000182F8823D1F020E030E0A9016DE0CE0120
:10E770000E940773882321F086E18C8310E004C097
:10E780000E9438378111F8CFCE010E94D871812FB5
:10E79000DF91CF911F910F91089587E18C83F4CF82
:10E7A00086E0EBCF1F93CF93DF93EC010E94CC71F7
:10E7B00020E030E0A9016CE0CE010E94077311E077
:10E7C000882319F010E083E08C83CE010E94D87179
:10E7D000812FDF91CF911F9108951F93CF93DF93E6
:10E7E000EC018F81833039F089E0440F551F661F9B
:10E7F000771F8A95D1F79A01AB0162E1CE010E94A1
:10E80000077311E0882319F010E085E08C83CE01B6
:10E810000E94D871812FDF91CF911F9108958F921F
:10E820009F92AF92BF92EF92FF920F931F93CF935D
:10E83000DF938C01EB017A010E949B724B015C011A
:10E840002CE2820E21E0921EA11CB11C0E943837DE
:10E85000F80186838F3F69F40E949B7268197909D9
:10E860008A099B0997FDF2CF81E1F8018483C0E01A
:10E8700021C08E3F71F5F1E0EF1AF1088FEF8EBDE8
:10E88000FE012FEF0DB407FEFDCF8EB581932EBD97
:10E89000CF018C1B9D0B8E159F05A0F30DB407FEB9
:10E8A000FDCF8EB5CE0DDF1D88830E9438370E94C4
:10E8B0003837C1E0C8010E94D8718C2FDF91CF9109
:10E8C0001F910F91FF90EF90BF90AF909F908F900E
:10E8D00008958FE0CACF0F931F93CF93DF93EC017E
:10E8E0008B010E94CC7140E052E0B801CE01DF9173
:10E8F000CF911F910F910C940F740F931F93CF938F
:10E90000DF93EC0189018F81833039F089E0440F76
:10E91000551F661F771F8A95D1F79A01AB0161E1F8
:10E92000CE010E94077381110AC040E052E0B80195
:10E93000CE01DF91CF911F910F910C940F7484E061
:10E940008C83CE010E94D87180E0DF91CF911F911E
:10E950000F9108950F931F93CF93DF93EC018B01D9
:10E9600020E030E0A90169E00E94077381110AC02C
:10E9700040E150E0B801CE01DF91CF911F910F919E
:10E980000C940F7480E18C83CE010E94D87180E0DA
:10E99000DF91CF911F910F9108958F929F92AF9227
:10E9A000BF92CF92DF92EF92FF920F931F93CF937C
:10E9B000DF93EC01162F1F821C824B830E949B72F7
:10E9C0006B017C0120EDC20E27E0D21EE11CF11C80
:10E9D000A89561E08B810E949E7161E08B810E940D
:10E9E0000F72209A289A219A2398229A81E00E94F5
:10E9F0003F3785E08D830E943F370AE08FEF0E940A
:10EA000033370150D9F7A89520E030E0A90160E044
:10EA1000CE010E9407738E83813081F00E949B7229
:10EA20006C197D098E099F0997FDEECF81E08C83DB
:10EA3000CE010E94D8711A8280E06AC0A8952AEAA5
:10EA400031E040E050E068E0CE010E94077385307D
:10EA500041F581E08F83A8958F81812C912C540101
:10EA6000823029F4812C912CA12C80E4B82E20E056
:10EA700030E0A90167E3CE010E940773A50194016C
:10EA800069E2CE010E9407738E838823F1F00E9411
:10EA90009B726C197D098E099F0997FDE8CF8AE06A
:10EAA000C6CF04E00E9438378E830150D9F78A3AE6
:10EAB00011F482E0CFCF0E949B726C197D098E0900
:10EAC0009F0997FDBCCF82E0B2CF8F818230C1F425
:10EAD00020E030E0A9016AE3CE010E940773882399
:10EAE00011F088E0A4CF0E943837807C803C11F47C
:10EAF00083E08F830E9438370E9438370E9438376E
:10EB0000CE010E94D87181E08A83173070F41D8392
:10EB1000DF91CF911F910F91FF90EF90DF90CF90F9
:10EB2000BF90AF909F908F90089588E18C8384CFA1
:10EB30001F920F920FB60F9211242F933F938F9332
:10EB40009F93AF93BF938091C0099091C109A09109
:10EB5000C209B091C3093091BF0923E0230F2D37BB
:10EB600058F50196A11DB11D2093BF098093C009DE
:10EB70009093C109A093C209B093C3098091C409BD
:10EB80009091C509A091C609B091C7090196A11D30
:10EB9000B11D8093C4099093C509A093C609B09391
:10EBA000C709BF91AF919F918F913F912F910F9086
:10EBB0000FBE0F901F90189526E8230F0296A11DF7
:10EBC000B11DD2CF8DE00E94B6298AE00C94B629FF
:10EBD000CF93DF93EC018991882319F00E94B62925
:10EBE000FACFDF91CF91089580910A178823C1F061
:10EBF000815080930A17E5E3F7E1882351F08150B3
:10EC0000990B2BE1289FF001299FF00D1124E55964
:10EC1000F84E8BE1A0E5B7E101900D928A95E1F7FE
:10EC200080910A17811105C09091151790649093F7
:10EC300015170895CF92DF92EF92FF9280911517EA
:10EC400082FF23C0C0901117D0901217E0901317C5
:10EC5000F090141780EE95E20E94C729C701B60113
:10EC60000E94F0E98FE20E94B62960910D17709121
:10EC70000E1780910F17909110170E94F0E9FF90E6
:10EC8000EF90DF90CF900C94E27582EF95E2FF90C9
:10EC9000EF90DF90CF900C94C7298091151784FFD7
:10ECA00004C08460877F809315170895CF92DF9208
:10ECB000EF92FF920F931F93CF93DF93CDB7DEB701
:10ECC000EDB6FEB6DC010D900020E9F79D01281B92
:10ECD000390B285F3F4FEDB7FEB7E21BF30B0FB6C2
:10ECE000F894FEBF0FBEEDBF0DB71EB70F5F1F4FED
:10ECF0009F938F938AE095E29F938F931F930F9337
:10ED00000F943C2D6801F4E0CF0ED11C0F900F90B2
:10ED10000F900F900F900F90D6018D916D01882369
:10ED200049F0082E000C990B0F947F37F6013197AC
:10ED30008083F2CF65E075E2C8010F94D52C4FE3D4
:10ED400050E0B8018DE198E00F94DB370FB6F894EE
:10ED5000FEBE0FBEEDBEDF91CF911F910F91FF90D0
:10ED6000EF90DF90CF900895FC01938591FF02C052
:10ED700080E00895987121E0903109F020E08091C1
:10ED8000151720FB85F980931517903141F0808588
:10ED9000873471F781E091859E3751F3089581E0C2
:10EDA000FDCFFC0120E03EE2DB014D91BD01403290
:10EDB00049F0283011F430833196DB0111974C91E2
:10EDC000408331962F5F2B3079F710820895EF92B0
:10EDD000FF920F931F93CF93DF93CDB7DEB7A0972A
:10EDE0000FB6F894DEBF0FBECDBF7C018B01BE0114
:10EDF0006F5F7F4FC7010E9475EA1816A4F4CE0119
:10EE000001960E94B476882391F3BE016F5F7F4F15
:10EE100084E694E10E94D17664E674E1C8010F941F
:10EE20009D37892B21F7A0960FB6F894DEBF0FBE51
:10EE3000CDBFDF91CF911F910F91FF90EF9008957B
:10EE4000CF92DF92EF92FF92CF936B017C01C42FA0
:10EE50008091D0139091D113A091D213B091D3137C
:10EE60008C159D05AE05BF0529F10E94086A811128
:10EE700008C0C0E08C2FCF91FF90EF90DF90CF9033
:10EE800008958091D9139091DA13DC01ED91FC91F2
:10EE90000088F189E02D20ED31E1B701A601199537
:10EEA000882339F3C092D013D092D113E092D213B9
:10EEB000F092D313CC2321F081E08093D813DACFE2
:10EEC000C1E0D8CF4F925F926F927F928F929F92C4
:10EED000AF92BF92CF92DF92EF92FF920F931F9368
:10EEE000CF93DF93EC01423051056105710590F439
:10EEF00080E0DF91CF911F910F91FF90EF90DF9015
:10EF0000CF90BF90AF909F908F907F906F905F90C9
:10EF10004F90089589859A85AB85BC850196A11D82
:10EF2000B11D84179507A607B70710F38F898031A5
:10EF3000C9F5852E962EA72EBB248B899C89AD8979
:10EF4000BE89880E991EAA1EBB1E280139016A01BE
:10EF50007B0141E0C501B4010E942077882341F282
:10EF60009F89903181F5DD24EE24FF24F601EE0F18
:10EF7000FF1FE053FE4E118300839A89923008F4FC
:10EF8000B8CF4D815E816F817885840E951EA61E57
:10EF9000B71E8092D4139092D513A092D613B0923C
:10EFA000D713A7CF803209F0A3CF8B899C89AD8975
:10EFB000BE894A015B01E7E0B694A79497948794D1
:10EFC000EA95D1F7BECFE894C7F8DD24EE24FF24FC
:10EFD000F601EE0FFF1FEE0FFF1FE053FE4E4082C3
:10EFE000518262827382C9CFCF92DF92EF92FF92F9
:10EFF0000F931F93CF93DF93FC0181859285A385A7
:10F00000B4850196A11DB11D84179507A607B70702
:10F0100050F480E0DF91CF911F910F91FF90EF901E
:10F02000DF90CF90089587898031A9F5BB27A72F5E
:10F03000962F852FC388D488E588F6888C0D9D1D72
:10F04000AE1DBF1DE9016A017B018F014091D01304
:10F050005091D1136091D2137091D31384179507F7
:10F06000A607B70749F5F8018789803169F5B70127
:10F07000A601552766277727440F551F40535E4E3C
:10F08000FA0180819181B0E0A0E088839983AA830E
:10F09000BB8381E0BFCF803209F0BBCFC388D48867
:10F0A000E588F688DB01CA01C7E0B695A795979574
:10F0B0008795CA95D1F7C2CF40E0BC01CD010E942F
:10F0C00020778111D0CFA5CFB701A6014F77552763
:10F0D00066277727440F551F440F551F40535E4E38
:10F0E000FA0180819181A281B381BF70CECF4F920E
:10F0F0005F926F927F92AF92BF92CF92DF92EF9228
:10F10000FF920F931F93CF93DF9300D01F92CDB741
:10F11000DEB78C0149835A836B837C835901C12CF0
:10F12000D12C7601412C82E0582E612C712C498122
:10F130005A816B817C819E012F5F3F4FC8010E94E5
:10F14000F477882319F1F8018585A301920104C0A1
:10F15000220F331F441F551F8A95D2F7DA01C901C8
:10F16000C80ED91EEA1EFB1E49815A816B817C8123
:10F1700087898031F1F481E0483F5F4F6105710577
:10F18000B0F2F501C082D182E282F3820F900F903B
:10F190000F900F90DF91CF911F910F91FF90EF9003
:10F1A000DF90CF90BF90AF907F906F905F904F9027
:10F1B000089581E0483F5F4F6F4F7F4008F4B7CF1D
:10F1C000E0CF0F931F93CF93DF93FC012381222382
:10F1D00031F080E0DF91CF911F910F9108958B0165
:10F1E000EC01FB018789803139F582E08B831D8A30
:10F1F0001E8A1F8A188E808D918DB0E0A0E025E0D8
:10F20000880F991FAA1FBB1F2A95D1F7898B9A8B4C
:10F21000AB8BBC8B1A8F098F81E089831886198686
:10F220001A861B861C821D821E821F82188A1C86DB
:10F230001D861E861F86CECF803259F683E08B83D3
:10F24000428D538D648D758D4D8B5E8B6F8B788F5A
:10F250009E012F5E3F4FC8010E9477788111DACF5F
:10F26000B8CF3F924F925F926F927F928F929F9210
:10F27000AF92BF92CF92DF92EF92FF920F931F93C4
:10F28000CF93DF93CDB7DEB72C970FB6F894DEBFE0
:10F290000FBECDBF5C01DC0159968D909C90F401AE
:10F2A00081859285A385B4859C01AD012F5F3F4F79
:10F2B0004F4F5F4F29873A874B875C87D50114965C
:10F2C0004D905D906D907C901797411451046104AE
:10F2D000710409F459C0BFEF4B1A5B0A6B0A7B0A31
:10F2E000312C730162011D821E821F821886F40177
:10F2F00081859285A385B4852D813E814F81588576
:10F30000281739074A075B0708F056C089859A8590
:10F31000AB85BC858C159D05AE05BF0550F482E01C
:10F32000C82ED12CE12CF12C92E0492E512C612CCD
:10F33000712C9E012F5F3F4FB701A601C4010E94AF
:10F34000F4778823C9F189819A81AB81BC81892BAB
:10F350008A2B8B2B01F1260137019FEF491A590A9D
:10F36000690A790A2D813E814F8158852F5F3F4F71
:10F370004F4F5F4F2D833E834F8358873FEFC31A14
:10F38000D30AE30AF30AB3CF4080518062807380CE
:10F3900033243394A6CFC414D504E604F70411F73C
:10F3A0000FEF1FEF2FEF3FE0B701A601C4010E944E
:10F3B0006277782E81111AC0712C872D2C960FB68A
:10F3C000F894DEBF0FBECDBFDF91CF911F910F919B
:10F3D000FF90EF90DF90CF90BF90AF909F908F9075
:10F3E0007F906F905F904F903F900895F50144811A
:10F3F000558166817781411551056105710539F0A7
:10F4000097018601C4010E9462778823A9F2D50181
:10F410001496CD92DD92ED92FC921797332051F025
:10F42000D701C6010196A11DB11DF401808391830E
:10F43000A283B383F50185899689A789B08D892B2D
:10F440008A2B8B2B09F0B9CFC58AD68AE78AF08E32
:10F45000818180688183B1CFCF93DF93EC01462F08
:10F4600041706C857D858E859F850E9420778823DD
:10F4700051F0888920E2829FC001112480539E4E62
:10F48000DF91CF91089590E080E0FACFCF93DF93A2
:10F49000EC018B81882349F1898187FF22C061E0DB
:10F4A000CE010E942C7AFC01892BF9F08081853EE7
:10F4B000E1F08B81823040F489899A89AB89BC89DB
:10F4C000848F958FA68FB78F8D899E89938F828F1A
:10F4D0008D899E89AF89B88DB58BA48B89818F77F3
:10F4E0008983DF91CF910C94086A81E0888380E062
:10F4F000DF91CF9108958F929F92AF92BF92CF925A
:10F50000DF92EF92FF920F931F93CF93DF93EC0163
:10F510008B8181110EC080E0DF91CF911F910F91FF
:10F52000FF90EF90DF90CF90BF90AF909F908F9023
:10F53000089509891A892B893C890417150726071C
:10F54000370748F34A015B01823031F48886998697
:10F55000AA86BB8681E0E0CF81149104A104B104A6
:10F5600049F4188619861A861B861C821D821E8203
:10F570001F82F0CF088519852A853B85E98DFA8D94
:10F58000858590E00996B901A801415051096109AA
:10F590007109082E04C076956795579547950A948A
:10F5A000D2F775016401E1E0CE1AD108E108F10853
:10F5B00004C0F694E794D794C7948A95D2F7C416FA
:10F5C000D506E606F70620F0012B022B032B11F5DA
:10F5D0008D899E89AF89B88D8C839D83AE83BF83CF
:10F5E0008E010C5F1F4FC114D104E104F10409F432
:10F5F000ADCF4C815D816E817F819801898D9A8D1F
:10F600000E94F47791E0C91AD108E108F10881114C
:10F61000EACF81CFC41AD50AE60AF70AE1CF2F92C2
:10F620003F924F925F926F927F928F929F92AF9292
:10F63000BF92CF92DF92EF92FF920F931F93CF93DF
:10F64000DF9300D01F92CDB7DEB78C014B011A01BA
:10F65000DC0113968C911397813009F0CFC011967D
:10F660008C9181FFCBC082FDB5C06101D801189695
:10F670004D915D916D917C911B97C114D10409F45A
:10F680001BC159968D919C915A97FC0174802FEF64
:10F69000270D2A013B0139E07694679457944794EB
:10F6A0003A95D1F7722E74207A01F1E0FF227110A1
:10F6B00020C0E114F104E9F414964D915D916D912F
:10F6C0007C911797411551056105710509F09CC0A2
:10F6D00055968D919D910D90BC91A02D0097A105FF
:10F6E000B10509F0AAC0C8010E943179882309F444
:10F6F00085C0A12C82E0B82EAE18BF08CA14DB0466
:10F7000008F45601D80159964D915C915A97149678
:10F710008D919D910D90BC91A02D0297A109B109E9
:10F72000FA01258504C0880F991FAA1FBB1F2A95BF
:10F73000D2F74685578560897189840F951FA61F6A
:10F74000B71F9C01AD01270D311D411D511D290120
:10F750003A01A11432E0B30609F07DC08091D013C4
:10F760009091D113A091D213B091D313481659069A
:10F770006A067B0669F41092D8138FEF9FEFDC01C5
:10F780008093D0139093D113A093D213B093D3133B
:10F790008091D9139091DA13DC01ED91FC910288EC
:10F7A000F389E02D9401B301A2011995882331F169
:10F7B000F80180859185A285B3858A0D9B1DA11DC9
:10F7C000B11D80879187A287B3878A0C9B1CCA18BA
:10F7D000DB084CCFF801418952896389748980859F
:10F7E0009185A285B385481759076A077B0709F4F5
:10F7F0003CCFC8010E947B7A811137CF81E0D801CC
:10F800008C938FEF9FEF6EC09E012F5F3F4F0E9442
:10F81000F477882399F389819A81AB81BC81F801BF
:10F82000218D328DF9012789203169F4883FFFEF5E
:10F830009F07A105B10508F056CFF8018483958391
:10F84000A683B78356CF883F2FEF9207A2072FE0FA
:10F85000B20798F348CFE114F10431F5F80140857F
:10F8600051856285738581899289A389B4894817F6
:10F8700059076A077B07C0F00E94086A882309F4C9
:10F88000BDCF81E08093D8134092D0135092D11312
:10F890006092D2137092D313A501B401C7018053B3
:10F8A0009E4E0F94943784CF41E0C301B2010E9471
:10F8B00020778111F1CFA2CFF80181899289A389A4
:10F8C000B48984179507A607B70738F48181418B5F
:10F8D000528B638B748B80688183F801818183FDF7
:10F8E00018C0C1010F900F900F900F90DF91CF9132
:10F8F0001F910F91FF90EF90DF90CF90BF90AF904E
:10F900009F908F907F906F905F904F903F902F903F
:10F910000895C8010E94467A8111E3CF6FCF2F92DC
:10F920003F924F925F926F927F928F929F92AF928F
:10F93000BF92CF92DF92EF92FF920F931F93CF93DC
:10F94000DF93EC014B017A018B81811115C08FEFA0
:10F950009FEFDF91CF911F910F91FF90EF90DF907C
:10F96000CF90BF90AF909F908F907F906F905F905F
:10F970004F903F902F900895898180FFE8CF89892B
:10F980009A89AB89BC89488559856A857B85841BA2
:10F99000950BA60BB70BA70170E060E084179507E5
:10F9A000A607B70708F47C0167011E0124E0220EB8
:10F9B000311CC114D10409F4A9C0488559856A8550
:10F9C0007B855A0181E0B822898D9A8D2A013B01FD
:10F9D00029E076946794579447942A95D1F72B8120
:10F9E000FC01223081F5628D738D848D958D640DBF
:10F9F000751D861D971D00E012E00A191B09C0162F
:10FA0000D10608F486010115E2E01E0771F440906A
:10FA1000D0135090D1136090D2137090D31364150B
:10FA200075058605970509F04EC040E00E942077D5
:10FA3000882309F48CCFB50160537E4EA801C40120
:10FA40000F94943752C0148111501421A114B104A1
:10FA500071F411110CC0452B462B472B51F58D89A4
:10FA60009E89AF89B88D8C839D83AE83BF83E98DDA
:10FA7000FA8D4C805D806E807F8022E0421A5108B2
:10FA800061087108858504C0440C551C661C771CF0
:10FA90008A95D2F786859785A089B189480E591E27
:10FAA0006A1E7B1EC301B201610F711D811D911D74
:10FAB000A2CF4C815D816E817F8191010E94F4779C
:10FAC0008111D5CF44CFA091D913B091DA13ED9124
:10FAD000FC9111970088F189E02D9401AB01BC01E4
:10FAE000CD011995882309F432CF800E911E8885A7
:10FAF0009985AA85BB85800F911FA11DB11D88879F
:10FB00009987AA87BB87C01AD10A53CFC70121CFD3
:10FB1000CF93DF93EB01FC012381211104C080E02E
:10FB2000DF91CF9108952250223028F48FE288830C
:10FB3000198281E0F5CF60E00E942C7A009779F37A
:10FB4000DC0160E080E09EE22D91203299F0883067
:10FB500031F49E01260F311DF90190836F5F9E01E4
:10FB6000260F311DAD0141505109FA014081F901C3
:10FB700040836F5F8F5F8B3039F7FE01E60FF11D19
:10FB80001082D7CFCF93DF93EC01CB01E881F981CD
:10FB9000608171810E94887D28813981D901ED9130
:10FBA000FC91AA81BB818C919081992359F089366F
:10FBB000C8F4CF010196F901918380838C918F5F06
:10FBC0008C93EACF893670F48FE28083E881F981E3
:10FBD00080819181019691838083EA81FB8180817C
:10FBE0008F5F8083DF91CF9108950F931F93CF9301
:10FBF000DF9300D000D01F92CDB7DEB79C012F5FFE
:10FC00003F4F3F832E832FE2FC01208381E08D83D1
:10FC1000CE0106969A83898301979C838B8310E09B
:10FC20000BE180910A17181758F4109FB0011124A6
:10FC30006559784ECE0101960E94C27D1F5FF1CFBB
:10FC40008D818B3558F469E778E1CE0101960E94E9
:10FC5000C27D8E819F8101979F838E83EE81FF817C
:10FC6000108227960FB6F894DEBF0FBECDBFDF918E
:10FC7000CF911F910F910895CF93DF93EC010E94D4
:10FC8000467A1B82DF91CF910895109213098091DB
:10FC900015178F77809315170E940827882321F066
:10FCA00089E798E10C943C7E0895CF93C091151795
:10FCB000C2FF10C0C7FD0EC00E94082780FBC7F915
:10FCC000C0931517809115178F7E80648093151748
:10FCD000CF9108950E94457EF5CFCF93DF93809119
:10FCE00015178F7E8093151780913817882321F080
:10FCF00085E397E10E943C7E80911617909117173B
:10FD0000DC01ED91FC910190F081E02D45E360E094
:10FD1000199581110EC00E944A2E89EF94E20E942B
:10FD2000C7298091151784FF34C0DF91CF910C94BF
:10FD3000F769C0911617D091171761E0CE010E94A4
:10FD4000E1EF81110BC060E0CE010E94E1EF811173
:10FD500005C00E94DD2D85EE94E2E1CF64EF74E1F1
:10FD600085E397E10E94E178811105C00E94DD2DB5
:10FD700084ED94E2D4CF809115178061809315179C
:10FD80000E944A2E88EC94E20E94C7290E94D5DA8C
:10FD9000C8CF80915D08882339F061E088EB94E258
:10FDA000DF91CF910C94E2C2DF91CF91089540E0B2
:10FDB00050E0BA010C947B7A0F931F93CF93DF939B
:10FDC000CDB7DEB7EB970FB6F894DEBF0FBECDBF51
:10FDD0008091151700E010E084FF23C080E597E1D3
:10FDE0000E94D77E8BE1E0E5F7E1DE01919601907C
:10FDF0000D928A95E1F710E000E0BE016F5F7F4F42
:10FE0000CE0181960E9475EA18163CF4CE01019647
:10FE10000E94B476080F111DF0CFCE0181960E948A
:10FE2000AE22C801EB960FB6F894DEBF0FBECDBF71
:10FE3000DF91CF911F910F9108950F931F93CF934F
:10FE4000DF93CDB7DEB76B970FB6F894DEBF0FBE6A
:10FE5000CDBF8C0180E597E10E94D77E8BE1E0E584
:10FE6000F7E1DE01119601900D928A95E1F7B80154
:10FE7000CE0101960E94E776CE0101960E94AE2245
:10FE80006B960FB6F894DEBF0FBECDBFDF91CF915A
:10FE90001F910F9108952F923F924F925F926F9210
:10FEA0007F928F929F92AF92BF92CF92DF92EF920A
:10FEB000FF920F931F93CF93DF93CDB7DEB7C45458
:10FEC000D1090FB6F894DEBF0FBECDBF7C014B0148
:10FED0005A01222E19821C821C8E1F8E61157105FB
:10FEE00011F410E0B3C1DC0113968C918111F9CFAC
:10FEF000FA0180818B018F32D1F4DB0113968C9152
:10FF000013978250823060F059966D917C91CE01AA
:10FF10004C960E94E1788E01045E1F4F882309F3FE
:10FF2000C5015C010196F50120812F32D1F39E01BC
:10FF30002F5F3F4F6901290130E2332E2496CFAE67
:10FF400024972596DFAE25973E013CE1630E711C98
:10FF500022963FAE229721963FAE21973FAE3EAE0E
:10FF60003DAE3CAE3BAE3AAE39AE38AE3FAA95019F
:10FF700090E047E0D9018D91882361F18F3251F1F2
:10FF80008E3239F44A3009F4ACCF98E04AE09D0152
:10FF9000F1CFE4E9F4E22491222321F03196821397
:10FFA000FACF9FCF491708F49CCF813208F499CF3C
:10FFB0008F3709F496CF3FE9380F3A3108F420EE35
:10FFC000E7E3F0E0EC0FFD1FE90FF11D820F8083E6
:10FFD0009F5FDDCF8FA9803209F483CF5901D9010A
:10FFE0008C912F5F3F4F8F32C9F38823A9F00815FA
:10FFF000190519F0C8010E943C7E24969FAD2497F4
:020000021000EC
:1000000025968FAD25974C145D0411F4962D872D00
:100010008601C92ED82E9CCFF801818D928DD701F3
:100020005A969C938E935997C8010E94D77EC12CF3
:10003000F80180859185A285B385418952896389BC
:10004000748984179507A607B70708F053C025E001
:10005000B695A795979587952A95D1F7F82FFF70B4
:10006000DF2ED80113968C91823008F43ACF41E00C
:1000700050E0BE016E5B7F4FC8010E948F7C0197EC
:1000800009F02FCFF80180859185A285B3854F9621
:10009000A11DB11D80879187A287B387F0E2DF9E03
:1000A000B001112460537E4E6115710509F419CF1A
:1000B000DB018C91882341F0853E09F04DC0CC20B6
:1000C00029F0CC24C394B4CFC1100EC08091D013BA
:1000D0009091D113A091D213B091D313F7018487DB
:1000E0009587A687B787D08ADB018C918111E9CFEC
:1000F000CC24C394822D8274823409F0F2CECC20B9
:1001000009F4C7C0F701D08861E0C7010E942C7ACA
:10011000009709F4E6CE20E2DC011D922A95E9F76A
:100120002BE0FE01F796DC0101900D922A95E1F794
:1001300021E238E2FC01318B208B40E058E0578708
:100140004687338B228B318F208F578B468B0E94B3
:10015000086A81110AC0C5CE4BE050E0CE01C796B7
:100160000F948737892B09F063CF2D2D30E0F901EB
:10017000B5E0EE0FFF1FBA95E1F7DF01A053BE4EC9
:100180001B968C91817121F0822D827109F020C122
:10019000D70159968D919C915A974091D0135091C7
:1001A000D1136091D2137091D3131C964D935D932C
:1001B0006D937C931F975096DC925097E053FE4EC0
:1001C00084889588B12CA12C5401992488245596B3
:1001D0008D929D92AD92BC925897428D538D70E056
:1001E00060E0482959296A297B2955964D935D93EA
:1001F0006D937C935897A5E0220F331FAA95E1F7E2
:10020000D901A053BE4E1B962C91287109F0D2C083
:10021000848D958DA68DB78DF701818B928BA38BE5
:10022000B48B81E08383822D8F70F70181831482E8
:10023000158216821782108611861286138611E0A7
:1002400024FE04C0C7010E94C8EC182FCE014C96B2
:100250000E94AE22CE0101960E94AE22812FCC5B7D
:10026000DF4F0FB6F894DEBF0FBECDBFDF91CF9149
:100270001F910F91FF90EF90DF90CF90BF90AF90C4
:100280009F908F907F906F905F904F903F902F90B6
:100290000895D80113968C911397823009F421CEDA
:1002A00051968D919D910D90BC91A02D803E9F4FB8
:1002B000AF41B10508F015CEC8010E9431798823FD
:1002C00009F40FCE0E94086A882309F40ACED801E7
:1002D0005996ED91FC915A9714968D909D90AD9002
:1002E000BC901797B2E08B1A9108A108B1088585D8
:1002F00004C0880C991CAA1CBB1C8A95D2F7868561
:100300009785A089B189880E991EAA1EBB1E81E01F
:100310008093D8138092D0139092D113A092D213CD
:10032000B092D313E0EDF1E180E092E0DF019C01B7
:100330001D9221503040E1F7DD24D394D801599625
:10034000ED91FC918481D816C0F48091D9139091DD
:10035000DA13DC01ED91FC910288F389E02D20EDA8
:1003600031E1B501A4014D0D511D611D711D19959E
:10037000882309F4B6CDD394E1CF258580E092E0BF
:10038000A0E0B0E004C0880F991FAA1FBB1F2A95E8
:10039000D2F7F8014189528963897489840F951FC6
:1003A000A61FB71F818B928BA38BB48B80ED91E13D
:1003B000D12CB1CE203161F497012F5E3F4F0E94C6
:1003C0007778882329F084E0D70113968C932BCF7C
:1003D000D70113961C9285CD1F93CF93DF93CDB792
:1003E000DEB76D970FB6F894DEBF0FBECDBF1D8E82
:1003F0001C8EAC01BE01645E7F4F80E00E945CED0C
:1004000010E00097A9F019821C826C8D7D8D21E08F
:10041000AC01CE0101960E944B7F182F882321F05A
:10042000CE0101960E943C7ECE0101960E94AE2232
:10043000812F6D960FB6F894DEBF0FBECDBFDF9152
:10044000CF911F910895EF92FF921F93CF93DF9367
:1004500000D000D000D01F92CDB7DEB780910B172F
:10046000882309F447C08091151784FF0E946D7E90
:100470008091151784FF3CC00E949C22811138C0D6
:1004800080910B1790E08F969F938F9383E096E275
:100490009F938F93CE0101967C019F938F930F942E
:1004A0003C2D809115170F900F900F900F900F908B
:1004B0000F9084FF1DC0C7010E94EC81182F882374
:1004C000B9F00E94F769C7010E94567680910B1718
:1004D0008F5F80930B17812F2A960FB6F894DEBF9B
:1004E0000FBECDBFDF91CF911F91FF90EF90089588
:1004F00010920B1710E0EFCFCF9321E04EEB52E0BC
:1005000065E377E18AE197E10E944B7FC82F88235A
:1005100021F08AE197E10E943C7E8C2FCF910895D3
:10052000682F70E090E080E00C94F0E98F929F9249
:10053000AF92BF92CF92DF92EF92FF92CF936B0177
:100540007C01B42E20E030E0A9010F94A52D87FF97
:1005500007C08DE20E94B629F7FAF094F7F8F094FC
:10056000C0E060E070E080E09FE3CB1541F02DEC4F
:100570003CEC4CEC5DE30F940B2ECF5FF6CFA70164
:1005800096010F946D346B017C010F94E0354B01A3
:100590005C010E94F0E9CC2371F1C501B4010F9414
:1005A000AA2D9B01AC01C701B6010F946C346B01FD
:1005B0007C018EE20E94B629C150E8F020E030E0D4
:1005C00040E251E4C701B6010F940B2E6B017C0190
:1005D0000F94E0354B015C010E94F0E9C501B401C4
:1005E0000F94AA2D9B01AC01C701B6010F946C3486
:1005F0006B017C01E1CFCF91FF90EF90DF90CF9026
:10060000BF90AF909F908F900895EF92FF920F93BD
:100610001F93CF937B018A01C2E48F3F09F0C4E5A9
:1006200080E20E94B6298C2F0E94B6298AE30E949C
:10063000B629F701608171818281938142E00E9435
:10064000968284E894E20E94C729F8016081718152
:100650008281938142E00E94968262E070E080E0B5
:1006600090E0CF911F910F91FF90EF900C946872E2
:100670001F93CF93DF9300D000D01F921F92CDB76E
:10068000DEB7182F60913D1470913E14072E000CB8
:10069000880B990B0F94AC2D6D837E838F83988785
:1006A0008091391490913A14A0913B14B0913C146C
:1006B00089839A83AB83BC83AE014B5F5F4FBE01DE
:1006C0006F5F7F4F80E80E940583609126147091D0
:1006D0002714072E000C880B990B0F94AC2D6D83FB
:1006E0007E838F8398878091221490912314A09108
:1006F0002414B091251489839A83AB83BC83AE0103
:100700004B5F5F4FBE016F5F7F4F8FEF0E9405838E
:10071000609128141F3F39F087E11802F00111247D
:10072000EB5CFB4E628570E08CE894E20E949231B3
:100730006091281470E087E894E20E949231289634
:100740000FB6F894DEBF0FBECDBFDF91CF911F91E2
:1007500008952F923F924F925F926F927F928F9265
:100760009F92AF92BF92CF92DF92EF92FF920F9340
:100770001F93CF93DF93CDB7DEB765970FB6F8948D
:10078000DEBF0FBECDBF8A8B6B8B20918607298B76
:100790001092860781E0809322021A821B821C82BB
:1007A0001D8219861A861B861C861D863CE33E87A1
:1007B0004CE14F8756E4588B312C212C80E88C8BF0
:1007C0009FEB9D8B1982A1E0A887812C912C54016D
:1007D00060913D1470913E14072E000C880B990B0C
:1007E0000F94AC2D7B018C01232D322D4C895D891A
:1007F0000F94A52D8823B9F02091391430913A1423
:1008000040913B1450913C14BB89B701C801B11110
:10081000E4C00F94A52D881F8827881F89833E2C4C
:100820002F2C0C8B1D8B0E949B726B017C01DC01B9
:10083000CB0129853A854B855C85821B930BA40BE4
:10084000B50BB7FD2EC0D701C60188519C4FAF4FE5
:10085000BF4F89879A87AB87BC878A890E94388374
:1008600080E994E20E94C72981149104A104B10493
:1008700009F4E3C0C501B4016053784F8F4F9F4F17
:100880006C197D098E099F0928EE33E040E050E0A5
:100890000F94E933CA01B9010E945AEA8AE00E9422
:1008A000B62980E00E9450370E949B7260935C14CE
:1008B00070935D1480935E1490935F14909139143B
:1008C0009E83A0913A14AF8300913B1410913C1485
:1008D000292F3A2FA801632D722D8C899D890F94A1
:1008E0006C342B013C0120E030E0A9010F94CD369F
:1008F00087FF04C077FA709477F87094811491049C
:10090000A104B10409F09DC020E030E040E85FE3BD
:10091000C301B2010F94A52D87FF10C0B885812CAB
:10092000912C5401BB2331F08AE9882E82E0982E65
:10093000A12CB12C8C0C9D1CAE1CBF1C2981222328
:10094000A9F18A819B81AC81BD81892B8A2B8B2B5C
:1009500061F0D701C6012A813B814C815D81821BF8
:10096000930BA40BB50BB7FD21C02E813F81A801CD
:100970006D857E858F8598890F946C3420E030E0FA
:1009800040EC5FE30F94A52D87FD2BC0D701C60176
:10099000805A9541AF4FBF4F8A839B83AC83BD8301
:1009A0009E819D87AF81AE870F87188B8091220231
:1009B0008823B9F081149104A104B10461F0B0ED71
:1009C000CB1AB7E0DB0AE108F108C818D908EA0831
:1009D000FB08F7FE06C01886FBCE0F94A52D87FFF7
:1009E00026C0209122022983222321F01092220284
:1009F0000E942CEC298920938607898165960FB681
:100A0000F894DEBF0FBECDBFDF91CF911F910F9144
:100A1000FF90EF90DF90CF90BF90AF909F908F901E
:100A20007F906F905F904F903F902F9008953E2C55
:100A30002F2C0C8B1D8B1982F6CE8FE30E94B629CA
:100A40002DCF20E030E040E450E4C301B2010F9428
:100A5000CD3618160CF072CF460157016FCF0F93A9
:100A60001F93CF93DF93809117028F3708F49DC0B7
:100A70008F5790913F149093BA09992309F493C02A
:100A80002C9A209128142093B909909102012111E8
:100A900090959072909300018F5F809317028091E0
:100AA000B80991E089278093B80980911602980FC0
:100AB00085300CF090E0823009F4D2C00CF082C096
:100AC000882309F497C0813009F4BEC090931602C0
:100AD00080918507882309F454C0809114028E5FA9
:100AE0008F778093140281114CC08CB185FB8827CD
:100AF00080F9C82F80E0D82F8091030181FDC2606A
:100B00004B99C4600091B5091091B6090C171D07E7
:100B1000C1F10C2700FF08C08BE794E20E94C729AF
:100B20008C2F81700E94A21F01FF0AC082E794E20D
:100B30000E94C729CE019695879581700E94A21FB9
:100B400002FF0CC089E694E20E94C729CE01969567
:100B500087959695879581700E94A21F86E694E2FC
:100B60000E94C7296091B40970E08DE00E9430F1C5
:100B70008091B40980958093B409D093B609C0934D
:100B8000B5090E940CBB8091B60A9091B70A0097F4
:100B900029F001979093B70A8093B60ADF91CF911D
:100BA0001F910F9108952C986CCF9091BA098917D5
:100BB00008F02C989091B909891708F46DCF90919D
:100BC000020167CF843009F463C00CF45CC0853047
:100BD00009F07CCF2091B709211102C08093B70999
:100BE0008091B70981508093B709882309F46ECFAB
:100BF00095E06CCF809115028F5F80311CF480935B
:100C0000150264CF109215028091B309811113C0AF
:100C100020913514309136143093381420933714C2
:100C200020911E1430911F1430932114209320140E
:100C300081E08093B309109236141092351410920B
:100C40001F1410921E1442CF88E080937B0085E42D
:100C500080937C0080917A00806480937A0036CF04
:100C600080917A0086FD27C04091780050917900EC
:100C70002091351430913614240F351F30933614DB
:100C80002093351423CF88E080937B0086E4E0CF67
:100C900080917A0086FD11C04091780050917900D2
:100CA00020911E1430911F14240F351F30931F14F0
:100CB00020931E140BCF92E009CF94E007CF0F933F
:100CC0000FB70F9300916E000D7F00936E00789424
:100CD0000F930BB70F930CB70F921F922F933F9365
:100CE0004F935F936F937F938F939F93AF93BF9334
:100CF000EF93FF9311240E942F85FF91EF91BF91F5
:100D0000AF919F918F917F916F915F914F913F91A3
:100D10002F911F900F900CBF0F910BBF0F9102608E
:100D2000F89400936E000F910FBF0F9118952091CA
:100D30003D1430913E14263531053CF420912614A3
:100D4000309127142630310524F0882349F00C9483
:100D50002E27662329F081E00E94B2C80C942CEC67
:100D60000895CF93DF9310928607E5E3F4E11186AF
:100D700010861092810710928207109283071092BA
:100D8000840712862C98CEE1D4E1198618860E9439
:100D900059231A8680910201807280930001DF91AD
:100DA000CF910895CF92DF92EF92FF920F931F930E
:100DB000CF93DF93CDB7DEB72C970FB6F894DEBF95
:100DC0000FBECDBF182F6B017A0180915D08833073
:100DD00090F00E94DD2DC6010E94C7298EE393E2A8
:100DE0000E94C7291F3F89F58AE393E20E94C72921
:100DF0008AE00E94B6290E94B186A8958091880950
:100E0000811155C081E08093880982E080935D085C
:100E10000E94B18605E10150409A49F169E170E014
:100E200080E090E00E946872A895409868E270E0C7
:100E300080E090E00E946872A89568E270E080E02F
:100E400090E00E946872A895E6CF17FDD1CF88E3A5
:100E500093E20E94C729612F012E000C770B880BAB
:100E6000990B0E945AEA8AE00E94B629C1CF87E016
:100E70000E945AD8811111C08CE0EFE8F2E0DE0147
:100E8000119601900D928A95E1F7BE016F5F7F4F39
:100E900080E00E9457BE0E94F3AE61E373E21F3F01
:100EA00011F065E373E240E0C7010E9448352C96DB
:100EB0000FB6F894DEBF0FBECDBFDF91CF911F916B
:100EC0000F91FF90EF90DF90CF9008952F923F9277
:100ED0004F925F926F927F928F929F92AF92BF924A
:100EE000CF92DF92EF92FF920F931F93CF93DF93F6
:100EF00000D000D01F92CDB7DEB79F838E831B0139
:100F00006A01298381E090E02F3F11F090E080E0BA
:100F100025E0289FF001299FF00D1124EC5CF64F8D
:100F20008481882309F4A7C0EE81FF811482158291
:100F3000168217821086EE81FF8184818230B9F09B
:100F4000833009F41CC1813009F07CC025813681D1
:100F500047815085F10160817181828193810F9475
:100F6000A52D87FD6FC082E0EE81FF818483809193
:100F700013029701FF0C440B550B2A833B834C83D0
:100F80005D83882389F1398131112EC08091B50AA2
:100F9000882339F1F101C080D180E280F380EE81B5
:100FA000FF8185809680A780B0846A817B818C8157
:100FB0009D810F94AC2D2B013C0120E030E040E8F6
:100FC0005EE30F940B2E9B01AC01C501B4010F949D
:100FD0006C349B01AC01C701B6010F94CD3687FD7F
:100FE00075C080E8809312020E949B726B017C01A5
:100FF0006A817B818C819D810F94AC2D9B01AC011A
:10100000EE81FF8165817681878190850F946C34B4
:101010009B01AC01F10160817181828193810F9408
:10102000CD3687FD9EC09801A8EEB3E00F9435340D
:10103000C60ED71EE81EF91EEE81FF81C082D18246
:10104000E282F38227960FB6F894DEBF0FBECDBFC3
:10105000DF91CF911F910F91FF90EF90DF90CF9094
:10106000BF90AF909F908F907F906F905F904F90C8
:101070003F902F900895F60180809180A280B380E8
:10108000A5019401EE81FF8165817681878190853C
:101090000F94A52D882309F44ECFEE81FF81858220
:1010A0009682A782B086BB24B39420E030E0A901E9
:1010B000F60160817181828193810F94CD3618167B
:1010C0000CF0B12CEE81FF81B48235CF23E830ECF7
:1010D0004AEA5EE3C301B2010F940B2E9B01AC01FF
:1010E000C501B4010F946C349B01AC01C701B6017A
:1010F0000F94CD3687FD02C080E674CF20E030E04B
:1011000040E05FE3C301B2010F940B2E9B01AC01E1
:10111000C501B4010F946C349B01AC01C701B60149
:101120000F94CD3687FD02C080E45CCF2DEC3CEC03
:101130004CE45FE3C301B2010F940B2E9B01AC01A1
:10114000C501B4010F946C349B01AC01C701B60119
:101150000F94CD3687FD02C080E244CF1092120278
:1011600043CFEE81FF8180819181A281B381C81A32
:10117000D90AEA0AFB0AF7FC65CF83E0848346E4D8
:1011800054E266E574E2898127960FB6F894DEBFD3
:101190000FBECDBFDF91CF911F910F91FF90EF90C8
:1011A000DF90CF90BF90AF909F908F907F906F9087
:1011B0005F904F903F902F900C94D286CF93DF9307
:1011C000A89580913714909138140E94ABF26093E7
:1011D000391470933A1480933B1490933C1480918B
:1011E0002014909121140E94006B6093221470933C
:1011F00023148093241490932514C0913714D09114
:10120000381480911C0290911D02C817D90738F438
:1012100048E054E265E174E280E00E94D286809169
:101220003D1490913E141816190674F480911A0218
:1012300090911B028C179D0738F447E254E264E357
:1012400074E280E00E94D2862091BC093091BD09F1
:1012500080912014909121148217930738F448E06C
:1012600054E265E174E28FEF0E94D28680912614E9
:101270009091271418161906A4F4209118023091A1
:10128000190280912014909121142817390748F4ED
:1012900047E254E264E374E28FEFDF91CF910C9464
:1012A000D286DF91CF9108952F923F924F925F9215
:1012B0006F927F928F929F92AF92BF92CF92DF9266
:1012C000EF92FF920F931F93CF93DF93CDB7DEB7CB
:1012D00060970FB6F894DEBF0FBECDBF80915D085A
:1012E00081111AC0A89560960FB6F894DEBF0FBEA4
:1012F000CDBFDF91CF911F910F91FF90EF90DF90C5
:10130000CF90BF90AF909F908F907F906F905F90A5
:101310004F903F902F9008958091B2098111E3CFB3
:1013200081E08093B20980917E0781110BC080918A
:101330007D07811120C18091B30981110AC01092EB
:10134000B209D1CF41E070E060E08AE793E20E9409
:1013500048350E94DE881092B3090E949B724B01AF
:101360005C016091200270912102072E000C880B15
:10137000990B0F94AC2D9B01AC01609139147091C5
:101380003A1480913B1490913C140F94CD3618166A
:101390000CF44AC280913809882309F42AC260916A
:1013A0003D1470913E14072E000C880B990B0F947E
:1013B000AC2D69837A838B839C833AE0E32EF12CF6
:1013C0000CE310E020E0AE014F5F5F4F69E374E192
:1013D00082E195E10E946687C0903914D0903A145A
:1013E000E0903B14F0903C1460911E0270911F023B
:1013F000072E000C880B990B0F94AC2D9B01AC01B0
:10140000C701B6010F94CD3618160CF4C0C060E0C9
:1014100060933F148091810790918207A091830788
:10142000B09184070097A105B10569F1A501940168
:10143000281B390B4A0B5B0BDA01C901B7FD23C02E
:10144000C701B6010F94D93520917F0730918007ED
:10145000621773070CF45FC320913D1430913E1462
:101460002115310541F06E5F7F4F2450310962171D
:1014700073070CF474C310928107109282071092C4
:1014800083071092840720E030E046E153E4609146
:1014900022147091231480912414909125140F9498
:1014A000CD3618160CF417C38091790790917A07FE
:1014B000A0917B07B0917C070097A105B10509F4C5
:1014C000C9C1A5019401281B390B4A0B5B0BDA013A
:1014D000C901B7FDBFC1609122147091231480919E
:1014E0002414909125140F94D935209177073091C9
:1014F0007807621773070CF4A6C1E0912614F091E7
:101500002714309751F0AB014E5F5F4F9F0124507D
:101510003109421753070CF40FC310927907109248
:101520007A0710927B0710927C0720913D092223B5
:1015300009F4D9C2BF01FF0F880B990B0F94AC2D92
:1015400069837A838B839C8392E0E92EF12C02E3FA
:1015500010E02FEFAE014F5F5F4F62E274E18BE16D
:1015600095E10E94668780913D09882309F477C13F
:1015700010922814E4CE10927D070E94EDB30E94D1
:10158000F3AE8EEF0E949BB90E9427BAD4CE609131
:10159000200270912102072E000C880B990B0F94EA
:1015A000AC2D9B01AC01C701B6010F94A52D87FF9F
:1015B0002ECF60913D1470913E146115710509F4B0
:1015C000B2C2072E000C880B990B0F94AC2DA7010B
:1015D00096010F946C342B013C0120E030E040E296
:1015E00051EC0F94A52D87FD9EC280913809811181
:1015F0009AC220E030E040E251E4C301B2010F940E
:10160000CD3618160CF4C3C28091B109882391F02D
:101610001092AD091092AE091092AF091092B00964
:101620001092A9091092AA091092AB091092AC0964
:101630001092B1098091A9099091AA09A091AB09D2
:10164000B091AC098D839E83AF83B887A7019601C3
:1016500060919D0970919E0980919F099091A009C8
:101660000F946C34209148143091491440914A14DD
:1016700050914B140F940B2E2D813E814F81588534
:101680000F946C3420ED3CEC4CE45DE30F940B2E96
:101690002D813E814F8158850F946D346D837E83FB
:1016A0008F8398876093A9097093AA098093AB09E7
:1016B0009093AC0920914414309145144091461404
:1016C0005091471429873A874B875C872091AD0951
:1016D0003091AE094091AF095091B009C301B201F8
:1016E0000F946D34162F072F382E292E20E030E06E
:1016F000A9010F94A52D87FD4EC229853A854B85FA
:101700005C8560E070E08FE793E40F9467356D8748
:101710007E878F87988B212F302F432D522D0F944A
:10172000A52D87FF04C01D850E853F842888812F45
:10173000902FA32DB22D8093AD099093AE09A09365
:10174000AF09B093B00920914014309141144091F9
:10175000421450914314C301B2010F940B2E2B017C
:101760003C014092A1095092A2096092A309709293
:10177000A409212F302F432D522D69857A858B8521
:101780009C850F940B2E9B01AC012093A5093093EF
:10179000A6094093A7095093A809C301B2010F9469
:1017A0006D342D813E814F8158850F946D3420E03A
:1017B00030E0A9010F946D342B013C0120E030E0B2
:1017C000A9010F94A52D87FDB1C120E030E04FE7BE
:1017D00053E4C301B2010F94CD3618166CF56FE7D0
:1017E000C0929D09D0929E09E0929F09F092A009B3
:1017F0000FCE8091340990913509A0913609B091AE
:1018000037090097A105B10509F4C9CDA5019401D7
:10181000281B390B4A0B5B0BDA01C901B7FDBFCDA1
:1018200081E080933809BBCD48E054E265E174E281
:1018300080E00E94D286AECDC301B2010F94D935AB
:1018400075956795CDCF4CE553E26BE673E28FEF6C
:101850000E94D286E0912614F091271466CEC090A3
:101860002214D0902314E0902414F090251420E04A
:1018700030E040EA50E4C701B6010F94CD3687FD51
:101880000AC020E030E046E153E4C701B6010F94FE
:10189000A52D181624F460E06093281450CD6091B3
:1018A0002614709127146115710509F441C1072EA2
:1018B000000C880B990B0F94AC2DA70196010F9487
:1018C0006C344B015C0120E030E040E251EC0F94BD
:1018D000A52D87FD2DC120E030E040E251E4C50197
:1018E000B4010F94CD3618160CF44CC180912D1410
:1018F00090912E14A0912F14B09130148D839E835B
:10190000AF83B88780911102882391F010929909D2
:1019100010929A0910929B0910929C0910929509B5
:10192000109296091092970910929809109211023C
:101930002091990930919A0940919B0950919C09F5
:10194000C501B4010F946D34562E672E782E492EA2
:1019500020E030E0A9010F94A52D87FD21C12D8144
:101960003E814F81588560E070E08FE793E40F94EB
:101970006735162F072F382E292E252D362D472D6A
:10198000542D0F94A52D87FF04C0512E602E732C6B
:10199000422C852D962DA72DB42D809399099093D7
:1019A0009A09A0939B09B0939C0920912914309126
:1019B0002A1440912B1450912C14C501B4010F949A
:1019C0000B2E4B015C0180928D0990928E09A092A2
:1019D0008F09B0929009252D362D472D542D6D81FC
:1019E0007E818F8198850F940B2E6D837E838F83EC
:1019F00098876093910970939209809393099093CB
:101A000094094090950950909609609097097090BC
:101A10009809A70196016091890970918A098091BE
:101A20008B0990918C090F946C3420913114309172
:101A3000321440913314509134140F940B2EA3019F
:101A400092010F946C3420ED3CEC4CE45DE30F9478
:101A50000B2EA30192010F946D342B013C01409297
:101A60009509509296096092970970929809C092D0
:101A70008909D0928A09E0928B09F0928C092D8114
:101A80003E814F815885C501B4010F946D34A30187
:101A900092010F946D3420E030E0A9010F946D3471
:101AA0006B017C0120E030E0A9010F94A52D87FD9A
:101AB000F2CE20E030E04FE753E4C701B6010F94C7
:101AC000CD3618160CF461C0C701B6010F94D93594
:101AD00075956795E1CE48E054E265E174E28FEFD9
:101AE0000E94D286E1CC4091390950913A09609127
:101AF0003B0970913C09411551056105710509F4D7
:101B000019CD841A950AA60AB70AB7FC13CD21E0AD
:101B100020933D090FCD4CE553E26BE673E280E084
:101B20000E94D286B0CC81E08093B10960E058CEAB
:101B300081E080931102AFCE5093780740937707EE
:101B40000E949B72605E70448D4F9F4F6093790737
:101B500070937A0780937B0790937C077BCE70937A
:101B6000800760937F070E949B72605A75418F4F78
:101B70009F4F6093810770938207809383079093B0
:101B8000840781CC81E0809311026FE785CE81E0EC
:101B90008093B10924CE10E000E0312C212CC7CD78
:101BA000512C612C712C412CF4CE2F923F924F92EC
:101BB0005F926F927F928F929F92AF92BF92CF92DD
:101BC000DF92EF92FF920F931F93CF93DF93CDB7E6
:101BD000DEB7CC55D1090FB6F894DEBF0FBECDBF2E
:101BE0007C01162F21964FAF219727962FAF27976D
:101BF0000E949B726F87788B898B9A8B1F3F09F0AD
:101C00003FC024EB30E03A8329830E9484EE1F3FDB
